:100000000C944B070C947C070C947C070C947C0795
:100010000C947C070C947C070C947C070C947C0754
:100020000C947C070C947C070C947C070C947C0744
:100030000C947C070C94878C0C947C070C947C07A4
:100040000C947C070C94878A0C947C070C947C0796
:100050000C947C070C947C070C947C070C94B3895B
:100060000C947C070C940A820C94E0810C947C071D
:100070000C947C070C947C070C947C070C947C07F4
:100080000C94598A0C947C070C947C070C947C0784
:100090000C947C070C947C070C947C070C942F8F99
:1000A0000C947C070C947C070C942B8A0C947C0792
:1000B0000C947C070C947C070C947C070C94FD89B1
:1000C0000C947C070C947C070C947C070C947C07A4
:1000D0000C947C070C947C070C94AA810C9480816E
:1000E0000C947C070C9460790C94F3070C946708CB
:1000F0000C944B770C945B1A0C9441170C94AB77CF
:100100000C9483070C94C0780C94B3780C94540826
:100110000C94A3070C948B960C94E5780C948B1696
:100120000C9419090C94371E0C94ED080C94B280B1
:100130000C9438180C94D2780C944D790C94EA787D
:100140000C940E1C0C9470160C94CB1A0C94D818AA
:100150000C94AF780C94ED770C94C4780C94BA7826
:100160000C9409080C94D8780C9467290C949D770A
:100170000C9463080C9419180C944A770C947D1A0B
:100180000C94BE180C94029C0C9451190C944C774E
:100190000C940C1E0C947A770C9457090C94FA1654
:1001A0000C9490200C94CA780C9444080C947E080B
:1001B0000C943A780C9477080C94621E0C9463109B
:1001C0000C9467790C945F080C9409170C94971C95
:1001D0000C94041A0C94A5780C94B5160C9452083F
:1001E0000C94AB780C9457080C9410160C94DC1DEE
:1001F0000C945A760C94B61A0C944D770C94B778EC
:100200000C9442230C94E0780C94DC780C94661CDB
:100210000C9400700C947B090C944D090C94A31061
:100220000C94E08E0C9489770C943A190C943E79D6
:100230000C9449770C942E080C94AA9B0C944808B3
:100240000C9423080C9462180C94E6780C942C1CE3
:100250000C94CE780C94F9180C940D080C949479A5
:100260004E414E494E495459494E46CDCCCC3D0A9B
:10027000D7233C17B7D13877CC2B329595E6241F7E
:10028000B14F0A000020410000C84200401C462037
:10029000BCBE4CCA1B0E5AAEC59D7400407A10F30A
:1002A0005A00A0724E18090010A5D4E80000E876A4
:1002B00048170000E40B54020000CA9A3B000000FB
:1002C000E1F505000080969800000040420F000014
:1002D00000A08601000000102700000000E80300D5
:1002E0000000006400000000000A0000000000019F
:1002F00000000000002C76D888DC674F0823DFC19F
:10030000DFAE59E1B1B796E5E3E453C63AE6519959
:100310007696E8E6C28426EB898C9B62ED407C6F82
:10032000FCEFBC9C9F40F2BAA56FA5F490055A2A39
:10033000F75C936B6CF9676DC11BFCE0E40D47FE45
:10034000F520E6B500D0ED902E030094357705003A
:1003500080841E080000204E0A000000C80C3333C1
:1003600033330F986E12831141EF8D2114893BE6D0
:100370005516CFFEE6DB18D1844B381BF77C1D9059
:100380001DA4BBE424203284725E228100C9F124C2
:10039000ECA1E53D27436F6E74656E742D54797042
:1003A000653A20746578742F68746D6C0D0A0D0AB7
:1003B0003C68313E45504943204641494C3C2F68FA
:1003C000313E00485454502F312E302034303020EC
:1003D00042616420526571756573740D0A00416352
:1003E000636573732D436F6E74726F6C2D416C6C0B
:1003F0006F772D4F726967696E3A202A0D0A436F35
:100400006E74656E742D547970653A200053657270
:100410007665723A205765626475696E6F2F312E6A
:10042000370D0A00485454502F312E3020323030CE
:10043000204F4B0D0A00436F6E6E656374696F6EDB
:100440003A20636C6F73650D0A436F6E74656E744A
:100450002D547970653A206170706C6963617469BC
:100460006F6E2F782D7777772D666F726D2D757281
:100470006C656E636F64656400506F7374206661B1
:10048000696C65640055706C6F6164204661696CCD
:1004900065643A2000234E6F2073656E736F72207F
:1004A000666F722074656D7020262068756D6964B2
:1004B00069747921004E6F2053656E736F7221004D
:1004C00020666F722074656D7020262068756D69D6
:1004D0006469747921002353656E736F72204572CD
:1004E000726F72200053656E736F72204572726F67
:1004F0007221002357726F6E672073656E736F727F
:1005000020666F722074656D7020262068756D6995
:1005100064697479210057726F6E672053656E733A
:100520006F7221004320483D00543D0020202020D0
:1005300020202020202020202020202000202020DB
:1005400020202020202020202020202000202020CB
:100550002020202020202020202020200054696DF1
:10056000657374616D702075706C6F616420666175
:10057000696C65640053657474696E6720636C6FA1
:10058000636B2074696D6500495020616464726515
:1005900073733A2000416E676C654000496E766166
:1005A0006C696420534D207374657073207065729C
:1005B00020616E676C653D00534D207374657073E8
:1005C0002070657220616E676C653D003C703E5422
:1005D000696D653A20003C2F68333E0A003C627228
:1005E0003E4254206E616D653D003C62723E50613A
:1005F00074683D003C68333E53797374656D3A20EE
:1006000056657273696F6E3D00506172616D6574FD
:1006100065727320726573657420646F6E65210066
:100620002F6F652F736D6C69676874706F2F7333EC
:100630002F00616E676C6520646972656374696F11
:100640006E3A200043757272656E7420534D2069B6
:1006500073202300534D3A5461626C6520737465B6
:1006600070732070657220616E676C653D00534D3C
:100670003A506F6C6172697A657220737465707339
:100680002070657220616E676C653D00234448549C
:100690003D00236E65743D424C4500236E65743DFC
:1006A0005769466900236E65743D425400236674A1
:1006B0007020757365726E616D653A003A0023486B
:1006C0006F73742073657276657220495020616E75
:1006D0006420506F72743A002354696D652073650D
:1006E000727665722049503A002352656C61792018
:1006F000646576696365733A002352656C6179209D
:10070000737461747573206C6162656C733A200058
:100710002352656C6179207374617465733A0023A8
:1007200052656C61792070696E733A00234E6F2EAA
:10073000206F662072656C6179733D0046696E6456
:10074000696E672057694669204950004E45543DFF
:10075000426C7565746F6F7468204C45004E45544B
:100760003D426C7565746F6F7468004E45543D571B
:10077000694669005344206F70656E206661696C3C
:10078000004E6577206461746120636F6C6C6563F3
:1007900074696F6E2073746172746564004375725E
:1007A00072656E742073657474696E67733A005372
:1007B000797374656D2072657365742061742000AF
:1007C00023445320546865726D6F6D6574657220A3
:1007D00063616C6962726174656420666F72202364
:1007E00000496E76616C696420616E676C65206695
:1007F0006F722000207374657073207065722061C1
:100800006E676C653D00207374657073207065724F
:1008100020616E676C653D005461626C65205365B4
:1008200074203000235475726E7461626C652053BD
:100830006574203000506F6C6172697A6572205364
:10084000657420300023506F6C6172697A65722084
:100850005365742030005461626C652053657420C8
:100860003000235475726E7461626C652053657438
:10087000203000506F6C6172697A65722053657424
:1008800020300023506F6C6172697A657220536565
:1008900074203000576946692049503A004C6F6710
:1008A000676572204E616D653A20005265626F6F18
:1008B00074696E672E2E2E00536572766572205015
:1008C0006F727420757064617465640053504F5288
:1008D000543D00495020757064617465640053494B
:1008E000503D002354696D65205365727665722012
:1008F0004950207570646174656400545349503DDB
:10090000004352454C41590074696D6520696E740D
:10091000657276616C3D0054494D455354414D50CC
:100920003D0054494D455354414D50002377656275
:1009300073657276657220626567696E73005461D3
:10094000626C6520536574203000235475726E7498
:1009500061626C6520536574203000506F6C617269
:10096000697A65722053657420300023506F6C6182
:1009700072697A65722053657420300053797374FC
:10098000656D207265737461727465642100205313
:10099000797374656D207265737461727465642116
:1009A0000023436F6D6D616E644000546573742065
:1009B0004C616D70732F46616E7300444843502044
:1009C000537563636573730044484350204641493F
:1009D0004C45440053657474696E672044657669BC
:1009E0006365204950202E2E2E006572726F722092
:1009F0006F70656E696E672066696C653A20004CA1
:100A0000616D70204F74686572002354696D6520B4
:100A10002020202020446174652020202020536560
:100A2000636F6E647320506F6C6172697A657220B7
:100A30005461626C652054286F4329204828252979
:100A4000202000646F6E652100696E69742E206439
:100A50006F6E652E00534420696E69742E206661A6
:100A6000696C65642100696E69742E206661696C29
:100A7000656421002323204F452057656C636F6D0B
:100A80006520232300496E697469616C697A696E17
:100A90006720534420636172642E2E2E0075706CA3
:100AA0006F616420627920465450206661696C65EC
:100AB00064210075706C6F61642062792046545027
:100AC000204F4B210053797374656D2073746172EC
:100AD00074696E672E2E2E007C3C3E5E2B3D3F2FB0
:100AE0005B5D3B2C2A225C003C703E4C616D7020AB
:100AF000616E64204F7468657220537461747573FD
:100B0000EFBC9A3C2F703E003C21646F6374797097
:100B1000652068746D6C3E3C68746D6C3E3C686525
:100B200061643E3C6D6574612063686172736574D5
:100B30003D227574662D38223E3C7469746C653EA6
:100B40004F6E6C696E65206578706572696D656E53
:100B500074202D20506F6C6172697A6174696F6EB8
:100B60002065666665637473206F66206C696768CC
:100B7000743C2F7469746C653E3C2F686561643EFB
:100B80003C626F64793E3C68313E4F6E6C696E65C5
:100B9000206578706572696D656E74202D20506FC8
:100BA0006C6172697A6174696F6E206566666563EF
:100BB0007473206F66206C696768743C2F68313EDF
:100BC000003C68343E436F707972696768742843EB
:100BD00029323032302D323032322E50726F662E42
:100BE000205945554E4720596175205975656E3C11
:100BF0002F68343E3C2F626F64793E3C2F68746DE1
:100C00006C3E003C68313E43616E6E6F74206765D8
:100C1000742073656E736F722072656164696E67AC
:100C200073213C2F68313E00000020002300260085
:100C300029002C002F0032000001000003010601F2
:100C4000090100000A0B02090C0D0E08070304013C
:100C50000000000000000000000000000000000094
:100C60000000000000000000000000000000121161
:100C70001000000000000000000000000000000064
:100C800000000000000000004E6574776F726B205A
:100C90006D61696E7461696E656420617420000025
:100CA000002200250028002B002E00310034000215
:100CB000010000050108010B0100002100240027AC
:100CC000002A002D0030003300010100000401075C
:100CD000010A0101021020200808102040102040C5
:100CE00080020102010804020101020408102040F0
:100CF000808040201008040201800402018040200E
:100D00001008040201080402010102040810204036
:100D1000800102040810204080050505050705082C
:100D2000080808020202020A0A080804040404016E
:100D30000101010101010103030303030303030490
:100D40000707070C0C0C0C0C0C0C0C020202020620
:100D5000060606060606060B0B0B0B0B0B0B0B41D0
:100D60007070656E64206D6561732E200053696E2E
:100D7000676C65206D6561732E2000536176652078
:100D80006D65617375726520746F3A0020202020B4
:100D90002020202020202020202020200020202073
:100DA00020202020202020202020202020000000A3
:100DB000010001001010020001000100B00000005D
:100DC00016000000280000001000000020000000B5
:100DD0000100010000000000000000000000000011
:100DE0000000000000000000000000000000000003
:100DF000FF000000FFFF0000FFFF0000FFFF0000FA
:100E0000CFBF0000C7BF0000C3BF0000C1BF0000CC
:100E1000C0BF000000000000C0BF0000C1BF000054
:100E2000C3BF0000C7BF0000CFBF0000FFFF00002E
:100E3000FFFF0000000000000000000000000000B4
:100E400000000000000000000000000000000000A2
:100E50000000000000000000000000000000000092
:100E60000000000000000000000000000000000082
:100E700000000000557365722D6167656E743A203D
:100E80002A0D0A446973616C6C6F773A202F0D0A42
:100E90000000029CAA9B11241FBECFEFD1E2DEBF4F
:100EA000CDBF00E00CBF1AE0A0E0B2E0EAE9FDE649
:100EB00001E00BBF02C007900D92A230B107D9F735
:100EC00026E1A2E0BAE001C01D92AD30B207E1F721
:100ED00017E0CAE4D7E000E006C021970109802F9F
:100EE000FE010E94D4B3C934D10780E00807A9F7F6
:100EF0000E94A89F0C94BBB60C9400008EBD0DB44C
:100F000007FEFDCF0895DC015996ED91FC913097D5
:100F1000B9F083899489A589B6894285538564850A
:100F20007585841B950BA60BB70B811520E89207DE
:100F3000A105B10538F08FEF9FE7A0E0B0E008957C
:100F400090E080E00895CF93DF931F92CDB7DEB796
:100F50006983DC01ED91FC910280F381E02D41E099
:100F600050E0BE016F5F7F4F19950F90DF91CF91D9
:100F70000895FC0120812EBD9B012150310941F0D3
:100F800051810DB407FEFDCF4EB55EBD4193F5CF47
:100F900061507109860F971F0DB407FEFDCF2EB566
:100FA000FC0120830895E091780CF091790C9081F8
:100FB0008091770C80958923808308958EBD0000F1
:100FC0000DB407FEFDCF8EB5089590E020917A0C08
:100FD000233339F40C96982F990F990F990F80E0CD
:100FE00008954896F8CFCF93DF931F92CDB7DEB721
:100FF0006983DC01ED91FC910280F381E02D41E0F9
:1010000050E0BE016F5F7F4F19950F90DF91CF9138
:101010000895FC01818D928D0895CF93DF931F92E7
:10102000CDB7DEB76983DC01ED91FC910280F381DD
:10103000E02D41E050E0BE016F5F7F4F19950F90AA
:10104000DF91CF910895FC019485FB01848598136D
:1010500003C081E0983008F080E00895CF93DF93DB
:101060001F92CDB7DEB76983DC01ED91FC91028060
:10107000F381E02D41E050E0BE016F5F7F4F199595
:101080000F90DF91CF910895FC01768765870895D1
:10109000DC01ED91FC91068CF78DE02D199591E026
:1010A00089270895862F089581E08627089521E0F5
:1010B000FC018485883008F020E0822F0895FC012F
:1010C000848595850895FC018489958908952CE08F
:1010D00034E0FC0131832083FB014089518962891E
:1010E0007389FC0142835383648375830895DC0113
:1010F000ED91FC91048CF58DE02D199490E080E049
:101100000895CF92DF92EF92FF921F93CF93DF93D8
:10111000EC0180E2689FF0011124ED57F34F9385B5
:10112000917161F0842F827449F080E0DF91CF915A
:101130001F91FF90EF90DF90CF900895142F6A8B4E
:101140008091840290918502A0918602B0918702DD
:101150008E879F87A88BB98BC488D588F12CE12C0A
:101160007601DD24CC24CF8AD88EE98EFA8E828D4A
:10117000938DB0E0A0E0AC01BD014C295D296E2942
:101180007F294F8B588F698F7A8F83858871B1F44F
:10119000848D958DA68DB78D8B8B9C8BAD8BBE8BE7
:1011A00081E08D831F701C831E821F821886198622
:1011B0001A861B861C861D8681E0B8CF803109F017
:1011C000B4CF9E012D5E3F4F8B8D9C8D0E943C9332
:1011D000882309F4AACF84E0E4CFFC01818D928DAD
:1011E000009711F00C94A793089561E0FC018481AD
:1011F0000C944082CF93DF93EC018FEF8EBD2FEFE5
:101200008F819885AC014F5F5F4F58874F83813046
:10121000924028F40DB407FEFDCF2EBDF1CF0DB4E2
:1012200007FEFDCFCE010E94F5081E82DF91CF910F
:101230000895CF93DF93EC01E98DFA8D309749F44F
:1012400081E090E09B838A8390E080E0DF91CF9102
:10125000089513821282898D9A8D0E94FC94E98DE3
:10126000FA8D22813381232B59F7F0CFCF93DF936F
:101270001F92CDB7DEB741E050E0BE016F5F7F4FF8
:101280000E949C96019731F4898190E00F90DF9144
:10129000CF9108958FEF9FEFF9CFFC01818D928D53
:1012A000009711F00C9436098FEF9FEF08950F937C
:1012B0001F93CF93DF93EC01898D9A8D10E000E0AE
:1012C000009799F00E9436098C010F3F100769F0D2
:1012D000898D9A8DFC0142855385648575854150C1
:1012E0005109610971090E94D693C801DF91CF911C
:1012F0001F910F910895CF92DF92EF92FF920F937B
:101300001F93CF93DF93CDB7DEB7AF970FB6F894A7
:10131000DEBF0FBECDBF7C016A010CE014E01A8372
:1013200009831C861B8688EE93E0A0E0B0E08D87E1
:101330009E87AF87B88B86E993E09A878987188F55
:101340000F8B198E1A8E1B8E1C8E88E089A31BA70B
:101350000AA71CA61DA61EA61FA680914910909143
:101360004A10A0914B10B0914C108EA39FA3A8A738
:10137000B9A78B839C83AD83BE8318861F82AE0181
:10138000465D5F4FCE0101960E94538781309105E3
:10139000B1F4D701ED91FC910488F589E02D1DA3EE
:1013A0000CA38CA59DA5AEA5BFA58EA39FA3A8A7A2
:1013B000B9A7A601BE016C5D7F4FC7011995AF9615
:1013C0000FB6F894DEBF0FBECDBFDF91CF911F9156
:1013D0000F91FF90EF90DF90CF9008959F92AF9282
:1013E000BF92CF92DF92EF92FF920F931F93CF9312
:1013F000DF935C017B018B01D0E0C0E0F8019190AC
:101400008F016501CC0EDD1EC6010E940CB298163C
:1014100021F0692DC6010E9414B22196CE32F1E06E
:10142000DF0761F7C701DF91CF911F910F91FF9007
:10143000EF90DF90CF90BF90AF909F900895FF9274
:101440000F931F93CF93DF93F82ECAEDDBE08E014D
:1014500061E0D80112968C910E945D836091990B96
:10146000F80182810E94408264EF71E080E090E0A8
:101470000E94B3830E5F1F4FFBE0003E1F0741F742
:10148000FF2009F447C060919B0B8A810E94408233
:1014900068EE73E080E090E00E94B38360919B0B64
:1014A0008C810E94408268EE73E080E090E00E94B0
:1014B000B3836091990B8A810E94408268EE73E049
:1014C00080E090E00E94B38322968BE0CE3DD80767
:1014D000D1F668EE73E080E090E00E94B383CFEC39
:1014E000D2E00CED1BE0E991F991D8018C910E5FEF
:1014F0001F4FEE0FFF1FE756F44F60810E9440829E
:1015000068EC70E080E090E00E94B383B2E0C53DFB
:10151000DB0749F7DF91CF911F910F91FF9008955D
:1015200081E08093ED028091EE02882341F088E013
:101530008093051460E08AEF93E10C94448E089543
:101540008091EE028823F9F08091ED028823D9F092
:1015500081E00E94718E8BE39FE10197F1F760E0DB
:1015600080E00E94828E6DE475E08AEF93E10E9434
:10157000508161E080E00E94828E6DE375E08AEF29
:1015800093E10C94508108958F929F92AF92BF92F5
:10159000CF92DF92EF92FF920F931F93CF93DF933F
:1015A0008C01862F0B30110509F09FC09091831399
:1015B000992309F0F89462E10E94E683EC0180919E
:1015C0008313882309F07894209701F180E090EC50
:1015D000A9E7B4EC8093761390937713A0937813D4
:1015E000B093791380937A1390937B13A0937C1319
:1015F000B0937D13CE3F8FEFD80709F4A9C0CF3F3A
:10160000DC0709F462C0CCEFDFEF30C1C0917E137C
:10161000E0907F136E2D70E090E080E00E94EFB0CC
:101620002DEC3CEC4CEC5DE30E944EB14B015C01B7
:101630006C2F70E090E080E00E94EFB09B01AC0165
:10164000C501B4010E9496B260937613709377132C
:101650008093781390937913D0918013F090811335
:101660006D2F6F7770E090E080E00E94EFB04B014B
:101670005C016F2D70E090E080E00E94EFB02DECF7
:101680003CEC4CEC5DE30E944EB19B01AC01C5010A
:10169000B4010E9496B2D7FD26C060937A1370936E
:1016A0007B1380937C1390937D13CE0DCD0FCF0DC4
:1016B00081E090E020918213C21302C090E080E0AC
:1016C000892B09F493C0CFEFDFEFCE01DF91CF91EB
:1016D0001F910F91FF90EF90DF90CF90BF90AF9050
:1016E0009F908F9008959058D8CFCFEFDFEF0631BD
:1016F000110509F0BBC090918313992309F0F89468
:1017000061E00E94E683EC0180918313882309F055
:101710007894209701F180E090ECA9E7B4EC8093F5
:10172000761390937713A0937813B09379138093E3
:101730007A1390937B13A0937C13B0937D13CF3FC8
:10174000DC0719F2209709F451C0229609F05BCF0B
:10175000CEEFDFEF8BC0C0917F13D0917E136091ED
:101760007E1370917F1376276727762790E080E0BD
:101770000E94EDB02DEC3CEC4CEC5DE30E944EB1D0
:101780006093761370937713809378139093791303
:10179000E0908113F09080136F2D6F77762F6E2D70
:1017A00090E080E00E94EDB02DEC3CEC4CEC5DE371
:1017B0000E944EB1F7FC18C060937A1370937B13AC
:1017C00080937C1390937D138C2F8D0F8E0D8F0D36
:1017D000C1E0D0E090918213891302C0D0E0C0E054
:1017E000D195C195D109ABCF9058E6CFC090761373
:1017F000D0907713E0907813F090791320E030E0E8
:1018000048EC52E4C701B6010E94AAB3D0E0C0E0A0
:10181000181614F4CBEFDFEF20E030E0A901C70188
:10182000B6010E94E8B087FF02C0CAEFDFEFC090A8
:101830007A13D0907B13E0907C13F0907D1320E01E
:1018400030E048EC52ECC701B6010E94E8B087FFD7
:1018500002C0C9EFDFEF20E030E040EF52E4C70103
:10186000B6010E94AAB318160CF483C00C301105FF
:1018700009F02BCF81E08093B30E8CE58093B50EF9
:101880001092B40E1092B60E60E082EF9FE00E94BC
:10189000947981E00E94548D0E948E836B017C01BB
:1018A0008091AD0E811168C081E08093AD0E809370
:1018B000AC0E9FEF9093AB0E1092AA0E94E0909313
:1018C000A90E8093880E8091880E886B8093880E75
:1018D0008091870E813009F028C11092870E0E94F6
:1018E0008E836B017C018091880E8093BB00809178
:1018F000AF0E9091B00EA091B10EB091B20E892BA7
:101900008A2B8B2BA1F00E948E830091AF0E109139
:10191000B00E2091B10E3091B20E6C197D098E0976
:101920009F09061717072807390708F446C0809152
:10193000BC0083FDD8CF85EC8093BC000E948E83D1
:101940006B017C018091AD0E813009F4F0C0809173
:10195000AA0E853008F00DC18091AA0EA9E8BEE05C
:10196000E5EEFBE090E0981769F12D9121939F5FE0
:10197000FACFC8EFDFEF7ACF8091AF0E9091B00E23
:10198000A091B10EB091B20E892B8A2B8B2B09F44A
:1019900087CF0E948E830091AF0E1091B00E2091E0
:1019A000B10E3091B20E6C197D098E099F09061790
:1019B00017072807390708F073CF8091AE0E0E94F1
:1019C000338D80E01092760C8093750C082F10E018
:1019D000CEEFDFEF882309F478CECDEFDFEF0530CF
:1019E00011050CF472CEC2ECDAE082EF9FE00E94A7
:1019F0004D7988872196CE01825C9A4080179107A5
:101A0000A4F3C091CA0A0091CB0A602F70E090E065
:101A100080E00E94EFB02DEC3CEC4CEC5DE30E94CA
:101A20004EB16B017C016C2F70E090E080E00E9471
:101A3000EFB09B01AC01C701B6010E9496B26B01E9
:101A40007C01C092C20AD092C30AE092C40AF0920A
:101A5000C50AD091CC0A1091CD0A6D2F6F7770E036
:101A600090E080E00E94EFB04B015C01612F70E0DC
:101A700090E080E00E94EFB02DEC3CEC4CEC5DE39C
:101A80000E944EB19B01AC01C501B4010E9496B207
:101A9000D7FD71C06093C60A7093C70A8093C80AC5
:101AA0009093C90AC00FCD0FC10F8091CE0AC81301
:101AB0000ACE20E030E048EC52E4C701B6010E94B3
:101AC000AAB3D0E0C0E0181614F4CBEFDFEF20E0AB
:101AD00030E040EA50E4C701B6010E94E8B087FF59
:101AE00002C0CAEFDFEFC090C60AD090C70AE090EC
:101AF000C80AF090C90A20E030E040EF51ECC7017D
:101B0000B6010E94E8B087FF02C0C9EFDFEF20E016
:101B100030E040EF52E4C701B6010E94AAB31816A4
:101B20000CF0D3CDC8EFDFEFD0CD85EE05CF80919F
:101B3000AF0E9091B00EA091B10EB091B20E892B64
:101B40008A2B8B2B09F4FECE0E948E830091AF0E60
:101B50001091B00E2091B10E3091B20E6C197D092A
:101B60008E099F09061717072807390708F0EACEDC
:101B700024CF85E0F3CE90588DCFCF93DF93EC0147
:101B80000E94A793882311F01D8281E0DF91CF91FD
:101B900008953F924F925F926F927F928F929F92A1
:101BA000AF92BF92CF92DF92EF92FF920F931F936B
:101BB000CF93DF93CDB7DEB72C970FB6F894DEBF87
:101BC0000FBECDBF5C01DC015B968D909C905C9755
:101BD00016964D905D906D907C901997411451042C
:101BE0006104710409F468C0BFEF4B1A5B0A6B0A09
:101BF0007B0A312CF40181859285A385B4859C01F3
:101C0000AD012F5F3F4F4F4F5F4F29873A874B877B
:101C10005C87730162011D821E821F821886F40197
:101C200081859285A385B4852D813E814F8158851C
:101C3000281739074A075B0708F056C089859A8537
:101C4000AB85BC858C159D05AE05BF0550F482E0C3
:101C5000C82ED12CE12CF12C92E0492E512C612C74
:101C6000712C9E012F5F3F4FB701A601C4010E9456
:101C7000BB928823C9F189819A81AB81BC81892B70
:101C80008A2B8B2B09F1260137019FEF491A590A3C
:101C9000690A790A2D813E814F8158852F5F3F4F18
:101CA0004F4F5F4F2D833E834F8358873FEFC31ABB
:101CB000D30AE30AF30AB3CFF40140805180628073
:101CC00073803324339496CFC414D504E604F70408
:101CD00009F70FEF1FEF2FEF3FE0B701A601C40197
:101CE0000E941992811119C080E02C960FB6F894C9
:101CF000DEBF0FBECDBFDF91CF911F910F91FF903F
:101D0000EF90DF90CF90BF90AF909F908F907F909B
:101D10006F905F904F903F900895F50146815781F5
:101D200060857185411551056105710539F097018F
:101D30008601C4010E9419928823B1F2D50116963A
:101D4000CD92DD92ED92FC921997332051F0D7019C
:101D5000C6010196A11DB11DF40180839183A28368
:101D6000B383F5018789908DA18DB28D892B8A2B44
:101D70008B2B39F4C78AD08EE18EF28E84818068F5
:101D8000848381E0B2CF3F924F925F926F927F92B5
:101D90008F929F92AF92BF92CF92DF92EF92FF927B
:101DA0000F931F93CF93DF9300D000D000D01F92EA
:101DB0001F92CDB7DEB77C01DC0115968C918111A5
:101DC00015C0FE013196CE010C966F0130E23193C1
:101DD000E817F907E1F7DA0130E087E09D91B92EC5
:101DE000992329F19E3239F48A3011F480E0D9C068
:101DF00038E08AE0F3CFE8EDFAE04491442321F0A3
:101E000031969413FACFF2CF831780F34FED490F39
:101E10004E3560F74FE9490F4A3118F440EEB42EC1
:101E2000B90EF601E30FF11DB0823F5FD7CF898174
:101E30008032E1F2322E8B01FB01838D948DD7012C
:101E40005C969C938E935B97168217821086118600
:101E50001286138614861586F80182859385A485DB
:101E6000B585438954896589768984179507A607BE
:101E7000B70708F04DC025E0B695A79597958795CB
:101E80002A95D1F7F82FFF70AF2ED80115968C91B7
:101E9000823008F4ABCFC8010E94360997FDA6CF67
:101EA000F80182859385A485B5854F96A11DB11D46
:101EB00082879387A487B587F0E2AF9EB001112493
:101EC0006D57734F6115710509F490CFDB018C914B
:101ED000882341F0853E09F057C0BB2029F0BB2480
:101EE000B394BACFB1100EC0F701A28A80918402D8
:101EF00090918502A0918602B0918702868797878C
:101F0000A08BB18BDB018C918111E9CFBB24B39401
:101F1000832D8271823109F069CFBB2009F459C049
:101F2000C7010E94D790009709F460CF20E2FC011E
:101F300011922A95E9F72BE0F601DC0101900D9250
:101F40002A95E1F721E238E2DC0151963C932E9389
:101F5000509740E058E01F965C934E931E9753961F
:101F60003C932E93529759963C932E93589757969D
:101F70005C934E9356970E945390882309F436CF72
:101F8000432DF70162890AC04BE050E0C6010E9470
:101F90000AB6892B09F060CF432D6A2DC7010E9434
:101FA00081082B960FB6F894DEBF0FBECDBFDF9130
:101FB000CF911F910F91FF90EF90DF90CF90BF9046
:101FC000AF909F908F907F906F905F904F903F90D9
:101FD0000895F8018581823009F408CFC8010E9474
:101FE000C90D882309F402CFD8015B96ED91FC91CD
:101FF0005C9716968D909D90AD90BC901997B2E02D
:102000008B1A9108A108B108858504C0880C991C19
:10201000AA1CBB1C8A95D2F786859785A089B189B1
:10202000880E991EAA1EBB1E848124013501480E0C
:10203000511C611C711C84149504A604B70401F1A1
:10204000E1E04E1A5108610871080E9453908823FC
:1020500009F4CCCEE3E8FCE0119283E89EE08E1711
:102060009F07D1F7409284025092850260928602C7
:10207000709287028091E40B81608093E40BDBCF48
:10208000D8015B96ED91FC91258580E092E0A0E07F
:10209000B0E004C0880F991FAA1FBB1F2A95D2F772
:1020A000F8014389548965897689840F951FA61F95
:1020B000B71F838B948BA58BB68BD70152961C923E
:1020C00083E89CE033CFCF93DF93CDB7DEB76D9736
:1020D0000FB6F894DEBF0FBECDBF442391F1AB0124
:1020E000BC011C821B828EE693E09A8389831E8248
:1020F00022E0CE0101960E94C30E81110EC090E035
:1021000081E0911101C080E06D960FB6F894DEBFBA
:102110000FBECDBFDF91CF910895CE0101960E94F1
:102120006A94882361F3CE0101960E94D7900097AC
:1021300031F325EEFC0120831E820E945390982FDC
:10214000DFCF81E0E1CF1F93CF93DF93CDB7DEB731
:102150006D970FB6F894DEBF0FBECDBFAB011C82EA
:102160001B822EE633E03A8329831E8221E0BC01E4
:10217000CE0101960E94C30E11E081110CC010E047
:10218000812F6D960FB6F894DEBF0FBECDBFDF91E5
:10219000CF911F910895CE0101960E94BD0DF0CF01
:1021A0008FEF0E947E078EB508958F929F92AF9217
:1021B000BF92FF920F931F93CF93DF93EC01F62E04
:1021C00049015A018E81882319F0CE010E94FA0834
:1021D00060E08C810E9440828CE291E00E9438870E
:1021E0008F2D80640E947E0708E110E0D501C401B4
:1021F000002E04C0B695A795979587950A94D2F7B7
:102200000E947E0708501109083F8FEF180771F7E9
:1022100085E9FF2021F088E0F8120DC087E80E94D0
:102220007E0710E00E94D0108A8787FF06C01F3FFC
:1022300021F01F5FF7CF8FEFF2CFDF91CF911F918A
:102240000F91FF90BF90AF909F908F900895AF92A5
:10225000BF92CF92DF92EF92FF920F931F93CF9393
:10226000DF93EC016901C801820F931F8130924016
:1022700050F58E81882379F088819981AA81BB816C
:1022800084179507A607B70731F48F819885C8167C
:10229000D90608F042C0488359836A837B838B85C3
:1022A000833039F089E0440F551F661F771F8A95E8
:1022B000D1F79A01AB0161E1CE010E94D5108823CC
:1022C00089F083E08D83CE010E94F50880E0DF91E4
:1022D000CF911F910F91FF90EF90DF90CF90BF9023
:1022E000AF9008950E9482865B010E94D0108A8779
:1022F0008F3F69F40E9482866A197B096D327140B2
:10230000A0F38FE08D83CE010E94F508DCCF8E3FD5
:10231000B1F418861F8281E08E838FEF8EBD2FEF80
:102320008F8198858C159D0560F40DB407FEFDCF57
:102330002EBD8F819885019698878F83F1CF8DE090
:10234000E1CFC8010197F7012FEFAF014E195F09E7
:102350004817590738F40DB407FEFDCF3EB5319349
:102360002EBDF3CF0DB407FEFDCF2EB5E80EF91E3E
:10237000F70120838F819885080F191F18870F8315
:102380008985882319F00115124030F08E81882349
:1023900019F0CE010E94FA0881E099CF0F931F93A4
:1023A000CF93DF93EC01890182E14115510561056D
:1023B000710599F08B85833039F089E0440F551F02
:1023C000661F771F8A95D1F79A01AB0168E1CE01AC
:1023D0000E94D510882319F084E08D8338C08EEFD9
:1023E0008EBDF801C8019E5F0DB407FEFDCF2081B0
:1023F0002EBD0DB407FEFDCF21812EBD3296E8170C
:10240000F90791F70DB407FEFDCF8FEF0E947E070D
:102410008FEF0E947E070E94D0108A878F718530CF
:1024200089F488E592E00E9438878823A9F020E0AB
:1024300030E0A9016DE0CE010E94D510882371F033
:1024400084E1CBCF81E18D83CE010E94F508CE01DE
:102450000E94F50880E00AC085E1BFCF0E94D0103D
:102460008111EECFCE010E94F50881E0DF91CF917E
:102470001F910F910895FC01DB0112968D919C91A3
:102480001397938382838EE693E0918380831496DF
:102490008C911497848315968C9115978583169645
:1024A0004D915D916D917C9119974683578360871B
:1024B00071871A964D915D916D917C911D97428720
:1024C0005387648775871E964D915D916D917C91C0
:1024D000519746875787608B718B52968C91529794
:1024E000828B53964D915D916D917C915697438B64
:1024F000548B658B768B57964D915D916D917C9148
:102500005A97478B508F618F728F5B968D919C91FC
:10251000948F838F0895DC015996ED91FC9130974B
:1025200021F081E09581911101C080E00895CF9361
:10253000DF93EC01898D9A8D009741F00E94BD0DCB
:10254000898D9A8D0E9493B41A8E198EDF91CF9146
:102550000895EF92FF920F931F93CF93DF93EC01B7
:102560007B018A011B821A8288EE93E0A0E0B0E032
:102570008C839D83AE83BF838EEE93E099838883A3
:102580008DE190E00E94F7B39A8F898F009779F0E0
:102590002DE1F701DC0101900D922A95E1F74CE065
:1025A00050E0B801CE010C960E9462B6188EDF9101
:1025B000CF911F910F91FF90EF900895E091780CCB
:1025C000F091790C80819091770C892B808308950C
:1025D000AF92BF92CF92DF92EF92FF920F931F9331
:1025E000CF93DF9300D01F92CDB7DEB78C016B0184
:1025F0007A0180917A0C8333E9F45B016801C40E9F
:10260000D51EC016D106A9F10E94D3078FE00E9403
:10261000DE07812F0E94DE07802F0E94DE070F5FFA
:102620001F4F80E00E94DE07F50181935F010E9449
:10263000DE12E7CF843369F50E94D30719830A833A
:102640008F2D8F778B83EC8264E070E0CE01019652
:102650000E94B907A70170E060E0C6010E9432B68F
:10266000E114F10421F0B701C6010E94B9070E94EC
:10267000DE12C7010F900F900F900F90DF91CF9156
:102680001F910F91FF90EF90DF90CF90BF90AF9090
:1026900008950E94D3070F3F110509F030F4198205
:1026A0000A831B8263E070E0D1CF17FD0BC0198253
:1026B0000A8333E0169507953A95E1F7007E0860A6
:1026C0000B83F0CFC80126E0969587952A95E1F710
:1026D000807E19830A830115104C18F480618B8366
:1026E000E1CF8861FCCFCF93DF931F92CDB7DEB7E8
:1026F00020917B0C30E0322F2227260F371F90E0ED
:10270000982F882741E050E0BE016F5F7F4F820F16
:10271000931F0E94E81289810F90DF91CF91089555
:10272000AF92BF92CF92DF92EF92FF920F931F93DF
:10273000CF93DF9300D000D01F921F92CDB7DEB7AA
:102740008C017B016A0180917A0C8333E1F458019A
:10275000A40EB51EA016B10609F46FC00E94D307DF
:1027600080EF0E94DE07812F0E94DE07802F0E94EB
:10277000DE070F5F1F4FF70181917F010E94DE0787
:102780000E94DE12E7CF5B01A40EB51E8433C1F4B4
:102790000E94D30719830A838D2D80688B83CC8296
:1027A00064E070E0CE0101960E94B907AE14BF0448
:1027B00009F441C0F70181917F010E94DE07F6CF45
:1027C0000E94D3070F3F110509F028F419820A83EC
:1027D00084E08B830CC017FD17C019820A8333E095
:1027E000169507953A95E1F7007E0C600B8386E01D
:1027F000C816D104A0F5F701DE011496EA15FB0511
:1028000099F081918D93FACFC80126E0969587952E
:102810002A95E1F7807E19830A830115104C10F484
:102820008461D7CF8C61D5CFB6016D5F7F4FCE016C
:1028300001960E94B9070E94DE12C60128960FB6C3
:10284000F894DEBF0FBECDBFDF91CF911F910F91E6
:10285000FF90EF90DF90CF90BF90AF90089563E02E
:1028600070E0CE0101960E94B907F70181917F01C6
:102870000E94DE07AE14BF04C1F7DDCFCF93DF9314
:102880001F92CDB7DEB741E050E0BE016F5F7F4FD2
:1028900090E080E00E94E81289810F90DF91CF9153
:1028A0000895CF93DF93C4E1D0E00E943E148823C3
:1028B00061F061E070E080E090E00E94B3832197D6
:1028C000A1F780E0DF91CF91089581E0FBCFCF9316
:1028D000DF931F92CDB7DEB7898341E050E0BE01A0
:1028E0006F5F7F4F90E080E00E9490130F90DF9128
:1028F000CF91089563E070E00C947313DA01E091D6
:102900007B0CF0E0FE2FEE27E60FF71F90E0982FEC
:102910008827A901BD018E0F9F1F0C949013CF93A0
:10292000DF931F921F92CDB7DEB779836A8322E0CF
:1029300030E0AE014F5F5F4F60E170E00E947E14B7
:102940000F900F90DF91CF910895CF93DF931F9257
:102950001F92CDB7DEB779836A8322E030E0AE0103
:102960004F5F5F4F64E070E00E947E140F900F9005
:10297000DF91CF910895CF93DF931F92CDB7DEB74C
:1029800020917B0C30E0322F2227260F371F90E05A
:10299000982F8827498341E050E0BE016F5F7F4F49
:1029A000820F931F0E9490130F90DF91CF91089593
:1029B000CF93C82F462F61E070E00E94BB1461E006
:1029C00070E08C2F0E9473138111F9CFCF9108957D
:1029D000DA01E0917B0CF0E0FE2FEE27E60FF71F07
:1029E00090E0982F8827A901BD018E0F9F1F0C949E
:1029F000E8126F927F929F92AF92BF92CF92DF9236
:102A0000EF92FF920F931F93CF93DF931F921F922A
:102A1000CDB7DEB7982E8B013A01690122E030E094
:102A2000AE014F5F5F4F64E270E00E94E814E980FE
:102A3000FA80FE24EF24FE24E00EF11E9701377089
:102A400040917A0C092D10E0C801433309F04CC0C5
:102A50000896982F8827990F990F990F820F931F27
:102A6000473309F446C0A9014C0D5D1D4130584063
:102A700008F43FC060E078E05B01A21AB30AA50148
:102A8000B3010E949013A6014A195B09B3016A0DB4
:102A90007B1D80917A0C833349F5085F1F4F000F2F
:102AA000000F000F80E0902F0E949013EC0CFD1C93
:102AB000F982EA8222E030E0AE014F5F5F4F64E2CC
:102AC00070E0892D0E947E140F900F90DF91CF91BE
:102AD0001F910F91FF90EF90DF90CF90BF90AF903C
:102AE0009F907F906F9008954096B3CF005F1F4FE7
:102AF000D6CFA601B301D8CFEF92FF921F93CF9309
:102B0000DF931F921F92CDB7DEB7182F22E030E07F
:102B1000AE014F5F5F4F60E270E00E94E814E98011
:102B2000FA80FE24EF24FE2422E030E0AE014F5F65
:102B30005F4F60E270E0812F0E94E81489819A81E2
:102B4000982789279827E816F90689F487E0189FBF
:102B5000F0011124E35DF34FF582E482C7010F9089
:102B60000F90DF91CF911F91FF90EF9008957C011E
:102B7000DBCFFF920F931F93CF93DF931F921F9290
:102B8000CDB7DEB7F82E22E030E0AE014F5F5F4FE9
:102B900066E270E00E94E81409811A81102701277B
:102BA000102722E030E0AE014F5F5F4F66E270E039
:102BB0008F2D0E94E81489819A8198278927982768
:102BC0000817190749F4C8010F900F90DF91CF91B2
:102BD0001F910F91FF9008958C01E3CF44E050E0E6
:102BE000BC018FE090E00C94901308951F93CF9355
:102BF000DF93182F80E591E00E944C7A812F0E948C
:102C00007C15EC01812F0E947A14873121F08C31E0
:102C100011F0D0E0C0E0CE01DF91CF911F91089577
:102C2000FC018485883010F40C94F61590E080E067
:102C30000895CF92DF92EF92FF921F93CF93DF938D
:102C4000182F7B01EA014130584010F0C0E0D8E075
:102C500080E591E00E944C7A812F0E947C156C01E6
:102C6000812F0E947A14873111F08C3121F5CC1616
:102C7000DD0670F380E591E00E944C7A9E01A70189
:102C800070E060E0812F0E94F91460E270E0812F13
:102C90000E94D81462E070E0812F0E94731384FDBB
:102CA0000DC0812F0E947A148823B9F080E591E04D
:102CB0000E944C7AEFCFD0E0C0E0DCCF40E162E090
:102CC00070E0812F0E94BB14CE01DF91CF911F9144
:102CD000FF90EF90DF90CF900895D0E0C0E0F4CF68
:102CE0000F931F93CF93DF938C01EA01FC0184853E
:102CF000883048F40E941916892B39F481E090E05D
:102D0000F80193838283D0E0C0E0CE01DF91CF91C0
:102D10001F910F910895CF92DF92EF92FF920F9340
:102D20001F93CF93DF938B017A016C0129EBC20EC5
:102D3000D11CF6014081EC012A96442349F050E071
:102D4000BC0167567F4FCE010E947016F6011082BB
:102D5000A701B801CE01DF91CF911F910F91FF9094
:102D6000EF90DF90CF900C947016CF93DF93EC012F
:102D7000C754DF4FE88121E02E0F2883E80FF92F99
:102D8000F11DE756FF4F6083203249F4BC016756BE
:102D90007F4F40E250E00A960E947016188281E050
:102DA00090E0DF91CF9108951F93CF93DF931F920F
:102DB000CDB7DEB7182F80E591E00E944C7A812FC5
:102DC0000E94E50727E0129FF0011124E35DF34F15
:102DD00022813381377041E050E0BE016F5F7F4F49
:102DE000820F931F0E94E81289810F90DF91CF918B
:102DF0001F910895FC01808D883040F4218D328D23
:102E0000232B21F00E94D41690E008958FEF9FEFBE
:102E10000895CF93DF93FC012485283028F08FEFAD
:102E20009FEFDF91CF910895EC010190F081E02DAB
:102E30000084F185E02D1995892B89F38C850E94FA
:102E4000D41690E0EECF1F93CF93DF93182F87E037
:102E5000189FE0011124C35DD34F888199810097A9
:102E600061F480E591E00E944C7A812F0E94B915AF
:102E70002E81821B910999838883DF91CF911F91C5
:102E80000895FC018485883010F40C94231790E099
:102E900080E008954F925F927F928F929F92AF92BF
:102EA000BF92CF92DF92EF92FF920F931F93CF9337
:102EB000DF931F921F92CDB7DEB7782E6B014A01C8
:102EC000A82EB12C27E0829FC0011124FC01E35DF4
:102ED000F34F7F010081118180E591E00E944C7ADF
:102EE0000815190554F4872D0E94B915F70126819C
:102EF0008C01021B1109118300830115110519F5BD
:102F0000872D0E947A14843159F0882349F001E01A
:102F100010E08C3111F410E000E0119501951109D9
:102F2000C8010F900F90DF91CF911F910F91FF90EB
:102F3000EF90DF90CF90BF90AF909F908F907F9059
:102F40005F904F900895801691060CF4840187E0FD
:102F50008A9DF0018B9DF00D1124E35DF34FE2801B
:102F6000F380C114D10451F12701F7E05F22872DCE
:102F70000E94E507840D951D20917A0C273309F4F2
:102F800053C09801240D351D2130384008F44CC041
:102F900020E038E0490184189508A401B6010E9498
:102FA000E8122601480C591C6801C818D908872D59
:102FB0000E94E507A601B2010E94E812E00EF11E90
:102FC00087E08A9DF0018B9DF00D1124E35DF34FA6
:102FD000F382E28220813181201B310B31832083F7
:102FE0008681800F912F911D8A3F910510F4232B2C
:102FF000F1F487E08A9DF0018B9DF00D1124E35DD3
:10300000F34F1682F982EA8222E030E0AE014F5F90
:103010005F4F68E270E0872D0E947E1460E470E0EC
:10302000872D0E94D8147CCFA801B601C5CF868316
:1030300077CFCF93DF93FC01218D328D21153105A0
:1030400029F48FEF9FEFDF91CF910895EC01808DF0
:103050004217530708F0A9010E944A1718161906CB
:1030600084F7298D3A8D281B390B3A8F298FEBCFA6
:103070000F931F93CF93DF931F92CDB7DEB7FC0161
:10308000218D328D232B41F48FEF9FEF0F90DF9135
:10309000CF911F910F9108958C0141E050E0BE0146
:1030A0006F5F7F4FFC01808D0E944A17181619062A
:1030B0005CF7F801818D928D0197928F818F8981C4
:1030C00090E0E4CF0F931F93CF93DF9300D000D015
:1030D0001F921F92CDB7DEB78C01D80159964D9142
:1030E0005C915A974115510551F0ED91FC91048C7A
:1030F000F58DE02D70E060E0C8011995EECFF80184
:10310000808D0E942317892BB1F148E050E0BE0169
:103110006F5F7F4FD80158968C910E944A171816FE
:103120001906F4F4D801509684E0FE01319601901E
:103130000D928A95E1F78D8190E0982F88272E8156
:10314000820F911DF801958B848B8F81282F30E0A1
:10315000322F22278885820F932F911D928F818F86
:1031600028960FB6F894DEBF0FBECDBFDF91CF918A
:103170001F910F91089590E080E0F2CFCF93DF93FD
:103180001F92CDB7DEB741E050E0BE016F5F7F4FC9
:10319000FC0184850E944A171816190634F48981A7
:1031A00090E00F90DF91CF9108958FEF9FEFF9CFCF
:1031B000FC018485883010F40C944A1790E080E07C
:1031C0000895CF93C82F80E591E00E944C7A68E083
:1031D00070E08C2FCF910C94D814CF93C82F80E53A
:1031E00091E00E944C7A60E170E08C2FCF910C94BA
:1031F000D814CF92DF92EF92FF920F931F93CF9349
:10320000DF9300D000D0CDB7DEB78C016B017A011F
:10321000FC01808D883010F40E94ED188CE094E061
:103220009A838983F60182819381A481B5818B83FE
:103230009C83AD83BE83B701CE0101960E94547C6E
:10324000F801808F8830A0F4F586E486128E118E06
:1032500081E026960FB6F894DEBF0FBECDBFDF919A
:10326000CF911F910F91FF90EF90DF90CF90089535
:1032700080E0EFCFCF93DF93EC01888D883020F48E
:103280000E94ED1888E0888FDF91CF910895CF9349
:10329000C82F80E591E00E944C7A8C2FCF910C943E
:1032A0007A14EF92FF920F931F93CF93DF937C01D9
:1032B00080917A0CD4E0833309F0D8E005E61CE075
:1032C000C0E0F801219131918F01F701848195814E
:1032D0002817390729F0CF5FDC13F3CF80E006C051
:1032E0008C2F0E9447198431B1F781E0DF91CF9193
:1032F0001F910F91FF90EF9008959F92AF92BF9210
:10330000CF92DF92EF92FF920F931F93CF93DF93B1
:10331000EC017B0180917A0C811121C01B821A8201
:1033200088EE93E0A0E0B0E08C839D83AE83BF8302
:1033300080EC93E09983888388E08C8788EE93E023
:103340009E878D87CE01DF91CF911F910F91FF90C6
:10335000EF90DF90CF90BF90AF909F90089534E0B2
:10336000932E833311F028E0922E85E6C82E8CE050
:10337000D82E10E098E0B92EA12CD6012D913D91C8
:103380006D01F701848195812817390791F4812F08
:103390000E944719082F873111F08C3139F5812FA0
:1033A0000E942317892B59F50C3119F4812F0E94A3
:1033B000E1181F5F9112E1CFA11008C0D701ED9174
:1033C000FC910084F185E02DC70119951B821A82BA
:1033D00088EE93E0A0E0B0E08C839D83AE83BF8352
:1033E00080EC93E099838883BC86A8CF843149F030
:1033F0008111DFCFF601329711821082DACFB12E20
:10340000D8CFAA24A394D5CF8F929F92AF92BF9288
:10341000CF92DF92EF92FF920F931F93CF93DF93A0
:10342000CDB7DEB72F970FB6F894DEBF0FBECDBF76
:103430005C014B017A0180917A0C8823C9F104E088
:10344000833309F008E0B501CE0101960E947D1991
:1034500085E6C82E8CE0D82E10E0F601219131913E
:103460006F01F501848195812817390751F4812F67
:103470000E944719873129F4A701B401812F0E94C6
:1034800019161F5F0113E9CFC7012F960FB6F894E5
:10349000DEBF0FBECDBFDF91CF911F910F91FF9087
:1034A000EF90DF90CF90BF90AF909F908F90089556
:1034B000F12CE12CE9CFCF93DF93EC018C858830A0
:1034C000D0F40E944719843189F0882379F088313B
:1034D00069F021E08C3159F4E881F9810084F185AB
:1034E000E02DCE01199521E0892B09F420E0822FEF
:1034F000DF91CF91089580E0FBCFCF92DF92EF92E2
:10350000FF92CF93DF93EC018C85883068F40E94A2
:10351000E1180E9482866B017C018C850E9447190C
:10352000811109C088E08C87DF91CF91FF90EF90E7
:10353000DF90CF90089561E070E080E090E00E941D
:10354000B3830E948286AB01BC014C195D096E09F0
:103550007F098D859E85B0E0A0E0481759076A076E
:103560007B07D8F28C850E94ED18DCCFCF93DF93D8
:10357000EC018C85883060F40E944719873111F086
:103580008C3131F48C850E94F6158115984088F3B2
:10359000DF91CF910895CF92DF92EF92FF920F9338
:1035A0001F93CF93DF93CDB7DEB7AF970FB6F894E5
:1035B000DEBF0FBECDBF8C016B017A018CE094E0C1
:1035C0009A8389831B821C821D821E821C861B8615
:1035D00048EE53E060E070E04D875E876F87788B40
:1035E00026E933E03A872987988F8F8B198E1A8EB8
:1035F0001B8E1C8E28E029A39BA78AA71CA61DA6AC
:103600001EA61FA6D8011C968C91883060F40E94DB
:103610004719882321F0F80184850E94E11888E089
:10362000D8011C968C938091491090914A10A091DA
:103630004B10B0914C108EA39FA3A8A7B9A78B8362
:103640009C83AD83BE8318861F82AE01465D5F4FAB
:10365000B601CE0101960E9453870097C1F0D801B0
:10366000ED91FC910684F785E02D8CE094E09DA31C
:103670008CA38CA59DA5AEA5BFA58EA39FA3A8A72F
:10368000B9A7A701BE016C5D7F4FC8011995AF9620
:103690000FB6F894DEBF0FBECDBFDF91CF911F9163
:1036A0000F91FF90EF90DF90CF9008958F929F92AF
:1036B000AF92BF92CF92DF92EF92FF920F931F9340
:1036C000CF93DF9300D000D000D01F92CDB7DEB7EC
:1036D00090917A0C911115C018E0812F2A960FB69F
:1036E000F894DEBF0FBECDBFDF91CF911F910F9138
:1036F000FF90EF90DF90CF90BF90AF909F908F9012
:10370000089528E0F22E933311F494E0F92E6B0122
:10371000082F80E591E00E944C7A9E012F5F3F4F79
:103720005901490110E0812F0E947A14F40181931C
:103730004F018823C1F01F5FF112F5CFF12CF50185
:1037400091915F019D3149F0983139F09A51923051
:1037500020F0F3941F11F3CFBFCF60E170E08F2D05
:103760000E94D8141F2DE12EF12CF701EE0FFF1F40
:10377000EB59F34F1182108283EE93E00197F1F73A
:10378000402F70E060E0812F0E94BB144FEF62E099
:1037900070E0812F0E94BB14B601CD2889F480917E
:1037A0008E0290918F0201968115F0EC9F0798F19F
:1037B00090938F0280938E0260918E0270918F029F
:1037C000812F0E94A51461E070E0812F0E94D8141F
:1037D00027E02E9DC0012F9D900D11249C01235D9B
:1037E000334F7901F9011182108222E030E0AE01FD
:1037F000475F5F4F68E270E0812F0E94E81489857F
:103800009A85982789279827F701938382831682C0
:103810001582148262CF80E090ECCACF0F931F9381
:10382000CF93DF93EC018B01888D883010F40E94D8
:10383000ED18B80182E00E94561B888F883050F442
:103840001D870C871A8E198E81E0DF91CF911F9111
:103850000F91089580E0F9CF9F92AF92BF92CF92DF
:10386000DF92EF92FF920F931F93CF93DF938C0120
:103870005B01942EE52EFC01C688D788F08C80E58C
:1038800091E00E944C7A8F2D0E947C15C92DDE2D6F
:103890008C179D0708F4EC019E01A501B6018F2D40
:1038A0000E94F914F801868997898C0F9D1F978BC8
:1038B000868BCE01DF91CF911F910F91FF90EF90FA
:1038C000DF90CF90BF90AF909F900895CF93FC0171
:1038D000C08D80E591E00E944C7A60E270E08C2F10
:1038E0000E94D81462E070E08C2F0E94731384FD54
:1038F00016C062E070E08C2F0E94731383FF0AC031
:1039000048E162E070E08C2F0E94BB1480E090E000
:10391000CF91089580E591E00E944C7AE3CF40E199
:1039200062E070E08C2F0E94BB1481E0F0CFFF9228
:103930000F931F93CF93DF93EB01FC01178A168A35
:103940002A81211109C02B81211106C02C8121114E
:1039500003C02D81222301F141155105E9F08A01AF
:10396000FC01F08C80E591E00E944C7AAE014E5F44
:103970005F4F24E030E06CE070E08F2D0E947E14F9
:10398000B8018F2D0E948F1481E090E0DF91CF91DC
:103990001F910F91FF90089580E0F7CF7F928F9253
:1039A0009F92AF92BF92CF92DF92EF92FF920F93CE
:1039B0001F93CF93DF93CDB7DEB7A6970FB6F894DA
:1039C000DEBF0FBECDBF8C01762E942E852E20E259
:1039D000A22ECE0101967C01DC01EA2D1D92EA9512
:1039E000E9F76801F3E4CF0ED11C8CE094E09AA3D0
:1039F00089A38FEF8BA38CA38DA38EA343E450E008
:103A0000BE016F5D7F4FC6010E94971C019609F4AD
:103A1000BFC081E089838A8386E0B82EBB821C8286
:103A2000D80114966D917D918D919C9117970E946C
:103A3000DCB36D837E838F83988789869A8680E83E
:103A400090E09C878B874CE150E0B701C6010E9453
:103A50002C1CFE0137968AE1DF011D928A95E9F759
:103A60004801B8E08B0E911CF401D70101900D9232
:103A7000BA94E1F740E150E0B701C6010E942C1C66
:103A8000F7011192AA94E9F796E0A92EB12C40E231
:103A900050E0B701C6010E942C1CF1E0AF1AB1083A
:103AA000B1F783E6898392E89A8393E59B838C83BD
:103AB00085E38D8381E08E837F829DE3988797E005
:103AC00099878A8786E0F401DE011B9601900D92AA
:103AD0008A95E1F78CE0898B8A8B6EE074E0CE01E9
:103AE00043960E944DB6D8011B966C91CE01499623
:103AF0000E94917BF8016485CE014B960E94917BD8
:103B0000D8011D966C91CE014D960E94917B4EE19D
:103B100050E0B701C6010E942C1CB3E07B121EC00E
:103B200082E3898384E08A83F80196859B83978565
:103B30009C8390899D8391899E8396E39F83888748
:103B4000828D8987838D8A87848D8B87858D8C87ED
:103B50004CE050E0B701C6010E942C1C87E389832A
:103B600086E08A8391E09B8393E09C838D838FE042
:103B70008E838AE38F838BE388878FEF898749E081
:103B800050E0B701C6010E942C1CC6010E94661CB1
:103B9000A6960FB6F894DEBF0FBECDBFDF91CF91D2
:103BA0001F910F91FF90EF90DF90CF90BF90AF905B
:103BB0009F908F907F9008950F931F93CF938C01C8
:103BC000FC016481758181E20E94561BC82F8830F8
:103BD000F8F480E591E00E944C7A8C2F0E947A14D0
:103BE000833131F08C2FCF911F910F910C94E118FC
:103BF00062E070E08C2F0E94D814F80184819581D6
:103C0000EC2FF0E0EE0FFF1FEB59F34F9183808311
:103C1000CF911F910F9108950F931F93CF93DF932F
:103C20001F921F92CDB7DEB7FC0124852830E0F447
:103C30008C0180E591E00E944C7A22E030E0AE01F8
:103C40004F5F5F4F60E170E0F80184850E94E814E7
:103C500089819A819827892798270F900F90DF9163
:103C6000CF911F910F91089590E080E0F6CF0F93D0
:103C70001F93CF93DF931F921F92CDB7DEB7FC0146
:103C800024852830E0F48C0180E591E00E944C7A94
:103C900022E030E0AE014F5F5F4F64E070E0F8017A
:103CA00084850E94E81489819A819827892798271A
:103CB0000F900F90DF91CF911F910F91089590E099
:103CC00080E0F6CFCF92DF92EF92FF921F93CF93D7
:103CD000DF93EC017B016A018C85883048F40E94F7
:103CE0004719882319F08C850E94E11888E08C8799
:103CF000F70182819381A481B5810097A105B10567
:103D000051F490E080E0DF91CF911F91FF90EF9010
:103D1000DF90CF9008958F3F9F4FAF4FBF4F89F3F4
:103D200070E060E081E20E94561B182F8C8788307B
:103D300040F780E591E00E944C7AA7014E5F5F4F0B
:103D400024E030E06CE070E0812F0E947E14B60128
:103D5000812F0E948F1464E070E0812F0E94D8149C
:103D60000E9482866B017C018C850E9447198731F5
:103D700011F18C3101F1882321F20E948286AB017E
:103D8000BC014C195D096E097F098D859E85B0E0E7
:103D9000A0E084179507A607B70738F061E070E048
:103DA00080E090E00E94B383DFCF8C850E94ED1805
:103DB00088E08C87A6CF81E090E0A5CFCF93DF93FA
:103DC000EC018CE094E0998388831A821B821C8228
:103DD0001D8280E591E00E944C7ABE016E5F7F4FAC
:103DE00044E050E08FE090E00E94E812CE01DF91C5
:103DF000CF9108954F925F926F927F928F929F9290
:103E0000AF92BF92CF92DF92EF92FF920F931F93E8
:103E1000CF93DF93EC01181619061CF44C0104979C
:103E20002CF0C1E0D0E063E0862E912C8E01000FD3
:103E3000111F7E01EE0CFF1CEE0CFF1C8C169D0664
:103E40000CF4B3C09701295C3D4F5901F901808101
:103E50009181A281B381970123523D4F69011816C8
:103E600019061A061B063CF50E94DA8AF601408004
:103E70005180628073806419750986099709F5017C
:103E80004080518062807380461657066806790626
:103E900058F410821182128213820E94DA8AF6018B
:103EA000608371838283938321960E5F1F4FF4E0BA
:103EB000EF0EF11CC3CF98012B523D4F3901F90190
:103EC00080819181980123533D4F5901F90120814F
:103ED000318182179307C1F0880F991FFC01E756C3
:103EE000F44F6081F801E652F44F80810E944082D5
:103EF000F30180819181F501918380836CE271E00F
:103F000080E090E00E94B383F60180819181A281DC
:103F1000B381181619061A061B0634F60E94DA8AAF
:103F2000F6012081318142815381621B730B840B26
:103F3000950BF701E354FD4F20813181428153817C
:103F4000261737074807590708F0AECFF601108249
:103F50001182128213829801295B3D4F6901F90198
:103F600080819181F501208131818217930709F4C5
:103F70009BCF880F991FFC01E756F44F6081F80131
:103F8000E652F44F80810E944082F6018081918147
:103F9000F50191838083F301918380836CE271E06A
:103FA00080E090E00E94B3837FCFDF91CF911F919B
:103FB0000F91FF90EF90DF90CF90BF90AF909F90C8
:103FC0008F907F906F905F904F900895CF93DF9385
:103FD000FC0124813581232B69F0EC01BC0185E5CE
:103FE0009FE00E943C81BE0188EB9EE0DF91CF9173
:103FF0000C943C81DF91CF910895CF93DF93FC0126
:1040000024813581232B69F0EC01BC0185E59FE01B
:104010000E942E81BE0188EB9EE0DF91CF910C942F
:104020002E81DF91CF910895CF93DF93FB01228101
:104030003381DC0113963C932E9312974481558172
:104040006681778114964D935D936D937C9317975A
:10405000408551856285738518964D935D936D9368
:104060007C931B971C96EF012C969C01275E3F4F7B
:1040700049914D93A217B307D9F7218D328DFC01D9
:10408000328F218FDF91CF9108950F931F93CF939C
:10409000DF938C01EB01FE0164912196662349F0C8
:1040A000D801ED91FC910190F081E02DC8011995A6
:1040B000F2CFDF91CF911F910F910895EF92FF9270
:1040C0000F931F93CF93DF93EC017B018A0164E28E
:1040D00074E00E9445206DE074E0CE010E9445200E
:1040E0006EED73E0CE010E944520B701CE010E9423
:1040F00026816BEA79E0CE010E9426810115110527
:1041000021F0B801CE010E9426816BEA79E0CE0150
:10411000DF91CF911F910F91FF90EF900C9426812A
:10412000CF93DF93EC0163EC73E00E9445206DE0D8
:1041300074E0CE010E94452065E973E0CE01DF9175
:10414000CF910C944520CF93DF93EC01FB012481A8
:1041500035810E940B80CE01DF91CF910895CF92DF
:10416000DF92EF92FF920F931F93CF93DF9300D0D4
:1041700000D0CDB7DEB77C01FB01848195818A0137
:10418000081B190B101611069CF0C7010E94DB7F5B
:10419000C70126960FB6F894DEBF0FBECDBFDF91E4
:1041A000CF911F910F91FF90EF90DF90CF900895E6
:1041B000CE0101960E94ED7FCC24C394D12C61E600
:1041C00076E0CE0101960E94D17EFFEFCF1ADF0A82
:1041D0000C151D05A4F7BE016F5F7F4FC7010E943C
:1041E000DB7FCE0101960E94577FD2CFDF92EF9204
:1041F000FF920F931F93CF93DF93CDB7DEB76297F4
:104200000FB6F894DEBF0FBECDBF2091EE02222381
:1042100079F12091ED02222359F17A018C016F3F4F
:104220007F4FA1F560E080E00E94828ED12CB80122
:104230008AEF93E10E942E816CE275E08AEF93E1B0
:104240000E945081F801848160E08D0D0E94828E71
:104250000E9482866093830E7093840E8093850EF5
:104260009093860EB701FF0C880B990B0E94B383C5
:1042700062960FB6F894DEBF0FBECDBFDF91CF912F
:104280001F910F91FF90EF90DF90089560E080E024
:104290000E94828E0E94828628EE33E040E050E049
:1042A0000E9432B2CA01B90120E831E541E050E094
:1042B0000E9454B2AB01BC0120E0CE0101960E94E5
:1042C000957FBE016F5F7F4FCE0107960E94ED7F05
:1042D00067EE78E0CE0107960E945C7EBC01CE01BD
:1042E0000D960E94ED7FCE0107960E94577FCE016A
:1042F00001960E94577FBE01635F7F4F8AEF93E173
:104300000E942E81D98860E08D2D0E94828ECE0180
:104310000D960E94577F8BCFEF92FF920F931F93C2
:10432000CF93DF9300D000D0CDB7DEB78C017B01F7
:1043300067E174E00E94F67F8AE0E816F1042CF44D
:1043400067E177E0C8010E94D17EB701CE010196F6
:104350000E94447DBE016F5F7F4FC8010E94DB7EDB
:10436000CE0101960E94577FC80126960FB6F89499
:10437000DEBF0FBECDBFDF91CF911F910F91FF9098
:10438000EF9008952F923F924F925F926F927F929B
:104390008F929F92AF92BF92CF92DF92EF92FF9255
:1043A0000F931F93CF93DF93CDB7DEB7C258D109D8
:1043B0000FB6F894DEBF0FBECDBF6C015B0188EE77
:1043C000482E83E0582E612C712C0EEE13E09BE5F5
:1043D000892E912C8C0E9D1E8CE0880E911C1B0149
:1043E0009FEF291A390AD6015996ED90FC90F701F2
:1043F0008581823008F493C082859385A485B58534
:104400008F719927AA27BB27892B8A2B8B2B09F021
:1044100086C040E250E0BE016F5F7F4FC7010E943F
:104420009C96803209F07BC08981882309F477C08B
:10443000853E79F38E3269F38C8583FDEACF22962F
:104440001FAE1EAE22978EE693E09FAF8EAF2496EE
:104450001FAE2497BE016F5F7F4FE0E080E04EE229
:10446000DB019D91BD019032A1F0883049F426E72F
:1044700030E02C0F3D1F2E0F311DD9014C93EF5F03
:1044800026E730E02C0F3D1F2E0F311DD9019C93E4
:10449000EF5F8F5F8B3021F786E790E08C0F9D1FD9
:1044A0008E0F911DFC011082D60159966D917C9161
:1044B00021E0AE014A585F4FCE01CE960E94C30E56
:1044C000882369F1BE01625C7F4FCE0181960E9414
:1044D0003B12AE014A585F4FBE016F5D7F4FCE0168
:1044E000855A9F4F0E94A912CE01855A9F4F0E9464
:1044F0008B12882309F4ACC0F12CFA141B042CF5A0
:1045000069E0CE0101960E94C27FCE0101960E9411
:10451000FD1FCE0101960E94577FF394EECF6F9658
:104520001FAE1EAE6F97A3964CAE5DAE6EAE7FAE65
:10453000A3976D961FAF0EAF6D97E6961FAE1EAE9A
:10454000E697A8961FAEA897CFCFB401CE010196EB
:104550000E94F67FCE0101960E94FD1FCE010196BA
:104560000E94577FE696EEADFFADE697309709F4CF
:1045700047C08581823008F443C06EE474E0CE0108
:1045800001960E94F67FCE0101960E94E61FCE01A1
:1045900001960E94577F6F968EAD9FAD6F979C835B
:1045A0008B83A3968CAD9DADAEADBFADA3978D8330
:1045B0009E83AF83B887A7968CAD9DADAEADBFADE2
:1045C000A79789879A87AB87BC871A8309838DE071
:1045D000F401DE011D9601900D928A95E1F7E696B1
:1045E0008EAD9FADE6979B8F8A8FB101CE0101966C
:1045F0000E94C221CE01855A9F4F0E949712F3CE8E
:1046000065E174E0CE0101960E94F67FCE0101962D
:104610000E94FD1FCE0101960E94577FE696EEADE7
:10462000FFADE69740E050E0BA01309721F04389B2
:10463000548965897689CE0101960E94707DCE01EC
:1046400001960E94E61FCE0101960E94577FD2CFAD
:10465000CE57DF4F0FB6F894DEBF0FBECDBFDF9150
:10466000CF911F910F91FF90EF90DF90CF90BF906F
:10467000AF909F908F907F906F905F904F903F9002
:104680002F900895CF92DF92EF92FF920F931F9396
:10469000CF93DF93CDB7DEB7C455D1090FB6F894E9
:1046A000DEBF0FBECDBF65965FAF4EAF6597209161
:1046B000130C3091140C2F5F3F4F3093140C209348
:1046C000130C2091120C2111C1C08B016C0181E0EF
:1046D0008093120C1092140C1092130C67E174E08A
:1046E000CE01895B9F4F0E94F67F67E174E0CE01A7
:1046F000835B9F4F0E94F67F50E040E068E174E0EA
:10470000C6010E945E200130110509F08EC067E1EC
:1047100074E082E192E10E943A7D67E174E08EEEFE
:1047200091E10E943A7D6596EEADFFAD659780817F
:10473000882309F474C000E210E09E012F5F3F4F10
:1047400040E250E0BE016F5D7F4FCE018D5A9F4F1A
:104750000E94937A049739F3BE016F5D7F4FCE01BB
:104760008F5B9F4F0E94F67FBE016F5B7F4FCE0134
:10477000895B9F4F0E941E7FCE018F5B9F4F0E94DF
:10478000577FBE016F5F7F4FCE018F5B9F4F0E94AF
:10479000F67FBE016F5B7F4FCE01835B9F4F0E9410
:1047A0001E7FCE018F5B9F4F0E94577F2D968EAD4F
:1047B0009FAD2D970297029730F461E374E08EEE7F
:1047C00091E10E943A7DBE01695B7F4F82E192E1F7
:1047D0000E94DB7E63968EAD9FAD6397892B09F4B3
:1047E000A2CF64E676E0CE018F5B9F4F0E94F67FFA
:1047F000BE01635B7F4FCE018F5B9F4F0E94727E35
:1048000061E676E00E945C7EBC0182E192E10E945A
:10481000DB7ECE018F5B9F4F0E94577F84CF62E18A
:1048200072E18EEE91E10E94DB7E1092120CCE01BD
:10483000835B9F4F0E94577FCE01895B9F4F0E94F1
:10484000577F0FB6F894DEBF0FBECDBFCC5ADF4FF7
:104850000FB6F894DEBF0FBECDBFDF91CF911F9191
:104860000F91FF90EF90DF90CF9008950F931F93DB
:10487000CF93DF93CDB7DEB72C970FB6F894DEBF9A
:104880000FBECDBF4C895D89FE017496AAEDBBE0D9
:1048900090E080E032964817590734F0208131814A
:1048A0002D933D930196F6CF8091DE0B9091DF0B17
:1048B00001969093E10B8093E00B8C8D9D8D9093EE
:1048C0009A0B8093990B8E8D9F8D90939C0B809368
:1048D0009B0BAD968FADAD97BE0164597F4F8F3264
:1048E00009F0BAC1CE0107960E94F67F68E374E032
:1048F000CE0101960E94F67FBE01695F7F4FCE0117
:1049000001960E94727EBC0182EA93E10E94077FB9
:10491000CE0101960E94577FCE0107960E94577FD5
:1049200062EA73E1CE0101960E94ED7FCE0101960D
:104930000E94E61FCE0101960E94577F6EE474E04C
:10494000CE0101960E94F67FBE016F5F7F4F82EA23
:1049500093E10E94217E182FCE0101960E94577F7D
:104960004091A6135091A713112309F47CC1BA01F9
:104970006250710982EA93E10E94107E682FCE0195
:1049800001960E94C27FBE016F5F7F4F84E893E172
:104990000E941E7FCE0101960E94577F68E772E158
:1049A000CE0107960E94F67F60E574E0CE01019685
:1049B0000E94F67FBE01695F7F4FCE0101960E9483
:1049C000727EBC018CE993E10E94077FCE010196C3
:1049D0000E94577FCE0107960E94577F24968FAD85
:1049E00024971F928F9323968FAD23971F928F93B7
:1049F00022968FAD22971F928F9321968FAD21978C
:104A00001F928F9386E594E09F938F938AEC9BE0AF
:104A10009F938F930E948BB6CE52DF4F88819981EE
:104A2000C25DD04090936C0280936B02BE016C52C9
:104A30007F4FCE0101960E94F67FBE016F5F7F4FD0
:104A400086E993E10E941E7FCE0101960E94577F66
:104A5000BE0161527F4FCE0101960E94F67FBE01DA
:104A60006F5F7F4F80E993E10E941E7FCE01019628
:104A70000E94577F409194135091951342505109D1
:104A800060E973E1CE0101960E94A320CE01019658
:104A90000E94A87D6C5960939502CE0101960E94F8
:104AA000577FCC5EDE4F688179818A819B81C451BA
:104AB000D1400E94EFB00FB6F894DEBF0FBECDBF5D
:104AC0009B01AC010E94AFB3882389F08CE390E096
:104AD000A0E0B0E0CC5EDE4F88839983AA83BB83DD
:104AE000C451D140CD5EDE4F1882C351D140CD5E5E
:104AF000DE4F8881C351D140882399F0CC5EDE4FD0
:104B000088819981AA81BB81C451D14080938A0256
:104B100090938B02A0938C02B0938D0281E08093DE
:104B2000800CC85EDE4F688179818A819B81C85183
:104B3000D1409B01AC010E94AFB3882361F080E0BB
:104B400090E0A0E7B2E4C85EDE4F88839983AA8331
:104B5000BB83C851D140C45EDE4F68817981CC519E
:104B6000D140072E000C880B990B0E94EFB09B01DF
:104B7000AC010E94AFB3882341F082E090E0C45EB4
:104B8000DE4F99838883CC51D140C45CDE4F0881CD
:104B90001981CC53D140B801012E000C880B990B20
:104BA0000E94EFB09B01AC010E94AFB3811103C022
:104BB0001016110644F080E590E0C45CDE4F998346
:104BC0008883CC53D140C45CDE4F88819981CC531B
:104BD000D140909332028093310288E2FE01E55188
:104BE000FF4FAEE9BBE001900D928A95E1F7CE5CF4
:104BF000DE4F88819981AA81BB81C253D1408093C5
:104C00001C0290931D02A0931E02B0931F02CA5C67
:104C1000DE4F88819981AA81BB81C653D1408093A0
:104C2000180290931902A0931A02B0931B02C65C5B
:104C3000DE4F88819981CA53D1409093500280936E
:104C40004F022C960FB6F894DEBF0FBECDBFDF919A
:104C5000CF911F910F910895CE0107960E94F67F84
:104C60006DE374E045CE4150510962EA73E1CE0133
:104C700001960E94A320BE016F5F7F4F84E893E1FD
:104C80000E941E7FCE0101960E94577F62EA73E167
:104C9000CE0101960E94ED7F6EE474E0CE01019694
:104CA0000E945C7EBC0182EA93E10E94077F72CE83
:104CB0000F931F93CF93DF9300D000D0CDB7DEB713
:104CC00020919D0B2223A9F08C0169E078E0CE01B0
:104CD00001960E94F67FB801CE0101960E94727E75
:104CE000BC0185E59FE00E943C81CE0101960E94B7
:104CF000577F26960FB6F894DEBF0FBECDBFDF916B
:104D0000CF911F910F910895DF92EF92FF920F9331
:104D10001F93CF93DF93CDB7DEB762970FB6F894AA
:104D2000DEBF0FBECDBF8C011092CF0A67E174E0E9
:104D3000CE010D960E94F67FFF24F39485E59FE057
:104D40000E94AB772091CF0A181619067CF5211125
:104D50002DC085E59FE00E9489778A3009F07EC0EA
:104D600089899A89892B09F481C0F092CF0A62E679
:104D700074E0CE0101960E94F67FBE01635F7F4F13
:104D8000CE0101960E94727EBC01CE0107960E9460
:104D9000ED7FCE0107960E945826CE0107960E940D
:104DA000577FCE0101960E94577F60C0F12CE12C05
:104DB000DD24D394222309F460C089899A8901975C
:104DC00009F045C069ED74E0CE0107960E94F67FB8
:104DD000BE01695F7F4FCE010D960E94417EF12C8E
:104DE000811115C062E774E0CE0101960E94F67F42
:104DF000BE016F5F7F4FCE010D960E94417EFF2462
:104E0000F3948111F12CCE0101960E94577FCE01BF
:104E100007960E94577FFF20A1F050E040E0BE01BE
:104E2000635F7F4FCE0101960E94A320BE016F5F9A
:104E30007F4F85EB91E10E941E7FCE0101960E947B
:104E4000577F64E170E080E090E00E94B383BE0190
:104E5000635F7F4FC8010E94DB7F8EC08D3009F4F5
:104E60007FCF682FCE010D960E94AF7E6AE070E082
:104E700080E090E00E94B38361CF88EB9EE00E94C7
:104E8000AB771816190614F588EB9EE00E94897717
:104E90008A30A9F08D3099F09091CF0A91110FC00E
:104EA000682FCE010D960E94AF7E8FEFE81AF80AA8
:104EB00065E070E080E090E00E94B383DECF8989F6
:104EC0009A89892BA9F3D092CF0AF2CF64E170E0DE
:104ED00080E090E00E94B383EF2809F43FC0898905
:104EE0009A89892BD9F180919D0B882389F169E0FA
:104EF00078E0CE0101960E94F67FBE016F5F7F4F82
:104F0000CE010D960E94417EF82ECE0101960E94A0
:104F1000577FF1101DC06BE674E0CE0101960E9430
:104F2000F67FCE0101960E94FD1FCE0101960E94E0
:104F3000577FBE01635F7F4FCE0101960E94ED7FD8
:104F4000CE0101960E94E61FCE0101960E94577F76
:104F500064E170E080E090E00E94B38389899A89DF
:104F60002091CF0A21112BCF009709F028CF67E1BC
:104F700074E0C8010E94F67FCE010D960E94577F13
:104F8000C80162960FB6F894DEBF0FBECDBFDF91A9
:104F9000CF911F910F91FF90EF90DF9008950F93A5
:104FA0001F93CF93DF93CDB7DEB72C970FB6F8944E
:104FB000DEBF0FBECDBF8C010E947F8CBC01C8013B
:104FC0000E948C210E94778CBC01CE0107960E9422
:104FD0008C2165E477E0CE0101960E94F67FBE0148
:104FE000695F7F4FCE0101960E94727EBC01C801AD
:104FF0000E94DB7ECE0101960E94577FCE0107966C
:105000000E94577F61E676E0C8010E94D17E0E942F
:105010006F8CBC01CE0101960E948C21BE016F5F96
:105020007F4FC8010E94DB7ECE0101960E94577F10
:1050300064E774E0C8010E94D17E0E94678CBC01C5
:10504000CE0101960E948C21BE016F5F7F4FC80187
:105050000E94DB7ECE0101960E94577F64E774E0D8
:10506000C8010E94D17E0E945D8CBC01CE010196D8
:105070000E948C21BE016F5F7F4FC8010E94DB7EC2
:10508000CE0101960E94577FC8012C960FB6F89466
:10509000DEBF0FBECDBFDF91CF911F910F9108955D
:1050A000CF93DF9300D000D0CDB7DEB70E94A00A27
:1050B000CE0101960E94CF274AE050E06FEF7FEFCC
:1050C000CE0101960E94F620CE0101960E94577FE4
:1050D00061E080E00E94828ECE0101960E94DE1E79
:1050E0006AEF73E1CE0101960E94B28066E774E038
:1050F0008AEF93E10E9426810E94828660931D0CB4
:1051000070931E0C80931F0C9093200C26960FB664
:10511000F894DEBF0FBECDBFDF91CF9108950F93FE
:105120001F93CF93DF9300D000D0CDB7DEB78C01B3
:10513000CE0101960E94CF274AE050E06FEF7FEF4B
:10514000CE0101960E94F620CE0101960E94577F63
:10515000B801CE0101960E94ED7F6AE070E0CE01B9
:1051600001960E94AF8ECE0101960E94577F26962F
:105170000FB6F894DEBF0FBECDBFDF91CF911F9168
:105180000F9108950F931F93CF93DF93CDB7DEB7A1
:105190002C970FB6F894DEBF0FBECDBF8C010E94D6
:1051A0007F8CBC01C8010E948C210E94778CBC01BD
:1051B000CE0107960E948C2165E477E0CE0101962E
:1051C0000E94F67FBE01695F7F4FCE0101960E946B
:1051D000727EBC01C8010E94DB7ECE0101960E9456
:1051E000577FCE0107960E94577F0E94DA8A0E945D
:1051F000648B6091050C70E0CE0107960E948C21B3
:1052000065E477E0CE0101960E94F67FBE01695FFA
:105210007F4FCE0101960E94727EBC01C8010E94A0
:10522000DB7ECE0101960E94577FCE0107960E9439
:10523000577F61E676E0C8010E94D17E0E946F8CA4
:10524000BC01CE0101960E948C21BE016F5F7F4F91
:10525000C8010E94DB7ECE0101960E94577F64E761
:1052600074E0C8010E94D17E0E94678CBC01CE010F
:1052700001960E948C21BE016F5F7F4FC8010E9482
:10528000DB7ECE0101960E94577F64E774E0C8017F
:105290000E94D17E0E945D8CBC01CE0101960E94CD
:1052A0008C21BE016F5F7F4FC8010E94DB7ECE0163
:1052B00001960E94577FC8012C960FB6F894DEBF66
:1052C0000FBECDBFDF91CF911F910F910895EF9247
:1052D000FF920F931F93CF93DF9300D01F92CDB710
:1052E000DEB78C017B01FB0184858830A8F08CE05F
:1052F00094E0F801918380831282138214821582D4
:10530000C8010F900F900F900F90DF91CF911F91D8
:105310000F91FF90EF90089580E591E00E944C7A04
:1053200024E030E0AE014F5F5F4F6CE070E0F701CA
:1053300084850E94E814BE016F5F7F4FC8010E9400
:105340007481DECF3F924F925F926F927F928F92E5
:105350009F92AF92BF92CF92DF92EF92FF920F9304
:105360001F93CF93DF93CDB7DEB7EA970FB6F894CC
:10537000DEBF0FBECDBF7C012A013B0169010E9447
:1053800082864B015C0187010D5B1F4FC8010E94A3
:105390006218181619069CF00E948286681979090D
:1053A0008A099B09461657066806790608F466C1FD
:1053B00062E370E080E090E00E94B383E7CF42E2D6
:1053C00050E0BE016F5F7F4FC8010E9419188981AC
:1053D0008230D1F0312C832DEA960FB6F894DEBFDF
:1053E0000FBECDBFDF91CF911F910F91FF90EF9036
:1053F000DF90CF90BF90AF909F908F907F906F90F5
:105400005F904F903F900895F80184899589833487
:10541000910501F76D817E818F8198850E94DCB3B3
:105420004B015C01F60180829182A282B38246E048
:1054300050E0B701685F7F4FCE014D960E940AB6DB
:10544000892B41F6F70180819181A281B381881671
:105450009906AA06BB0608F4BDCF84819581A68172
:10546000B78188159905AA05BB0508F4B3CF8989CA
:105470009A89AB89BC8986879787A08BB18B4EECC4
:1054800050E070E060E0C8010E941918312CC7019B
:10549000829698AB8FA7F701B696FAABE9AB089660
:1054A0009CAB8BAB67019AE1C90ED11CBD96FEABDC
:1054B000EDABC701429698AF8FABFD97FAAFE9AF5E
:1054C0004701FEE18F0E911CF801818D928D181617
:1054D00019060CF080CFC8010E943818833391055B
:1054E00009F4B2C014F58130910509F464C044F4A4
:1054F000892B51F3C8010E943818AC01552775C09B
:105500008330910509F462C00697A1F7C8010E9493
:105510003818B82E44E050E0B401C8010E941918B0
:10552000EB2DE450FF0BAF0160C08A33910509F405
:105530005FC084F585339105B1F1C697D9F6C801EE
:105540000E9438185C01B601CE0189960E947481D0
:105550008BA59CA5ADA5BEA5892B8A2B8B2BB1F065
:10556000EDA9FEA94080518062807380B601CE0112
:1055700083960E9474818DA19EA1AFA1B8A5A501BB
:10558000481659066A067B0609F0B8CF44E050E099
:10559000B60118C08B33910509F440C08F3F9105C7
:1055A00009F492CFA7CFC8010E943818C8010E9401
:1055B0003818382E89CFC8010E94381844E050E0CE
:1055C0006FA978ADC8010E9419187ECFC8010E944A
:1055D0003818B82E44E050E069AD7AADC8010E9499
:1055E00019188B2D8450990BAC0170E060E0EACF64
:1055F000C8010E94381844E050E069A97AA9C8019E
:105600000E941918F70166A177A180A591A50E94B3
:10561000DCB366A377A380A791A756CFC8010E94E9
:10562000381844E050E06BA97CA9C8010E94191801
:10563000F70162A573A584A595A50E94DCB362A7B6
:1056400073A784A795A740CFC8010E94381844E0EB
:1056500050E06FA578A9C8010E941918F70162A14E
:1056600073A184A195A10E94DCB362A373A384A358
:1056700095A366A777A780AB91AB26CF33243A9446
:10568000AACE2F923F924F925F926F927F928F920B
:105690009F92AF92BF92CF92DF92EF92FF920F93C1
:1056A0001F93CF93DF9300D000D0CDB7DEB78C012E
:1056B0000E9453A82FEC37E040E050E00E9454B223
:1056C000DC01CB010196A11DB11DF80184839583F6
:1056D000A683B78380839183A283B3835801F3E4C5
:1056E000AF0EB11CC5010E943A1964E470E0C50117
:1056F0000E940E1C882309F445C10E9482862B015A
:105700003C01480182E4880E911C48EEC42E43E01F
:10571000D42EE12CF12C52E0252E1E821D82D401C4
:105720008C918330B1F1811166C0F801848195813B
:10573000A681B7810196A11DB11D84839583A6839F
:10574000B7830E9482866419750986099709A701A3
:1057500096010E9432B2A90161E0C8010E94CE1CEC
:1057600081E0D4018C938D819E810197C1F20E94CA
:1057700082866419750986099709D801D6962D91F4
:105780003D914D915C91D9972617370748075907E6
:1057900020F6C5010E943A19F80184819581A681FD
:1057A000B7810196A11DB11D84839583A683B7831C
:1057B0000E948286F801FE966083718382839383C0
:1057C0008D819E8126960FB6F894DEBF0FBECDBFA9
:1057D000DF91CF911F910F91FF90EF90DF90CF90CD
:1057E000BF90AF909F908F907F906F905F904F9001
:1057F0003F902F9008958430F1F4F80184819581D1
:10580000A681B7810196A11DB11D84839583A683CE
:10581000B7830E9482866419750986099709A701D2
:1058200096010E9432B2A90163E0C8010E94CE1C19
:10583000D4012C9298CF813051F5F80142AD53AD8F
:1058400064AD75AD9E012F5F3F4FC8010E94A22934
:10585000382EF2E08F1390C089819A81AB81BC8190
:10586000F80184839583A683B7830E948286641996
:10587000750986099709A70196010E9432B2A9010C
:1058800063E0C8010E94CE1CD4013C926CCF8230F0
:1058900009F069CFF80142AD53AD64AD75AD9E011D
:1058A0002F5F3F4FC8010E94A229382EF5E08F13C9
:1058B0005DC0E3E0D401EC93F80182A193A1A4A11F
:1058C000B5A1892B8A2B8B2B41F484E893E0A0E0CF
:1058D000B0E082A393A3A4A3B5A3F80186A197A1E6
:1058E000A0A5B1A5892B8A2B8B2B61F482A193A152
:1058F000A4A1B5A1B695A7959795879586A397A3DB
:10590000A0A7B1A7F80182A593A5A4A5B5A5892B49
:105910008A2B8B2BA9F482A193A1A4A1B5A1AC01E0
:10592000BD0123E076956795579547952A95D1F760
:10593000841B950BA60BB70B82A793A7A4A7B5A7AB
:10594000F80186A197A1A0A5B1A586A797A7A0ABAE
:10595000B1AB82A593A5A4A5B5A582AB93ABA4AB2F
:10596000B5AB81E090E09E838D83FDCE96E08913F8
:1059700003C0D4011C92F7CEBFEF3B12F4CEF4016A
:105980001082F1CE1E821D821BCF8F929F92AF920A
:10599000BF92EF92FF920F931F93CF93DF9300D0AC
:1059A00000D0CDB7DEB700917C0C10917D0CF12CAE
:1059B000E12C0115110509F4DAC00E9482864B0121
:1059C0005C0178012EE3E20EF11CF70180819181E8
:1059D000A281B381A5019401281B390B4A0B5B0BF3
:1059E000CA01B901683E33E0730781059105A0F152
:1059F00028EE33E040E050E00E9432B2861A970A67
:105A0000A80AB90AD7018D929D92AD92BC921397C4
:105A1000F80186A597A5A0A9B1A949015A01880C4A
:105A2000991CAA1CBB1C88159905AA05BB0508F082
:105A3000B0C016A617A610AA11AAF80182A993A9A8
:105A4000A4A9B5A988159905AA05BB0508F0AAC09F
:105A500012AA13AA14AA15AAF80186A597A5A0A9A7
:105A6000B1A9892B8A2B8B2B09F0A5C0EE5BFF4FC8
:105A70008081833009F09FC084E08083C8010E9448
:105A8000412B01967C01F80182A993A9A4A9B5A98B
:105A9000892B8A2B8B2BA1F4EE5BFF4F8081833007
:105AA00011F081110DC01082F8013E9684E1DF01F2
:105AB0001D928A95E9F7C8010E94412B03967C014B
:105AC000B2E0EB16F10429F0E4E0EE16F10409F07F
:105AD0004EC080E591E00E944C7A60917C0C709100
:105AE0007D0C625F7F4FCE0101960E947481CE01D2
:105AF00003960E94EE1560917C0C70917D0C6A5E9D
:105B00007F4FCE0101960E94748144E050E0BE01B7
:105B10006D5F7F4F81E090E00E94901360917C0C5C
:105B200070917D0C6E5E7F4FCE0101960E94748154
:105B300044E050E0BE016D5F7F4F85E090E00E9441
:105B4000901360917C0C70917D0C625E7F4FCE0152
:105B500001960E9474818B819C81AD81BE8180936E
:105B6000491090934A10A0934B10B0934C10C7016A
:105B700026960FB6F894DEBF0FBECDBFDF91CF9152
:105B80001F910F91FF90EF90BF90AF909F908F90DB
:105B90000895821B930BA40BB50B86A797A7A0AB08
:105BA000B1AB4BCF821B930BA40BB50B82AB93AB6A
:105BB000A4ABB5AB51CFF12CE12C65CFEF92FF92A6
:105BC0000F931F93CF93DF93CDB7DEB7E8970FB650
:105BD000F894DEBF0FBECDBF67E174E0CE018796BB
:105BE0000E94F67F67E174E0CE018D960E94F67FF9
:105BF00082E0E82EF12C2496FFAEEEAE249786E0EC
:105C0000E9EFF2E0DE01D39601900D928A95E1F77B
:105C100086E0FE01F396DE01AC5BBF4F01900D9272
:105C20008A95E1F72C961FAE1EAE2C9701E010E08E
:105C30002E961FAF0EAF2E9788E0EFEFF2E0DE0159
:105C4000599601900D928A95E1F788E0FE017996C8
:105C5000DE01A25BBF4F01900D928A95E1F788E1CA
:105C6000E7E0F3E0DE01119601900D928A95E1F7ED
:105C700088E1FE013196DE01AA5ABF4F01900D92D4
:105C80008A95E1F780911F0390912003A091210351
:105C9000B0912203E2968CAF9DAFAEAFBFAFE2975B
:105CA0006AE774E0CE0187960E943A7D60E0CE01FB
:105CB00087960E94AF7E4BA55CA5BE016E587F4FB4
:105CC000CE0187960E946B7B60E276E0CE018D96D6
:105CD0000E94E27E60ED74E084E893E10E943A7DE8
:105CE00060E0CE018D960E94AF7E49A95AA9BE01FF
:105CF00066567F4FCE018D960E946B7B67E174E004
:105D0000CE0187960E943A7D67E174E0CE018D96C0
:105D10000E943A7DC250DF4F19821882CE5FD04078
:105D200080916B0290916C02C050DF4F9983888301
:105D3000C050D14080E090E0A0E7B2E4CA5BDE4F03
:105D400088839983AA83BB83C654D140C65BDE4F48
:105D5000F982E882CA54D14080E090E0A0E2B2E447
:105D6000C45BDE4F88839983AA83BB83CC54D14024
:105D700080E090E0A4E3B2E4C05BDE4F88839983C7
:105D8000AA83BB83C055D14084EB90E0CC5ADE4F50
:105D900099838883C455D14088E790E0CA5ADE4F82
:105DA00099838883C655D1408CE291E0A0E0B0E0B1
:105DB000C85ADE4F88839983AA83BB83C855D140D4
:105DC000C45ADE4F19830883CC55D140C25ADE4FE6
:105DD000F982E882CE55D14060E086E993E10E94E5
:105DE000AF7E60E080E993E10E94AF7E40919A131C
:105DF00050919B13BE016E5F7E4F86E993E10E9436
:105E00006B7B4091941350919513BE01635F7E4F5D
:105E100080E993E10E946B7B88E2EEE9FBE0DE0122
:105E2000A75EBE4F01900D928A95E1F78CE390E05A
:105E3000A0E0B0E0CE5BDE4F88839983AA83BB836A
:105E4000C254D140CF5BDE4F1882C154D14084EEA2
:105E500098E3AEE8B2E4C05ADE4F88839983AA8300
:105E6000BB83C056D14084EE98E3AEE8B1E4CC5990
:105E7000DE4F88839983AA83BB83C456D140C85917
:105E8000DE4F19830883C856D14080E590E0C6599B
:105E9000DE4F99838883CA56D14084EF91E0909376
:105EA000830280938202BE016E5B7F4F0E94EE09E7
:105EB00064EF71E080E090E00E94B38369E076E0F7
:105EC000CE0181960E94E47FCE0181960E94E61F5A
:105ED000CE0181960E94577FCE018D960E94577FFA
:105EE000CE0187960E94577FE8960FB6F894DEBFE2
:105EF0000FBECDBFDF91CF911F910F91FF90EF901B
:105F000008959F92AF92BF92CF92DF92EF92FF924D
:105F10000F931F93CF93DF93CDB7DEB7C859D10945
:105F20000FB6F894DEBF0FBECDBF5C017B016A01E6
:105F300060EA72E1CE0189579F4F0E94F67F6EE4BE
:105F400074E08E010F5F1F4FC8010E94F67FB801F9
:105F5000CE0189579F4F0E94417E982EC8010E9412
:105F6000577F911014C06EE474E0C8010E94F67F60
:105F7000BE0169577F4FC8010E94727EBC01CE01ED
:105F800089579F4F0E94077FC8010E94577FB50124
:105F9000CE0183579F4F0E94F67F62E874E0E114C0
:105FA000F10471F060E974E021E0E216F10441F0DF
:105FB0006BE974E032E0E316F10411F063EA74E097
:105FC000CE0189579F4F0E94D17E60E0CE01895754
:105FD0009F4F0E94AF7EB601C8010E94ED7F6AE02C
:105FE000C8010E94C37EBC01CE018D569F4F0E9406
:105FF000ED7FC8010E94577FC557DF4F4881598107
:10600000CB58D040B801CE0189579F4F0E946B7B7F
:106010008091810C882399F16BEA74E0CE018F574F
:106020009F4F0E94F67FCE018F579F4F0E94FD1F0A
:10603000CE018F579F4F0E94577FBE0169577F4FF8
:10604000CE018F579F4F0E94ED7FCE018F579F4FFC
:106050000E94FD1FCE018F579F4F0E94577FB801AE
:10606000CE018F579F4F0E94F67FCE018F579F4FD3
:106070000E94FD1FCE018F579F4F0E94577FCC5625
:10608000DF4F8881C459D0408F93CD56DF4F888130
:10609000C359D0408F93C257DF4F8881CE58D0402C
:1060A0008F93C357DF4F8881CD58D0408F938BEBB0
:1060B00094E09F938F9382E0E82E8AE0F82EFF927F
:1060C000EF920E948BB640913102509132026AECFD
:1060D0007BE087E292E10E94CB1A0FB6F894DEBF14
:1060E0000FBECDBF019709F07CC01F930F9381ECC9
:1060F00094E09F938F9304E01BE01F930F930E9403
:106100008BB6B80187E292E10E9412818AEC9BE093
:106110009F938F9382ED94E09F938F931F930F93A0
:106120000E948BB6B80187E292E10E94128166E379
:1061300074E087E292E10E9450816BEA79E087E2A5
:1061400092E10E945780F70101900020E9F7CF010A
:1061500083509A409F938F938BED94E09F938F93FE
:106160001F930F930E948BB6B80187E292E10E94C1
:106170001281B70187E292E10E94268162E370E01A
:1061800080E090E00E94B38387E292E10E947D1A52
:106190000FB6F894DEBF0FBECDBF11E0CE018D5615
:1061A0009F4F0E94577FCE0183579F4F0E94577F7A
:1061B000CE0189579F4F0E94577F812FC856DF4FCE
:1061C0000FB6F894DEBF0FBECDBFDF91CF911F9108
:1061D0000F91FF90EF90DF90CF90BF90AF909F9086
:1061E000089569E774E0CE018F579F4F0E94E47FC6
:1061F000CE018F579F4F0E94E61FCE018F579F4FB2
:106200000E94577F65E874E0CE018F579F4F0E9430
:10621000E47FCE018F579F4F0E94FD1FCE018F5705
:106220009F4F0E94577F62E07AE0CE018F579F4FC9
:106230000E94F67FCE018F579F4F0E94E61FCE012E
:106240008F579F4F0E94577F10E0A8CFEF92FF9289
:106250000F931F93CF93DF93CDB7DEB76E970FB633
:10626000F894DEBF0FBECDBF81E08093120C0E9478
:10627000C52C8C0160ED77E080E090E00E94B38354
:106280008BE0E82EF12C0D7F0130110571F481E0D7
:10629000E81AF10851F00E94C52C8C0160ED77E0FE
:1062A00080E090E00E94B383EECF0E9471847C0175
:1062B00068EE73E080E090E00E94B3830BE010E0B2
:1062C000EF2899F40150110981F060ED77E080E04A
:1062D00090E00E94B3830E9471847C0168EE73E0B9
:1062E00080E090E00E94B383EBCF87EE90E10E94C4
:1062F000DC1D1092120C0E94502867E174E0CE0160
:106300000D960E94F67F68E875E0CE0143960E94E4
:10631000E47FCE0149960E94DE1E8E8D1F928F93E0
:106320008D8D1F928F938C8D1F928F938B8D1F92CB
:106330008F9386E594E09F938F9384E09BE09F93F7
:106340008F930E948BB664E07BE0CE0101960E94A1
:10635000F67FBE016F5F7F4FCE010D960E941E7FBC
:10636000CE0101960E94577FBE016D5E7F4FCE0128
:1063700001960E94ED7FBE01635F7F4FCE010196C3
:106380000E94727EBC01CE0107960E94ED7FCE0175
:1063900007960E94E61FCE0107960E94577FCE0106
:1063A00001960E94577FBE01635F7F4FCE01019629
:1063B0000E94ED7FAE014F5F5F4F63E070E08DE6BE
:1063C00092E00E94812F182FCE0101960E94577FE4
:1063D0000FB6F894DEBF0FBECDBF111122C060EF23
:1063E00074E0CE0101960E94F67FBE016D5E7F4F84
:1063F000CE0101960E94727E64EF71E10E94727E6E
:10640000BC01CE0107960E94ED7FCE0107960E9447
:10641000E61FCE0107960E94577FCE0101960E948B
:10642000577FCE0143960E94577FCE010D960E9462
:10643000577F6E960FB6F894DEBF0FBECDBFDF91CB
:10644000CF911F910F91FF90EF9008957F928F92BF
:106450009F92AF92BF92CF92DF92EF92FF920F93F3
:106460001F93CF93DF93CDB7DEB762970FB6F89443
:10647000DEBF0FBECDBF65E775E0CE0101960E947D
:10648000E47FCE0101960E94E61FCE0101960E9494
:10649000577F04E010E030EDC32E3AE0D32E40E306
:1064A000E42E53EEB52E66E0A62E7CEE972EE1E3A9
:1064B000FE2EFEE48F2EA4E37A2E68EB72E287ECC8
:1064C00091E10E940E1CF6018E2D11928A95E9F73A
:1064D000B092D00AA092D20A9092D30AF092DC0A2B
:1064E0008092DD0AF092DE0A7092DF0A63E372E0C6
:1064F000CE0101960E9474814BE750E0BE016F5FB0
:106500007F4F87EC91E10E94971C40E350E060EDE3
:106510007AE087EC91E10E942C1C87EC91E10E94CB
:10652000661C68EE73E080E090E00E94B38387EC25
:1065300091E10E946218892B09F04FC001501109A6
:1065400009F07CC08091000B9091010BA091020B8F
:10655000B091030B892B8A2B8B2B09F089C067E143
:1065600074E082E192E10E943A7D62E172E1CE0143
:1065700001960E94ED7FAE014F5F5F4F70E060E0DB
:1065800081E592E00E94812F182FCE0101960E9492
:10659000577F11110EC06DE575E0CE0101960E9486
:1065A000E47FCE0101960E94E61FCE0101960E9473
:1065B000577F62960FB6F894DEBF0FBECDBFDF9156
:1065C000CF911F910F91FF90EF90DF90CF90BF90F0
:1065D000AF909F908F907F90089540E350E060EDE2
:1065E0007AE087EC91E10E9419186091F80A7091A5
:1065F000F90A76276727762790E080E0CB01772796
:1066000066270091FA0A1091FB0A1027012710272C
:1066100030E020E0602B712B822B932B7E508A4A36
:1066200093480E94B58A0E94DA8A6093000B7093A7
:10663000010B8093020B9093030B84CF68EE73E001
:1066400080E090E00E94B3834091000B5091010BD9
:106650006091020B7091030B2AE085E59FE00E9498
:1066600066806BEA79E085E59FE00E94578025CF40
:1066700068EE73E080E090E00E94B3830E94DA8AC3
:106680006093210C7093220C8093230C9093240C24
:106690000E94DA8A6093250C7093260C8093270C55
:1066A0009093280CCE0101960E94C228CE0101963B
:1066B0000E94E61FCE0101960E94577F0E946F8CB8
:1066C000BC01CE0107960E948C2164E774E0CE01E4
:1066D00007960E94D17E0E94678CBC01CE01019674
:1066E0000E948C21BE016F5F7F4FCE0107960E94F2
:1066F000DB7ECE0101960E94577F64E774E0CE01F5
:1067000007960E94D17E0E945D8CBC01CE0101964D
:106710000E948C21BE016F5F7F4FCE0107960E94C1
:10672000DB7ECE0101960E94577F69EF74E0CE01B7
:1067300001960E94F67FBE01695F7F4FCE010196F0
:106740000E94727EBC01CE010D960E94ED7F4AE050
:1067500050E06FEF7FEFCE010D960E94F620CE0144
:106760000D960E94577FCE0101960E94577FCE0161
:1067700007960E94577F68EE73E080E090E00E94E9
:10678000B3830E947F8CBC01CE010D960E948C21A8
:106790000E94778CBC01CE0101960E948C2165E499
:1067A00077E0CE0107960E94F67FBE016F5F7F4FB4
:1067B000CE0107960E94727EBC01CE010D960E940A
:1067C000DB7ECE0107960E94577FCE0101960E9484
:1067D000577F0E94DA8A0E94648B6091050C70E0FA
:1067E000CE0101960E948C2165E477E0CE010796E8
:1067F0000E94F67FBE016F5F7F4FCE0107960E9419
:10680000727EBC01CE010D960E94DB7ECE01079602
:106810000E94577FCE0101960E94577F6FEF74E070
:10682000CE0101960E94F67FBE01635F7F4FCE01CD
:1068300001960E94727EBC01CE0107960E94ED7FF8
:106840004AE050E06FEF7FEFCE0107960E94F620FE
:10685000CE0107960E94577FCE0101960E94577F76
:10686000CE010D960E94577F68EE73E080E090E0C5
:106870000E94B383CE0101960E94CF274AE050E0E8
:106880006FEF7FEFCE0101960E94F6208ECECF9261
:10689000DF92EF92FF920F931F93CF93DF93CDB7C9
:1068A000DEB768970FB6F894DEBF0FBECDBF67E1C5
:1068B00074E0CE0143960E94F67F6CE277E0CE0151
:1068C00001960E94E47FCE0101960E94FD1FCE0139
:1068D00001960E94577F6CA17DA1CE0101960E9476
:1068E000447DCE0101960E94E61FCE0101960E94D2
:1068F000577F6FE177E0CE0101960E94E47FCE01E1
:1069000001960E94FD1FCE0101960E94577F7E01D5
:1069100088E2E80EF11C01E010E08CA19DA1801737
:1069200091070CF1F701619171917F01CE01019600
:106930000E94447DCE0101960E94FD1FCE0101966A
:106940000E94577F61E676E0CE0101960E94F67FB5
:10695000CE0101960E94FD1FCE0101960E94577F35
:106960000F5F1F4FDACF61E676E0CE0101960E94FD
:10697000F67FCE0101960E94E61FCE0101960E948D
:10698000577F60E177E0CE0101960E94E47FCE015F
:1069900001960E94FD1FCE0101960E94577F6091D3
:1069A000990B70919A0BCE0101960E94447DCE0105
:1069B00001960E94FD1FCE0101960E94577F61E65D
:1069C00076E0CE0101960E94F67FCE0101960E94EC
:1069D000FD1FCE0101960E94577F60919B0B709125
:1069E0009C0BCE0101960E94447DCE0101960E942F
:1069F000E61FCE0101960E94577F69EF76E0CE0137
:106A000001960E94E47FCE0101960E94FD1FCE01F7
:106A100001960E94577FBE01605D7F4FCE010196B7
:106A20000E94F67FCE0101960E94FD1FCE010196C5
:106A30000E94577F61E676E0CE0101960E94F67FC4
:106A4000CE0101960E94FD1FCE0101960E94577F44
:106A5000BE016C5C7F4FCE0101960E94F67FCE0195
:106A600001960E94E61FCE0101960E94577F69EEB3
:106A700076E0CE0101960E94E47FCE0101960E944D
:106A8000E61FCE0101960E94577F8E010C5D1F4FBD
:106A9000EE24E394F12C6801F8E0CF0ED11C8CA118
:106AA0009DA18E159F050CF449C0B701CE01079634
:106AB0000E94447D69E078E0CE0101960E94F67F55
:106AC000BE01695F7F4FCE0101960E94727EBC01BC
:106AD000CE010D960E94ED7FCE010D960E94FD1F06
:106AE000CE010D960E94577FCE0101960E94577FDE
:106AF000CE0107960E94577F65E477E0CE010196AC
:106B00000E94F67FCE0101960E94FD1FCE010196E4
:106B10000E94577FB801645E7F4FCE0101960E94AC
:106B2000F67FCE0101960E94E61FCE0101960E94DB
:106B3000577F8FEFE81AF80A8601ADCF68ED76E04F
:106B4000CE0101960E94E47FCE0101960E94FD1FB6
:106B5000CE0101960E94577F7E01E2EBEE1AEEEF26
:106B6000FE0A10E000E0F70161917F0170E0CE01C4
:106B700001960E94447DCE0101960E94FD1FCE0128
:106B800001960E94577F0330110571F06DEA75E0A0
:106B9000CE0101960E94F67FCE0101960E94FD1F54
:106BA000CE0101960E94577F0F5F1F4F04301105E1
:106BB000D1F661E676E0CE0101960E94F67FCE0125
:106BC00001960E94E61FCE0101960E94577FC45B8A
:106BD000DE4F68817981CC54D140072E000C880BA0
:106BE000990B0E94EFB09B01AC010E94AFB38823C8
:106BF00041F080E590E0C45BDE4F99838883CC54FC
:106C0000D140C45BDE4F88819981CC54D1409093B0
:106C10003202809331026EEB76E0CE0101960E9443
:106C2000E47FCE0101960E94FD1FCE0101960E94D5
:106C3000577F6AEC7BE0CE0101960E94F67FCE0181
:106C400001960E94FD1FCE0101960E94577F6CEBBA
:106C500076E0CE0101960E94E47FCE0101960E946B
:106C6000FD1FCE0101960E94577F60913102709105
:106C70003202CE0101960E94447DCE0101960E940F
:106C8000E61FCE0101960E94577F6DEA76E0CE01A5
:106C900001960E94E47FCE0101960E94FD1FCE0165
:106CA00001960E94577FBE016C5A7F4FCE0101961C
:106CB0000E94F67FCE0101960E94E61FCE0101964A
:106CC0000E94577F65E075E0CE0101960E94F67F35
:106CD000CE0101960E94FD1FCE0101960E94577FB2
:106CE000BE0164587F4FCE0101960E94F67FCE010F
:106CF00001960E94E61FCE0101960E94577FC05266
:106D0000DF4F88819981C05ED040892B71F465EA9C
:106D100076E0CE0101960E94E47FCE0101960E94AA
:106D2000E61FCE0101960E94577FC052DF4F888137
:106D30009981C05ED040019771F46BE976E0CE0195
:106D400001960E94E47FCE0101960E94E61FCE01CB
:106D500001960E94577FC052DF4F88819981C05EA3
:106D6000D040029771F462E976E0CE0101960E946C
:106D7000E47FCE0101960E94E61FCE0101960E949B
:106D8000577F6CE876E0CE0101960E94E47FCE0149
:106D900001960E94FD1FCE0101960E94577FCE51A1
:106DA000DF4F68817981C25ED040CE0101960E949A
:106DB000447DCE0101960E94E61FCE0101960E94FD
:106DC000577F4091190C50911A0C60911B0C7091D7
:106DD0001C0C21E0CE0107960E945F7F60E175E008
:106DE000CE0101960E94F67FBE01695F7F4FCE0102
:106DF00001960E94727E6BE175E00E945C7EBC0190
:106E0000CE010D960E94ED7FCE010D960E94E61FE9
:106E1000CE010D960E94577FCE0101960E94577FAA
:106E2000CE0107960E94577F4091150C5091160C89
:106E30006091170C7091180C21E0CE0107960E940A
:106E40005F7F60E275E0CE0101960E94F67FBE0191
:106E5000695F7F4FCE0101960E94727E6BE175E003
:106E60000E945C7EBC01CE010D960E94ED7FCE019A
:106E70000D960E94E61FCE010D960E94577FCE010F
:106E800001960E94577FCE0107960E94577F6EE6BB
:106E900076E0CE0101960E94E47FCE0101960E9429
:106EA000FD1FCE0101960E94577F40911C02509118
:106EB0001D0260911E0270911F0225E0CE01019615
:106EC0000E945F7FCE0101960E94E61FCE010196CF
:106ED0000E94577F64E576E0CE0101960E94E47F30
:106EE000CE0101960E94FD1FCE0101960E94577FA0
:106EF000409118025091190260911A0270911B0280
:106F000025E0CE0101960E945F7FCE0101960E948E
:106F1000E61FCE0101960E94577F64E476E0CE0121
:106F200001960E94E47FCE0101960E94FD1FCE01D2
:106F300001960E94577F6091880270918902CE016C
:106F400001960E94447DCE0101960E94E61FCE016B
:106F500001960E94577F62E376E0CE0101960E947F
:106F6000E47FCE0101960E94FD1FCE0101960E9492
:106F7000577FC65BDE4F68817981CA54D140CE010C
:106F800001960E94447DCE0101960E94E61FCE012B
:106F900001960E94577FCE0143960E94577F6896C4
:106FA0000FB6F894DEBF0FBECDBFDF91CF911F911A
:106FB0000F91FF90EF90DF90CF9008952F923F9226
:106FC0004F925F926F927F928F929F92AF92BF92F9
:106FD000CF92DF92EF92FF920F931F93CF93DF93A5
:106FE000CDB7DEB7EF970FB6F894DEBF0FBECDBFBB
:106FF0003C018B0170E060E00E94107E8F8F67E1A2
:1070000074E0CE0149960E94F67F809188029091AB
:107010008902019709F07AC082E090E00E94208BFB
:1070200088E090E0909317028093160289E090E048
:1070300090931502809314028091970B9091980B76
:107040009093960B8093950B809110029091110272
:10705000A0911202B091130280930C0290930D0242
:10706000A0930E02B0930F02809128029091290202
:10707000A0912A02B0912B0280932C0290932D02B2
:10708000A0932E02B0932F028091940B8093930BC8
:1070900080918F0B9091900BA091910BB091920BDE
:1070A00080938B0B90938C0BA0938D0BB0938E0BD6
:1070B0008AE390E090930B0280930A028091190C6E
:1070C00090911A0CA0911B0CB0911C0C8093C60BD4
:1070D0009093C70BA093C80BB093C90B8091080283
:1070E00090910902909307028093060280911C02FE
:1070F00090911D02A0911E02B0911F028093200268
:1071000090932102A0932202B093230280918802DF
:1071100090918902029709F07AC083E090E00E9482
:10712000208B8AE090E090931702809316028BE008
:1071300090E090931502809314028091890B9091B6
:107140008A0B9093960B8093950B809102029091FD
:107150000302A0910402B091050280930C02909367
:107160000D02A0930E02B0930F0280912402909121
:107170002502A0912602B091270280932C029093C1
:107180002D02A0932E02B0932F028091880B809342
:10719000930B8091840B9091850BA091860BB091FD
:1071A000870B80938B0B90938C0BA0938D0BB093DC
:1071B0008E0B8BE390E090930B0280930A028091F8
:1071C000150C9091160CA091170CB091180C80938F
:1071D000C60B9093C70BA093C80BB093C90B8091BB
:1071E0000002909101029093070280930602809121
:1071F000180290911902A0911A02B0911B0280937B
:10720000200290932102A0932202B09323022F8D9B
:107210002335C1F41092960B1092950B80919D0B23
:10722000882371F067E275E0CE0101960E94F67F37
:10723000CE0101960E94E61FCE0101960E94577F63
:10724000E12CFCC0C8010197029708F038C281E028
:1072500090E0A0E0B0E080930C0290930D02A09328
:107260000E02B0930F02D30114968D919C91029758
:1072700048F141E050E0B301CE0101960E94A32005
:10728000BE016F5F7F4FCE0149960E941E7FCE01E7
:1072900001960E94577FCE0149960130110581F574
:1072A0000E949D7D20E030E040E251E40E944EB11A
:1072B0000E9474B360930C0270930D0280930E02CF
:1072C00090930F02BF8D81E090E09093960B809396
:1072D000950BB13401F580919D0B882309F4B0CF53
:1072E0006CE275E0CE0101960E94F67FCE01019618
:1072F0000E94E61FCE0101960E94577FE12C6BC0D1
:107300000E949D7D20912002309121024091220215
:1073100050912302CBCFEF8DE63409F075C160E0C8
:10732000809114020E94408264E670E080E090E068
:107330000E94B38361E0809116020E94408264E65D
:1073400070E080E090E00E94B38360E080911402DE
:107350000E94408264E670E080E090E00E94B38387
:1073600061E0809116020E94408264E670E080E055
:1073700090E00E94B38302301105C1F4CE0149961A
:107380000E949D7D9B01AC016091C60B7091C70B63
:107390008091C80B9091C90B0E9495B26093C60B67
:1073A0007093C70B8093C80B9093C90B80919D0B72
:1073B000882371F065E375E0CE0101960E94F67FA7
:1073C000CE0101960E94FD1FCE0101960E94577FBB
:1073D000EE24E394F12C80919D0B882379F1409168
:1073E0000C0250910D0260910E0270910F022AE082
:1073F000CE0101960E94957FBE016F5F7F4FCE0147
:1074000007960E94ED7F69E475E0CE0107960E9421
:107410005C7EBC01CE010D960E94ED7FCE010D96E3
:107420000E94E61FCE010D960E94577FCE0107965F
:107430000E94577FCE0101960E94577F80910C02D7
:1074400090910D02A0910E02B0910F02181619062C
:107450001A061B060CF013C65F8D563409F41BC5C3
:10746000523509F41CC560E0809114020E944082EC
:1074700064E670E080E090E00E94B3836E2D80911E
:1074800016020E94408264E670E080E090E00E9474
:10749000B3836091950B809114020E94408261E059
:1074A00070E080E090E00E94B38360E0809114027D
:1074B0000E94408268EC70E080E090E00E94B3831C
:1074C000C12CD12C7601C39480910C0290910D02B5
:1074D000A0910E02B0910F02C816D906EA06FB066B
:1074E0000CF0DFC46091950B809114020E944082E1
:1074F00061E070E080E090E00E94B38360E0809102
:1075000014020E94408260912C0270912D028091A1
:107510002E0290912F020E94B38380912C029091B1
:107520002D02A0912E02B0912F020B97A105B1055B
:107530000CF464C0609120027091210280912202BB
:10754000909123029B01AC010E9496B20E9474B3F9
:107550009B01AC01C701B6010E9454B2672B682B96
:10756000692B09F04BC0023011050CF447C065E9E6
:1075700075E089EA91E10E94E27EC701B6010E94AE
:10758000EFB02091200230912102409122025091CF
:1075900023020E9402B3AB01BC0120E0CE0107969A
:1075A0000E945F7F69EA71E1CE0101960E94ED7F42
:1075B000BE01695F7F4FCE0101960E94727E6BE132
:1075C00075E00E945C7EBC0189EA91E10E94077F20
:1075D000CE0101960E94577FCE0107960E94577FE9
:1075E00069EA71E1CE0101960E94ED7FCE0101961C
:1075F0000E948F28CE0101960E94577F8FEFC81AF4
:10760000D80AE80AF80A60CFFF8DF23509F076CE85
:1076100060E0809114020E94408264E670E080E0A5
:1076200090E00E94B38360E0809116020E94408245
:1076300064E670E080E090E00E94B38360E08091B7
:1076400014020E94408264E670E080E090E00E94B4
:10765000B38360E0809116020E94408264E670E08D
:1076600080E090E00E94B38302301105C1F4CE01A6
:1076700049960E949D7D9B01AC016091C60B709163
:10768000C70B8091C80B9091C90B0E9496B2609372
:10769000C60B7093C70B8093C80B9093C90B809156
:1076A0009D0B882309F4CCCD6FE375E0CE010196E4
:1076B0000E94F67FCE0101960E94FD1F1BCE011590
:1076C000110521F00330110509F0BACD809188022F
:1076D0009091890220E137E240E050E0813091054D
:1076E00021F420E43CE940E050E029AB3AAB4BAB5D
:1076F0005CAB21E030E03093960B2093950B3093F8
:10770000500220934F02029759F40330110541F4BF
:1077100080916E1390916F139093500280934F025B
:1077200040914F025091500258AB4FA7551F55271B
:10773000551F5DAB81E090E09093500280934F0223
:1077400060E0809114020E94408264E670E080E074
:1077500090E00E94B3836DA9809116020E9440823E
:1077600064E670E080E090E00E94B38360E0809186
:1077700014020E94408264E670E080E090E00E9483
:10778000B3836DA9809116020E94408264E670E086
:1077900080E090E00E94B3838FEF9FEF9093070209
:1077A00080930602812C912C54011BA61CA61DA6B9
:1077B0001EA61FA218A619A61AA61BA21CA21DA2CD
:1077C0001EA2212C312C21011AAE1BAE1CAE1DAE07
:1077D0001EAA1FAA18AE19AE61E0809114020E9481
:1077E000408261E070E080E090E00E94B38360E05E
:1077F000809114020E94408261E070E080E090E09D
:107800000E94B383C501B40126E030E040E050E0BF
:107810000E9454B2672B682B692B09F0F8C0A2E0D4
:10782000B0E0BFAFAEAFC12CD12C760180910A027F
:10783000863308F0865320917B00982F9870277F1D
:10784000922B90937B008770806480937C00809162
:107850007A00806480937A0080917A0086FDFCCF64
:107860008091780060917900762F682F072E000CA8
:10787000880B990B0E94EFB09B01AC01C701B601C8
:107880000E9496B26B017C0162E070E080E090E0C3
:107890000E94B3832EAD3FAD2130310509F0ADC05C
:1078A00020E030EC4FEF54E4C701B6010E9402B370
:1078B0006B017C0180919D0B882399F12DEC3CECB0
:1078C0004CE45EE3C701B6010E94AAB387FD29C05C
:1078D00022E0B701A601CE0107960E945F7F60E516
:1078E00075E0CE0101960E94F67FBE01695F7F4F71
:1078F000CE0101960E94727EBC01CE010D960E94BF
:10790000ED7FCE010D960E94E61FCE010D960E94DE
:10791000577FCE0101960E94577FCE0107960E94A5
:10792000577F2AE939E949E95EE3C701B6010E94B8
:10793000AAB387FD13C0211431044104510411F48A
:10794000140125018FA198A5A9A5BAA5892B8A2B79
:107950008B2B21F48FA298A6A9A6BAA62DEC3CECFD
:107960004CE45EE3C701B6010E94E8B018160CF4BF
:1079700049C0211431044104510409F448C02BA129
:107980003CA14DA15EA1232B242B252B69F48BA5B3
:107990009CA5ADA5BEA5892B8A2B8B2B09F401C113
:1079A0008BA29CA2ADA2BEA22BA13CA14DA15EA127
:1079B000221633064406550654F58091060290912E
:1079C000070297FFF3C01092070210920602220EE0
:1079D000331E441E551ED201C101B595A79597953A
:1079E00087958AAF9BAFACAFBDAF1BA21CA21DA2F7
:1079F0001EA2212C312C21010AC0E1E0F0E0FFAFF2
:107A0000EEAF14CF211431044104510469F6E09023
:107A10000602F090070292E0E916F10434F4F7FC54
:107A2000E1C00330110509F0DDC089A89AA8ABA810
:107A3000BCA8AAE08A0E911CA11CB11C89A99AA914
:107A4000ABA9BCA988169906AA06BB060CF4C4CE3D
:107A5000E2E0EE16F1040CF479C06EA97FA988ADBE
:107A600099AD2AAD3BAD4CAD5DAD621B730B840B84
:107A7000950B0E94EFB04B015C01B701FF0C880B26
:107A8000990B0E94EFB09B01AC01C501B4010E94AB
:107A900002B320E030E044EB53E40E9402B36B01F8
:107AA0007C01C0922002D0922102E0922202F09248
:107AB000230220E030E040E85FE30E94AAB387FDA4
:107AC000ABC080918802909189028130910509F0C4
:107AD0008FC0C0926613D0926713E0926813F09241
:107AE0006913C0921C02D0921D02E0921E02F09215
:107AF0001F0268EB75E0CE0101960E94E47FCE0183
:107B000001960E94FD1FCE0101960E94577F409171
:107B1000200250912102609122027091230225E0FF
:107B2000CE0101960E945F7FCE0101960E94E61F62
:107B3000CE0101960E94577F84EF91E090938302DB
:107B40008093820268E472E10E94EE09033011051D
:107B500031F03DA9E32E0115110509F06FCCC301E9
:107B60000E949D7D6B017C01C092C60BD092C70B19
:107B7000E092C80BF092C90B20E030E044EB53E4F4
:107B8000C701B6010E94AAB387FD6AC020E030E0B9
:107B900044EB53E4C701B6010E9495B26B017C012E
:107BA000EBCF8BA69CA6ADA6BEA6FACE01151105FD
:107BB00009F02DCF019690930702809306022BA126
:107BC0003CA14DA15EA1220E331E441E551ED201C2
:107BD000C101B595A795979587958EAB9FABA8AF3B
:107BE000B9AF03CFBFEF8B1A9B0AAB0ABB0A26CFF4
:107BF000029709F07ECFC0926A13D0926B13E09285
:107C00006C13F0926D13C0921802D0921902E09298
:107C10001A02F0921B026DCF6CE975E0CE0101965D
:107C20000E94E47FCE0101960E94FD1FCE010196C5
:107C30000E94577F409120025091210260912202C0
:107C40007091230225E0CE0101960E945F7FCE0154
:107C500001960E94E61FCE0101960E94577F76CFC3
:107C600020E030E0A901C701B6010E94E8B087FF1B
:107C70000BC020E030E044EB53E4C701B6010E94A2
:107C800096B26B017C01ECCFC0928B0BD0928C0B27
:107C9000E0928D0BF0928E0B4BA45CA46DA47EA49D
:107CA0008FA198A5A9A5BAA5481A590A6A0A7B0AFC
:107CB00001151105D9F410928B0B10928C0B1092B8
:107CC0008D0B10928E0BAFA5B8A9812C912C54016D
:107CD0008394C12CD12C7601B7FF26C0C12CD12CA6
:107CE000760188248A94982C54011EC0EFA5F8A927
:107CF000812C912C54018394F7FF04C088248A942A
:107D0000982C5401C0908B0BD0908C0BE0908D0B75
:107D1000F0908E0B20E030E044E353E4C701B6015D
:107D20000E94E8B087FF92C0C701B6019058209129
:107D300020023091210240912202509123020E94A0
:107D40004EB16B017C01A3019201C501B4010E94F7
:107D500022B20E94EFB020E030E040E05FE30E94FA
:107D60004EB19B01AC01C701B6010E9495B20E94C1
:107D700074B360930C0270930D0280930E02909383
:107D80000F0280919D0B882309F441C02AE04BA586
:107D90005CA56DA57EA5CE010D960E94957F2AE07B
:107DA0004FA158A569A57AA5CE0107960E94957F97
:107DB00067E575E0CE0101960E94F67FBE01695F1E
:107DC0007F4FCE0101960E94727E61E676E00E94AE
:107DD0005C7EBE01635F7F4F0E94727EBC01CE015C
:107DE00043960E94ED7FCE0143960E94E61FCE018E
:107DF00043960E94577FCE0101960E94577FCE0185
:107E000007960E94577FCE010D960E94577F809162
:107E10000C0290910D02A0910E02B0910F02B7FFDB
:107E200036C0B095A095909581959F4FAF4FBF4FAD
:107E300080930C0290930D02A0930E02B0930F0258
:107E4000EE24E394F12C36E43F8FF8CA209120020F
:107E50003091210240912202509123022F8F38A3AA
:107E600049A35AA3A701960160E070E084EB93E474
:107E70000E9495B260938B0B70938C0B80938D0B4B
:107E800090938E0B2F8D38A149A15AA158CFE12C88
:107E900042E54F8FD3CAEE24E394F12CE4CAE12CDF
:107EA000E2CA0230110524F40115110509F0DFC002
:107EB00061E080E00E94828E0230110524F40115F9
:107EC000110509F09CC0C090C60BD090C70BE09084
:107ED000C80BF090C90B20E030E044EB53E4C7013D
:107EE000B6010E94AAB387FD0BC020E030E044EB4E
:107EF00053E4C701B6010E9495B26B017C01EBCF40
:107F000020E030E0A901C701B6010E94E8B087FF78
:107F10000BC020E030E044EB53E4C701B6010E94FF
:107F200096B26B017C01ECCFC092C60BD092C70B0E
:107F3000E092C80BF092C90B80918802909189025F
:107F40000197B1F460E175E089EA91E10E943A7D20
:107F50008091C60B9091C70BA091C80BB091C90B33
:107F60008093190C90931A0CA0931B0CB0931C0CCB
:107F700080918802909189020297B1F460E275E0E5
:107F800089EA91E10E943A7D8091C60B9091C70BDE
:107F9000A091C80BB091C90B8093150C9093160C4F
:107FA000A093170CB093180C4091C60B5091C70BBF
:107FB0006091C80B7091C90B20E0CE0107960E941A
:107FC0005F7F69EA71E1CE0101960E94ED7FBE01FB
:107FD000695F7F4FCE0101960E94727E6CE175E071
:107FE0000E945C7EBC0189EA91E10E94077FCE017C
:107FF00001960E94577FCE0107960E94577F01305D
:10800000110539F540910C0250910D0260910E025C
:1080100070910F0221E0CE0107960E94957F6FE5D7
:1080200075E0CE0101960E94F67FBE01695F7F4F29
:10803000CE0101960E94727EBC0189EA91E10E9404
:10804000077FCE0101960E94577FCE0107960E94BE
:10805000577F69EA71E1CE0101960E94ED7FCE0162
:1080600001960E948F28CE0101960E94577F1092A0
:108070000C0210920D0210920E0210920F028091CB
:108080008802909189028130910509F083C0809126
:10809000950B9091960B9093980B8093970B8091F2
:1080A0000C0290910D02A0910E02B0910F028093EC
:1080B000100290931102A0931202B09313028091C8
:1080C0002C0290912D02A0912E02B0912F0280934C
:1080D000280290932902A0932A02B0932B02809148
:1080E000930B8093940B80918B0B90918C0BA091B0
:1080F0008D0BB0918E0B80938F0B9093900BA09370
:10810000910BB093920B8091C60B9091C70BA091ED
:10811000C80BB091C90B8093190C90931A0CA093C3
:108120001B0CB0931C0C8091060290910702909357
:10813000090280930802012B81F480912002909122
:108140002102A0912202B091230280931C029093FD
:108150001D02A0931E02B0931F02CE0149960E94F9
:10816000577FEF960FB6F894DEBF0FBECDBFDF91FD
:10817000CF911F910F91FF90EF90DF90CF90BF9024
:10818000AF909F908F907F906F905F904F903F90B7
:108190002F900895029709F78091950B9091960B77
:1081A00090938A0B8093890B80910C0290910D0221
:1081B000A0910E02B0910F028093020290930302ED
:1081C000A0930402B093050280912C0290912D029D
:1081D000A0912E02B0912F02809324029093250249
:1081E000A0932602B09327028091930B8093880B73
:1081F00080918B0B90918C0BA0918D0BB0918E0B7D
:108200008093840B9093850BA093860BB093870B80
:108210008091C60B9091C70BA091C80BB091C90B70
:108220008093150C9093160CA093170CB093180C18
:1082300080910602909107029093010280930002C0
:10824000012B09F08ACF8091200290912102A09108
:108250002202B09123028093180290931902A093F6
:108260001A02B0931B0279CF2F923F924F925F92E6
:108270006F927F928F929F92AF92BF92CF92DF9236
:10828000EF92FF920F931F93CF93DF93CDB7DEB79B
:10829000C554D1090FB6F894DEBF0FBECDBF40E084
:1082A00052EC61E070E085E59FE00E944F7A40E883
:1082B00055E260E070E088EB9EE00E944F7A61E05A
:1082C00088E00E945D8361E089E00E945D8360E058
:1082D0008AE30E945D8361E088E00E94408260E062
:1082E00089E00E94408261E08AE00E945D8361E053
:1082F0008BE00E945D8360E08BE30E945D8361E020
:108300008AE00E94408260E08BE00E9440820E94EE
:10831000468384EF91E0909383028093820265EC20
:108320007AE085E59FE00E9450816BEA79E085E57F
:108330009FE00E94578060ED77E080E090E00E942F
:10834000B38385E59FE00E948977182F8EE1E82EA0
:10835000F12C11110BC085E59FE00E948977182F41
:108360006EE170E080E090E00E94B38321E0E21AC9
:10837000F10879F78091820290918302B6E78B2E03
:10838000B3E19B2E08E4C02E02E1D02EFC01E8549C
:10839000F2415F01C5018C0D9D1D0E940CB2F601DA
:1083A00081936F018E169F06A9F7609162137091F9
:1083B0006313072E000C880B990B0E94EFB09B01F2
:1083C000AC010E94AFB3882331F081E090E090933C
:1083D0006313809362136091641370916513072E89
:1083E000000C880B990B0E94EFB09B01AC010E941E
:1083F000AFB3882331F082E090E0909365138093CF
:1084000064131537B1F060915E1370915F13809122
:108410006013909161130E94EFB09B01AC010E9428
:10842000AFB3811106C08091481290914912819793
:10843000E0F02DB73EB72E5231400FB6F8943EBF54
:108440000FBE2DBFADB7BEB711968EE291E0E8E446
:10845000F2E101900D920197E1F70E94DE2D0FB637
:10846000F894DEBF0FBECDBF15E7EDB7FEB7EE52F5
:10847000F1400FB6F894FEBF0FBEEDBFADB7BEB76B
:1084800011968EE291E0E8E4F2E101900D920197FD
:10849000E1F70E9436240FB6F894DEBF0FBECDBFC1
:1084A000153711F01337D9F48DB79EB78E5291401E
:1084B0000FB6F8949EBF0FBE8DBFADB7BEB7119675
:1084C0008EE291E0E8E4F2E101900D920197E1F78C
:1084D0000E9447340FB6F894DEBF0FBECDBF63EBEA
:1084E0007AE08AEF91E10E94E27E6DE97AE084EF22
:1084F00091E10E94E27E0E944683A7E28A2E912C9F
:10850000A12CB12CD12CC12C01E00093B30E809290
:10851000B50E1092B40E1092B60E81E00E94548DEA
:108520008111A9C18092FE13FFEFCF1ADF0A2FEF4E
:10853000821A920AA20AB20A30E483169104A104B4
:10854000B10419F7CD2831F461E875E085E59FE0C5
:108550000E9412810E9446831092FF13809103149F
:10856000823018F098E09093FF13909104149923AF
:1085700039F0813029F48091FF1384608093FF13D8
:1085800062E370E080E090E00E94B38360910514A4
:108590008AEF93E10E94448E68EE73E080E090E001
:1085A0000E94B38360E38AEF93E10E94588E7BE4DC
:1085B000C72E76E4D72EC6010197F1F760E38AEF64
:1085C00093E10E94588EC6010197F1F760E38AEFAC
:1085D00093E10E94588E83E592E00197F1F760E203
:1085E0008AEF93E10E94588E8091FF1380620E946F
:1085F000718E84E0809300148CE00E94718E81E083
:108600000E94718EEBE3CE2EEFE1DE2EC6010197C4
:10861000F1F782E08093011486E00E94718E82E07F
:108620000E94718EC6010197F1F780E40E94718E5D
:10863000FAE7CF2EF2E0DF2EF60161916F018AEFAB
:1086400093E10E94E08EF2E8CF16F2E0DF06A1F798
:108650000E94A00A0E94900A64E670E080E090E028
:108660000E94B38365E87AE0CE0101960E94E47F20
:10867000CE0101960E94E61FCE0101960E94577F0F
:1086800061E085E30E945D8361E085E30E944082B2
:1086900061E08AE00E945D8361E08AE00E9440829E
:1086A00061E089E30E945D838091E010803308F0EF
:1086B00052C061E089E30E945D838091E010282F21
:1086C00030E0F901EE0FFF1FE20FF31FE35BFF4EF7
:1086D0009081907C996390831092E1101092E21047
:1086E0002CE0622F0E94B4B3829FB00111249B0141
:1086F0002E0D3F1DF901EE0FFF1FE20FF31FE35B8D
:10870000FF4E908196FD19C02FEFE21AF20A3CE06D
:10871000E316F10461F7813009F0C4C010928000C3
:1087200082E0809381001092850010928400B19ABB
:1087300080916F00826080936F00E091E0108E2F37
:1087400090E0FC01EE0FFF1FE80FF91FE35BFF4E07
:1087500080818064808368EC70E080E090E00E941B
:10876000B38368EE73E080E090E00E94B38364E737
:108770007AE0CE0101960E94E47F4AE050E06FEF7C
:108780007FEFCE0101960E94F620CE0101960E9455
:10879000577F109209101092071010920410109237
:1087A000031084E0809302100E9482867B0161E0C6
:1087B000809102100E945D838EEF9FE00E94F50879
:1087C00060E082E30E945D8361E083E30E945D8359
:1087D00061E084E30E945D8361E085E30E945D8344
:1087E00061E085E30E94408283E58CBD8DB58E7F7C
:1087F0008DBD0AE08FEF0E947E070150D9F760E03F
:10880000809102100E94408220E030E0A90160E0E7
:108810008EEF9FE00E94D510082F809308108130C2
:1088200009F46CC00E9482866E197F09613D774011
:1088300058F381E0809303108EEF9FE00E94F508CB
:1088400066E67AE0CE0101960E94E47FCE010196B1
:108850000E94E61FCE0101960E94577F65E57AE0EF
:10886000CE0101960E94E47F6AE070E0CE0101969D
:108870000E94AF8E60C1843009F059CE66E675E083
:1088800085E59FE00E94268120E1B501A40185E5F0
:108890009FE00E9466806BEA79E085E59FE00E9498
:1088A000578045CE823061F4109290008093910001
:1088B000109295001092940088BB809371003DCF78
:1088C000833069F41092A00082E08093A10010929E
:1088D000A5001092A40089BB809372002ECF811155
:1088E0002CCF1092200182E080932101109225016B
:1088F000109224018ABB809373001FCF2AEA31E0D3
:1089000040E050E068E08EEF9FE00E94D51082FFCB
:108910002AC00093091080910910812C912C5401D8
:10892000823029F4812C912CA12C30E4B32E20E04C
:1089300030E0A90167E38EEF9FE00E94D510A5010A
:10894000940169E28EEF9FE00E94D5108093081099
:108950008823C1F00E9482866E197F09613D7740AD
:1089600030F388E067CF04E00E94D01080930810B5
:108970000150D1F78A3A11F082E05CCF82E0809317
:108980000910C9CF809109108230D1F420E030E085
:10899000A9016AE38EEF9FE00E94D510882311F0B1
:1089A00086E048CF0E94D010807C803C19F483E0A0
:1089B000809309100E94D0100E94D0100E94D01005
:1089C0008EEF9FE00E94F5088DB58E7F8DBD8CB532
:1089D0008C7F8CBD8CB58CBD81E00E94F09088238B
:1089E00009F464C180912D1081112ACF809121104A
:1089F000803109F062C182E080932D1010923F1007
:108A0000109240101092411010924210809122104A
:108A100090912310B0E0A0E025E0880F991FAA1FD5
:108A2000BB1F2A95D1F780933B1090933C10A093E5
:108A30003D10B0933E108AE090E1909344108093F3
:108A4000431081E080932C1010922E1010922F1062
:108A50001092301010923110109232101092331088
:108A60001092341010923510109236101092371068
:108A7000109238101092391010923A1069E47AE08E
:108A8000CE0101960E94E47FCE0101960E94E61F6E
:108A9000CE0101960E94577F41E06EE474E0CE0162
:108AA00001960E94A397BE016F5F7F4F83EC93E115
:108AB0000E9414208091C5139091C6139C838B83D0
:108AC0008091C7139091C813A091C913B091CA1394
:108AD0008D839E83AF83B8878091CB139091CC1305
:108AE000A091CD13B091CE1389879A87AB87BC87AD
:108AF0008EEE93E09A8389838DE0EFECF3E1DE0163
:108B00001D9601900D928A95E1F78091DC1390916A
:108B1000DD139B8F8A8F70E060E0CE0101960E948A
:108B2000C22163E47AE0CE0101960E94E47FCE0187
:108B300001960E94E61FCE0101960E94577F68EEC3
:108B400073E080E090E00E94B38343E160EB72E069
:108B5000CE0101960E94A397BE016F5F7F4F8EEDFD
:108B600093E10E9414206AE07AE088EE91E10E948D
:108B7000E27E6FEF79E088EE91E10E94857E8EEDD6
:108B800093E10E948B12882309F4B6C063EA70E176
:108B900080EB92E00E94A37B811122C067E975E01F
:108BA000CE0101960E94F67FCE0101960E94FD1F24
:108BB000CE0101960E94577F60EB72E0CE010196D4
:108BC0000E94F67FCE0101960E94E61FCE0101961B
:108BD0000E94577F68EE71E18EED93E10E943C8127
:108BE0008EED93E10E94971266E970E080E090E0DC
:108BF0000E94B38369EA75E0CE0101960E94F67F78
:108C0000CE0101960E94E61FCE0101960E94577F79
:108C100010927E0C64ED79E0CE0101960E94E47F13
:108C2000CE0101960E94E61FCE0101960E94577F59
:108C30000E9471846C0168EE73E080E090E00E9415
:108C4000B383F12CE12CCD2809F017C5EAE0EE162C
:108C5000F10409F462C0B701CE0101960E94447D7F
:108C6000CE0101960E94E61FCE0101960E94577F19
:108C700060ED77E080E090E00E94B3830E94718411
:108C80006C0168EE73E080E090E00E94B383CE0157
:108C900001960E94DE1EBE016F5F7F4F85E59FE05B
:108CA0000E94FC80FFEFEF1AFF0ACDCF80E00E9408
:108CB000F090882309F4C4CD95CE803209F0C0CD60
:108CC00083E080932D1040912410509125106091E5
:108CD00026107091271040933F10509340106093DE
:108CE0004110709342102BE330E18AE090E10E9442
:108CF0003C938111A0CEA4CD6AEE79E0CE0101961D
:108D00000E94E47FCE0101960E94FD1FCE010196D4
:108D10000E94577F60EB72E06FCF68EC79E0CE0184
:108D200001960E94E47FCE0101960E94E61FCE01CB
:108D300001960E94577F68EE73E080E090E00E9409
:108D4000B38363EA70E18DE692E00E94A37B8823FF
:108D500031F063E670E18DE692E00E94A37B66E964
:108D600070E080E090E00E94B38343E16DE672E042
:108D7000CE0101960E94A397BE016F5F7F4F8EEDDB
:108D800093E10E94142081E080937E0CCE01019635
:108D90000E94DE1EBE016F5F7F4F8EED93E10E9449
:108DA000FC808EED93E10E94971262E370E080E018
:108DB00090E00E94B38310927E0C0E94263268EEEF
:108DC00073E080E090E00E94B3830E94263194E635
:108DD000E92EF12C11110BC085E59FE00E948977E7
:108DE000182F64E170E080E090E00E94B38321E0FE
:108DF000E21AF10879F76BEA79E0CE0101960E9458
:108E0000E47FCE0101960E948F28CE0101960E9438
:108E1000577F81E0123709F080E00E941F0A61EA63
:108E200079E082E192E10E94E27ECE0101960E9409
:108E3000C228BE016F5F7F4F82E192E10E94DB7E1C
:108E4000CE0101960E94577F6EE879E082E192E1BF
:108E50000E94857E6CE779E0CE0101960E94E47F56
:108E6000CE0101960E948F28CE0101960E94577F65
:108E700068E370E080916B0290916C020E94C40ADA
:108E80009093E30B8093E20B62E172E1CE010196D5
:108E90000E94ED7FAE014F5F5F4F62E070E08EE5B4
:108EA00092E00E94812F182FCE0101960E94577FD9
:108EB000111121C062E172E1CE0101960E94ED7FA5
:108EC0006FEA75E0CE0101960E945C7E64EF71E16D
:108ED0000E94727EBC01CE014C960E94ED7FCE01B5
:108EE0004C960E94E61FCE014C960E94577FCE0101
:108EF00001960E94577F62E172E1CE0101960E94C5
:108F0000ED7FAE014F5F5F4F63E070E081E592E07F
:108F10000E94812F182FCE0101960E94577F1111B8
:108F200021C062E172E1CE0101960E94ED7F6FEAFD
:108F300075E0CE0101960E945C7E64EF71E10E94B3
:108F4000727EBC01CE014C960E94ED7FCE014C9604
:108F50000E94E61FCE014C960E94577FCE010196DB
:108F60000E94577F68EE73E080E090E00E94B38338
:108F700067E174E0CE01805C9F4F0E94F67F67E15D
:108F800074E0CE01CA960E94F67F67E174E0CE01DC
:108F9000C4960E94F67FB7ED8B2EB2E09B2E14E6AE
:108FA000E12E12E1F12E01ECA02E02E0B02E81EEB6
:108FB000682E82E0782E630101E010E0F401119246
:108FC00011924F0164E572E1CE0188960E94F67F0E
:108FD000B701CE0182960E94F67FB801CE014C9671
:108FE0000E94447D6BEB75E0CE0101960E94F67FF6
:108FF000BE01645E7F4FCE0101960E94727E65E4E1
:1090000077E00E945C7EBE016E5D7F4F0E94727EA3
:1090100064E676E00E945C7EBE01685D7F4F0E9440
:10902000727EBC01CE01805C9F4F0E94DB7ECE0130
:1090300001960E94577FCE014C960E94577FCE0129
:1090400082960E94577FCE0188960E94577FF50135
:1090500011921192119211925F01F60111921192E7
:10906000119211926F01C8010E94FA1E0F5F1F4FEB
:10907000F8E0EF0EF11C0430110509F09FCF7FECF2
:10908000A72E72E0B72EEDEBEE2EE2E0FE2EF9E415
:10909000CF2EF2E0DF2E01E010E0A8EE2A2EA3E0B2
:1090A0003A2E412C512CF501619171915F01CE0155
:1090B00088960E94447D42E050E0BE01685D7F4F8B
:1090C000CE018E960E94AF20B801CE014C960E9430
:1090D000447D42E050E0BE01645E7F4FCE01829647
:1090E0000E94AF2069E078E0CE0101960E94F67FF1
:1090F000BE016E5D7F4FCE0101960E94727EBE0161
:10910000625D7F4F0E94727EBC01CE01C4960E94B8
:10911000077FCE0101960E94577FCE0182960E9462
:10912000577FCE014C960E94577FCE018E960E94AB
:10913000577FCE0188960E94577FF7016481758121
:1091400086819781A20191010E9454B2BA01A901BE
:1091500020E0CE0101960E94957F48E050E0BE01DC
:109160006F5F7F4FCE014C960E94AF20BE01645EC0
:109170007F4FCE01C4960E94DB7ECE014C960E94AA
:10918000577FCE0101960E94577FF6016191719140
:109190006F01CE0101960E94447D43E050E0BE0184
:1091A0006F5F7F4FCE014C960E94AF20BE01645E80
:1091B0007F4FCE01C4960E94DB7ECE014C960E946A
:1091C000577FCE0101960E94577FBE016C5C7F4F96
:1091D000CE01CA960E94DB7EF701148215821682A8
:1091E0001782F30111921192119211923F01C8015D
:1091F0000E94FA1E0F5F1F4FF4E0EF0EF11C0430C7
:10920000110509F050CFCE014C960E94C2286FEB99
:1092100075E0CE0101960E94F67FBE01645E7F4F2D
:10922000CE0101960E94727E61E676E00E945C7E2D
:10923000BE01605C7F4F0E94727EBC0182E192E1C0
:109240000E94077FCE0101960E94577FCE014C9667
:109250000E94577FCE0101960E94C22846E150E04D
:10926000BE016F5F7F4FCE014C960E94AF20BE01C2
:10927000645E7F4FCE0182960E94ED7FBE01665CE8
:109280007F4FCE0182960E94727EBC01CE01CA96AB
:109290000E94077FCE0182960E94577FCE014C9696
:1092A0000E94577FCE0101960E94577F62E172E1D2
:1092B000CE0101960E94ED7FCE0101960E94E61F2D
:1092C000CE0101960E94577F62E172E1CE010196C4
:1092D0000E94ED7FAE014F5F5F4F62E070E08EE570
:1092E00092E00E94812F182FCE0101960E94577F95
:1092F000111121C062E172E1CE0101960E94ED7F61
:109300006FEA75E0CE0101960E945C7E64EF71E128
:109310000E94727EBC01CE014C960E94ED7FCE0170
:109320004C960E94E61FCE014C960E94577FCE01BC
:1093300001960E94577FBE01665C7F4FCE01019669
:109340000E94ED7FAE014F5F5F4F63E070E081E50B
:1093500092E00E94812FCE0101960E94577FCE019C
:10936000C4960E94577FCE01CA960E94577FCE01B5
:10937000805C9F4F0E94577F64EF71E080E090E037
:109380000E94B38382E090E00E94208B83E090E013
:109390000E94208B01E010E0109389020093880264
:1093A0001093500200934F0269EC75E083EA91E15B
:1093B0000E943A7D1093500200934F0263EA71E1DC
:1093C000CE0101960E94ED7F62E070E0CE01019631
:1093D0000E94DE37CE0101960E94577F6BE679E04E
:1093E000CE0101960E94E47FCE0101960E94E61F05
:1093F000CE0101960E94577F6BE579E0CE01019680
:109400000E94E47FCE0101960E948F28CE01019632
:109410000E94577F67E177E083EA91E10E943A7DFD
:1094200063EA71E1CE0101960E94ED7F63E070E096
:10943000CE0101960E94DE37CE0101960E94577F31
:1094400082E090E090938902809388026AE479E058
:10945000CE0101960E94E47FCE0101960E94E61F94
:10946000CE0101960E94577F6EE379E0CE0101960E
:109470000E94E47FCE0101960E948F28CE010196C2
:109480000E94577F69EC75E083EA91E10E943A7D82
:1094900080916E1390916F1397FF06C06DEC75E08D
:1094A00083EA91E10E943A7D63EA71E1CE0101967F
:1094B0000E94ED7F62E070E0CE0101960E94DE37EF
:1094C000CE0101960E94577F67E177E083EA91E140
:1094D0000E943A7D82E090E0909389028093880216
:1094E00063EA71E1CE0101960E94ED7F63E070E0D6
:1094F000CE0101960E94DE37CE0101960E94577F71
:1095000080916E1390916F1391958195910990932D
:109510006F1380936E1301E010E0109350020093DC
:109520004F0284EF91E0909383028093820268E47B
:1095300072E10E94EE0964E670E080E090E00E9433
:10954000B383109389020093880280E090E79093A0
:10955000581180935711209179112830D8F4822F17
:1095600090E0FC01EE0FFF1FEE0FFF1FE75AFE4ECB
:1095700041ED55E0518340832F5F20937911880F8F
:10958000991F880F991FFC01E55AFE4E82E493E271
:1095900091838083209179112830D8F4822F90E034
:1095A000FC01EE0FFF1FEE0FFF1FE75AFE4E47EDC7
:1095B00055E0518340832F5F20937911880F991FC5
:1095C000880F991FFC01E55AFE4E8AE596E79183C4
:1095D000808387EE90E10E94DC1D6CE279E0CE0191
:1095E00001960E94E47FCE0101960E94E61FCE0103
:1095F00001960E94577F0E94DA8A60930E0C709346
:109600000F0C8093100C9093110C1092120C0E946E
:1096100050280E94DA8A6093290C70932A0C809358
:109620002B0C90932C0C809147138093800C8823F3
:1096300051F00E94DA8A6093210C7093220C80937F
:10964000230C9093240CCB5BDF4F0FB6F894DEBF56
:109650000FBECDBFDF91CF911F910F91FF90EF9083
:10966000DF90CF90BF90AF909F908F907F906F9042
:109670005F904F903F902F9008956BEB79E04FCB28
:109680002F923F924F925F926F927F928F929F9212
:10969000AF92BF92CF92DF92EF92FF920F931F9300
:1096A000CF93DF93CDB7DEB7E3970FB6F894DEBF65
:1096B0000FBECDBF61EC71E1CE018E960E94ED7FB1
:1096C0000EA51FA50115110571F0D8018D918D0111
:1096D000882349F0082E000C990B0E9402B6F8016D
:1096E00031978083F2CF6BED75E0CE0101960E9439
:1096F000F67FBE016F5F7F4FCE018E960E94417E46
:10970000182FCE0101960E94577F112309F401C141
:1097100045E050E061EC71E1CE0101960E94A3208A
:10972000BE016F5F7F4F83EA91E10E941E7FCE01F1
:1097300001960E94577F83EA91E10E94B37D60E029
:1097400083EA91E10E94AF7E4091A7115091A81148
:1097500060EA72E183EA91E10E946B7B6EE474E05F
:10976000CE0101960E94F67FBE016F5F7F4F83EAB4
:1097700091E10E94417E182FCE0101960E94577FF1
:1097800068E374E0111102C06DE374E0CE0101964C
:109790000E94F67F63EA71E1CE0101960E94727E1B
:1097A000BC0182EA93E10E94077FCE0101960E94EC
:1097B000577F82EA93E10E94B37D4091A6135091B6
:1097C000A7134150510962EA73E1CE0101960E944C
:1097D000A320BE016F5F7F4F84E893E10E941E7F4C
:1097E000CE0101960E94577F84E893E10E94A87DF4
:1097F0000E94EFB09B01AC010E94AFB3882309F433
:1098000048C06091A6137091A7136250710982EA53
:1098100093E10E94107E682FCE0101960E94C27FC4
:10982000BE016F5F7F4F84E893E10E941E7FCE01EF
:1098300001960E94577F6EE474E0CE0101960E946B
:10984000F67FBE016F5F7F4F84E893E10E94417E07
:10985000182FCE0101960E94577F1123D1F06091FD
:10986000A6137091A7136350710982EA93E10E94D5
:10987000107E682FCE0101960E94C27FBE016F5FED
:109880007F4F84E893E10E941E7FCE0101960E94E3
:10989000577F84EF91E0909383028093820268E483
:1098A00072E10E94EE0964E670E080E090E00E94C0
:1098B000B38380913002882371F061EC71E1CE01B5
:1098C00001960E94ED7FCE0101960E945826CE019E
:1098D00001960E94577FCE018E960E94577F81E0AD
:1098E000E3960FB6F894DEBF0FBECDBFDF91CF91E8
:1098F0001F910F91FF90EF90DF90CF90BF90AF90AE
:109900009F908F907F906F905F904F903F902F909F
:10991000089561EE75E0CE0101960E94F67FBE01CA
:109920006F5F7F4FCE018E960E94417E182FCE0131
:1099300001960E94577F112309F447C045E050E08B
:1099400061EC71E1CE0101960E94A320BE016F5F20
:109950007F4F83EA91E10E941E7FCE0101960E9413
:10996000577F83EA91E10E94B37D60E083EA91E151
:109970000E94AF7E4091A7115091A81168E772E153
:1099800083EA91E10E946B7B68E772E1CE014C961D
:109990000E94F67F60E574E0CE0101960E94F67F9A
:1099A000BE01645E7F4FCE0101960E94727EBC01B3
:1099B0008CE993E10E94077FCE0101960E94577FB8
:1099C000CE014C960E94577F64CF67EE75E0CE01C2
:1099D00001960E94F67FBE016F5F7F4FCE018E968B
:1099E0000E94417E182FCE0101960E94577F1123BD
:1099F000E1F043E050E061EC71E1CE0101960E949C
:109A0000A320BE016F5F7F4F83EA91E10E941E7F1A
:109A1000CE0101960E94577F63EA71E1CE01019663
:109A20000E94ED7FCE010196CDCF6BEE75E0CE01A9
:109A300001960E94F67FBE016F5F7F4FCE018E962A
:109A40000E94417E182FCE0101960E94577F11235C
:109A500001F144E050E061EC71E1CE0101960E9419
:109A6000A320BE016F5F7F4F83EA91E10E941E7FBA
:109A7000CE0101960E94577F83EA91E10E94A87D62
:109A8000709307136093061370936C0260936B02DC
:109A900000CF60EF75E0CE0101960E94F67FBE0117
:109AA0006F5F7F4FCE018E960E94417E182FCE01B0
:109AB00001960E94577F112309F449C045E050E008
:109AC00061EC71E1CE0101960E94A320BE016F5F9F
:109AD0007F4F83EA91E10E941E7FCE0101960E9492
:109AE000577F83EA91E10E94A87D7093631360938E
:109AF000621384EF91E0909383028093820268E482
:109B000072E10E94EE0964E670E080E090E00E945D
:109B1000B38369E078E0CE0101960E94F67F61ECA4
:109B200071E1CE0101960E94727EBC01CE014C967D
:109B30000E94ED7FCE014C960E94E61FCE014C960E
:109B40000E94577FCE0101960E94577FB2CE66EFEA
:109B500075E0CE0101960E94F67FBE016F5F7F4FD8
:109B6000CE018E960E94417E182FCE0101960E9452
:109B7000577F1123E1F044E050E061EC71E1CE0148
:109B800001960E94A320BE016F5F7F4F83EA91E19F
:109B90000E941E7FCE0101960E94577F83EA91E1C9
:109BA0000E94A87D7093651360936413A2CF6BEF3E
:109BB00075E0CE0101960E94F67FBE016F5F7F4F78
:109BC000CE018E960E94417E182FCE0101960E94F2
:109BD000577F1123A1F044E050E061EC71E1CE0128
:109BE00001960E94A320BE016F5F7F4F83EA91E13F
:109BF0000E941E7FCE0101960E94577F84CF60E0B5
:109C000076E0CE0101960E94F67FBE016F5F7F4F26
:109C1000CE018E960E94417E182FCE0101960E94A1
:109C2000577F1123A1F047E050E061EC71E1CE01D4
:109C300001960E94A320BE016F5F7F4F83EA91E1EE
:109C40000E941E7FCE0101960E94577F2CCE68E0B5
:109C500076E0CE0101960E94F67FBE016F5F7F4FD6
:109C6000CE018E960E94417E182FCE0101960E9451
:109C7000577F1111D8CF60E176E0CE0101960E94A6
:109C8000F67FBE016F5F7F4FCE018E960E94417EB0
:109C9000182FCE0101960E94577F112321F081E0F9
:109CA0000E941F0A00CE6AE176E0CE0101960E9472
:109CB000F67FBE016F5F7F4FCE018E960E94417E80
:109CC000182FCE0101960E94577F112319F00E9490
:109CD0002631E9CD62E279E0CE0101960E94E47F6F
:109CE000BE016F5F7F4FCE018E960E94417E182F7E
:109CF000CE0101960E94577F112309F485C067E1C8
:109D000079E0CE0101960E94E47FBE016F5F7F4F34
:109D1000CE018E960E94417E182FCE0101960E94A0
:109D2000577F112309F454C04AE050E061EC71E11F
:109D3000CE0101960E94A320BE016F5F7F4F83EA90
:109D400091E10E941E7FCE0101960E94577F83EA17
:109D500091E10E94A87D0E94B58A0E94DA8A6093F0
:109D6000210C7093220C8093230C9093240C0E945E
:109D7000DA8A6093250C7093260C8093270C9093BD
:109D8000280CCE014C960E94C22861E276E0CE01FA
:109D900001960E94F67FBE01645E7F4FCE01019660
:109DA0000E94727EBC01CE0182960E94ED7FCE01A0
:109DB00082960E94E61FCE0182960E94577FCE01B6
:109DC00001960E94577FCE014C960E94577F71CD1D
:109DD0004BE050E061EC71E1CE0101960E94A320BE
:109DE000BE016F5F7F4F83EA91E10E941E7FCE012B
:109DF00001960E94577F83EA91E10E94A87D6058F6
:109E00007F488F4F9F4FA7CF69E877E0CE0101963B
:109E10000E94F67FBE016F5F7F4FCE018E960E943B
:109E2000417E182FCE0101960E94577F112309F41D
:109E30006AC045E050E061EC71E1CE0101960E94FC
:109E4000A320BE016F5F7F4F83EA91E10E941E7FD6
:109E5000CE0101960E94577F0E94DA8A6093210CFE
:109E60007093220C8093230C9093240C83EA91E14D
:109E70000E94A87D60938A0270938B0280938C026B
:109E800090938D02609348137093491380934A1303
:109E900090934B13209147132093800C672B682BD2
:109EA000692B11F41092800C84EF91E0909383025F
:109EB0008093820268E472E10E94EE0964E670E039
:109EC00080E090E00E94B38368E079E0CE010196E3
:109ED0000E94E47FCE0101960E94FD1FCE010196F3
:109EE0000E94577F40918A0250918B0260918C02B0
:109EF00070918D02CE0101960E94707DCE01019677
:109F00000E94E61FCCC162E376E0CE0101960E947A
:109F1000F67FBE016F5F7F4FCE018E960E94417E1D
:109F2000182FCE0101960E94577F1123D9F14AE0E4
:109F300050E061EC71E1CE0101960E94A320BE01C8
:109F40006F5F7F4F83EA91E10E941E7FCE010196F1
:109F50000E94577F83EA91E10E94A87D61307105DC
:109F60008105910519F481E08093471383EA91E11B
:109F70000E94A87D672B682B692B11F41092471360
:109F8000809147138093800C882309F4B2CD0E94FE
:109F9000DA8A6093210C7093220C8093230C9093A7
:109FA000240CA7CD6DE376E0CE0101960E94F67FEA
:109FB000BE016F5F7F4FCE018E960E94417E182FAB
:109FC000CE0101960E94577F1123A1F048E050E096
:109FD00061EC71E1CE0101960E94A320BE016F5F8A
:109FE0007F4F83EA91E10E941E7FCE0101960E947D
:109FF000577F8FCD66E476E0CE0101960E94F67F12
:10A00000BE016F5F7F4FCE018E960E94417E182F5A
:10A01000CE0101960E94577F112321F145E050E0C7
:10A0200061EC71E1CE0101960E94A320BE016F5F39
:10A030007F4F83EA91E10E941E7FCE0101960E942C
:10A04000577F83EA91E10E94A87D6130710521F478
:10A0500081E08093810C2DCC672B09F02ACC1092E3
:10A06000810C27CC6CE476E0CE0101960E94F67F4D
:10A07000BE016F5F7F4FCE018E960E94417E182FEA
:10A08000CE0101960E94577F112309F46AC066E051
:10A0900070E081EC91E10E94107E682FCE01019664
:10A0A0000E94C27FBE016F5F7F4F83EA91E10E94F1
:10A0B0001E7FCE0101960E94577F83EA91E10E94A4
:10A0C000B37D60E083EA91E10E94AF7E83EA91E193
:10A0D0000E94A87D6B01CB010197039708F0E9CBA3
:10A0E00048E050E061EC71E1CE0101960E94A320AE
:10A0F000BE016F5F7F4F83EA91E10E941E7FCE0118
:10A1000001960E94577F83EA91E10E94B37D80917E
:10A11000A7119091A8110997A8F028E030E050E02D
:10A1200040E063EA71E1CE0101960E940B80BE011E
:10A130006F5F7F4F83EA91E10E941E7FCE010196FF
:10A140000E94577FB60113E0660F771F1A95E1F75B
:10A15000645A7D4E48E050E083EA91E10E946B7BB7
:10A1600098CB61E079E0CE0101960E94E47FBE01C8
:10A170006F5F7F4FCE018E960E94417E182FCE01D9
:10A1800001960E94577F112309F4BCC064E676E073
:10A19000CE0101960E94F67F46E050E0BE016F5F5F
:10A1A0007F4FCE018E960E94C1A68C01CE010196F2
:10A1B0000E94577F980146E050E0BE01625D7F4FEC
:10A1C000CE0101960E940B80CE0101960E94A87DCF
:10A1D0006B01CE0101960E94577F67E174E0CE01CA
:10A1E00001960E94F67FA8014F5F5F4FBE01625D3E
:10A1F0007F4FCE014C960E94A320BE01645E7F4F2C
:10A20000CE0101960E941E7FCE014C960E94577F80
:10A2100063E576E0CE014C960E94F67FBE01645E57
:10A220007F4FCE0101960E94417E182FCE014C96A1
:10A230000E94577F1123B1F141E050E0BE016F5FF2
:10A240007F4FCE014C960E94A320CE014C960E94D7
:10A25000A87D8B010A5C1F4FCE014C960E94577F50
:10A26000F6013196EE0FFF1FE85BFD4E1183008370
:10A27000F601EE0FFF1FE652F44F1183008384EFC7
:10A2800091E0909383028093820268E472E10E94DD
:10A29000EE0964E670E080E090E00E94B383CE01B6
:10A2A000019693CD62E077E0CE014C960E94F67F56
:10A2B000BE01645E7F4FCE0101960E94417E182F41
:10A2C000CE014C960E94577F112379F041E050E077
:10A2D000BE016F5F7F4FCE014C960E94A320CE013E
:10A2E0004C960E94A87D8B01B7CFCE0101960E94AB
:10A2F000A87D0091DC0B1091DD0B01501109060FB8
:10A30000171FAECF61E374E0CE014C960E94F67F3A
:10A31000BE01645E7F4FCE018E960E94417E11E0A9
:10A32000811115C065E576E0CE0101960E94F67FA9
:10A33000BE016F5F7F4FCE018E960E94417E11E07D
:10A34000811101C010E0CE0101960E94577FCE011D
:10A350004C960E94577F112309F411C261E676E002
:10A36000CE014C960E94F67F6CE576E0CE01019618
:10A370000E94F67FAE01445E5F4FBE016F5F7F4F6C
:10A38000CE018E960E94C8A5CE0101960E94577FED
:10A39000CE014C960E94577F61E676E0CE014C9646
:10A3A0000E94F67F6EE576E0CE0101960E94F67F70
:10A3B000AE01445E5F4FBE016F5F7F4FCE018E9650
:10A3C0000E94C8A5CE0101960E94577FCE014C96EF
:10A3D0000E94577F61E676E0CE014C960E94F67FA0
:10A3E00060E676E0CE0101960E94F67FAE01445E03
:10A3F0005F4FBE016F5F7F4FCE018E960E94C8A552
:10A40000CE0101960E94577FCE014C960E94577F45
:10A4100064E676E0CE014C960E94F67F63E676E035
:10A42000CE0101960E94F67FAE01445E5F4FBE01F1
:10A430006F5F7F4FCE018E960E94C8A5CE01019618
:10A440000E94577FCE014C960E94577F64E676E0CB
:10A45000CE014C960E94F67F61EA78E0CE0101962B
:10A460000E94F67FAE01445E5F4FBE016F5F7F4F7B
:10A47000CE018E960E94C8A5CE0101960E94577FFC
:10A48000CE014C960E94577FCE018E960E94B37DDE
:10A490000E94DA8A60930E0C70930F0C8093100C5C
:10A4A0009093110C56E0E52EF12C64E6462E512CCB
:10A4B000612C712C22242394312C5701B3E0AB0E74
:10A4C000B11C8AA99BA90197A816B90608F0F1C981
:10A4D000B701CE018E960E94107E682FCE014C9659
:10A4E0000E94C27F6701E2E0CE0ED11CFFEFEF1A9F
:10A4F000FF0A9601A701BE01625D7F4FCE01019662
:10A500000E940B80CE0101960E94A87D8B01CE0196
:10A5100001960E94577F0130110521F400916213CA
:10A52000109163130330110521F40091641310910D
:10A53000651361E676E0CE0101960E94F67FA601E2
:10A54000BE016F5F7F4FCE018E960E94C1A66C0147
:10A55000CE0101960E94577F67E174E0CE0101961B
:10A560000E94F67F480181E0881A91081C141D049E
:10A570002CF59601A501BE01625D7F4FCE0182964A
:10A580000E940B80BE016E5D7F4FCE0101960E943E
:10A590001E7FCE0182960E94577F93E08916910418
:10A5A00020F17601AFEFEA1AFA0ACE0101960E9475
:10A5B000577FCE014C960E94577F7FCFA501BE01E9
:10A5C000625D7F4FCE0182960E94A320BE016E5D28
:10A5D0007F4FCE0101960E941E7FCE0182960E947F
:10A5E000577FB3E08B16910400F770E060E0CE0176
:10A5F0004C960E94107E823509F061C0CE01019612
:10A600000E94A87D672B682B692BB1F4F801EE0F2F
:10A61000FF1FEB52FD4F11821082F801EE0FFF1F5A
:10A62000EE0FFF1FE354FD4F82E090E0A0E0B0E0AA
:10A6300080839183A283B383CE0101960E94A87D7B
:10A640006130710581059105A9F5F801EE0FFF1F35
:10A65000EB52FD4F31822082000F111F000F111F9E
:10A66000F801E354FD4F80819181A281B3811816D6
:10A6700019061A061B0624F04082518262827382F8
:10A68000CE0101960E94A87D623071058105910579
:10A690003CF0F801E354FD4F608371838283938320
:10A6A0000E94DA8A03521D4FD8016D937D938D93DA
:10A6B0009C9313971C141D040CF473CF76CF86342F
:10A6C000E9F5CE0101960E94A87D672B682B692BC6
:10A6D00039F4F801EE0FFF1FE95BFD4F1182108284
:10A6E000CE0101960E94A87D61307105810591051A
:10A6F00039F4F801EE0FFF1FE95BFD4F3182208234
:10A70000000F111F000F111FF801E354FD4F80814E
:10A710009181A281B381181619061A061B0624F02E
:10A7200040825182628273820E94DA8A03521D4FF4
:10A73000F8016083718382839383BCCF843461F496
:10A74000CE0101960E94A87D000F111F000F111F5E
:10A75000F801E95CFD4FA0CF843509F0ABCFCE0105
:10A7600001960E94A87D000F111F000F111FF80114
:10A77000E354FD4F6083718382839383D5CF6BEF66
:10A7800078E0CE0101960E94E47FBE016F5F7F4FAB
:10A79000CE018E960E94417E182FCE0101960E9416
:10A7A000577F112309F49CC045E050E061EC71E152
:10A7B000CE0101960E94A320BE016F5F7F4F83EA06
:10A7C00091E10E941E7FCE0101960E94577F83EA8D
:10A7D00091E10E94B37D60E083EA91E10E94AF7E47
:10A7E0006DEA75E0CE014C960E94F67F63EA71E156
:10A7F000CE0101960E94ED7FAE014E5D5F4FBE011E
:10A80000645E7F4FCE0101960E94DDA6182FCE0117
:10A8100001960E94577FCE014C960E94577F1123CC
:10A8200009F447C88E010E5D1F4F52E7A52E53E174
:10A83000B52E63E3C62E62E0D62EF12CE12CD801B2
:10A840006D918D01F50161935F01D6016D936D01ED
:10A85000CE0101960E9450A5CE0101960E94FD1FD7
:10A86000CE0101960E94577FB3E0EB16F10471F020
:10A870006DEA75E0CE0101960E94F67FCE01019649
:10A880000E94FD1FCE0101960E94577FEFEFEE1A46
:10A89000FE0AF4E0EF16F10491F667E174E0CE01F0
:10A8A00001960E94F67FCE0101960E94E61FCE011E
:10A8B00001960E94577F68E472E180918202909134
:10A8C00083020E94EE0964E670E080E090E00E945E
:10A8D000B38363EE78E0CE0101960E94E47F0ECB55
:10A8E0006EED78E0CE0101960E94E47FBE016F5FBD
:10A8F0007F4FCE018E960E94417E182FCE01019689
:10A900000E94577F112309F47CC044E050E061ECC1
:10A9100071E1CE0101960E94A320BE016F5F7F4FBF
:10A9200083EA91E10E941E7FCE0101960E94577F2B
:10A9300083EA91E10E94B37D60E083EA91E10E94A5
:10A94000AF7E4091A7115091A8116AEC7BE083EA99
:10A9500091E10E946B7B6DEA75E0CE014C960E94FE
:10A96000F67F63EA71E1CE0101960E94ED7FAE01B0
:10A970004E5D5F4FBE01645E7F4FCE0101960E9427
:10A98000DDA6182FCE0101960E94577FCE014C966E
:10A990000E94577F112311F40C94594C8E010E5DC7
:10A9A0001F4F44E7E42E42E1F42E6E0186E2C80E0A
:10A9B000D11CD8016D918D01F70161937F01CE010A
:10A9C00001960E9450A5CE0101960E94E61FCE017D
:10A9D00001960E94577FC016D10659F784EF91E087
:10A9E000909383028093820268E472E10E94EE09F0
:10A9F00064E670E080E090E00E94B38363ED78E06D
:10AA00006ACF6CEC78E0CE0101960E94E47FBE0133
:10AA10006F5F7F4FCE018E960E94417E182FCE0130
:10AA200001960E94577F1123F1F146E050E061EC5E
:10AA300071E1CE0101960E94A320BE016F5F7F4F9E
:10AA400083EA91E10E941E7FCE0101960E94577F0A
:10AA500083EA91E10E94B37D8091A7119091A811A2
:10AA6000892B11F40C94594C83EA91E10E94A87D42
:10AA7000709371136093701370933202609331027C
:10AA800084EF91E0909383028093820268E472E104
:10AA90000E94EE0964E670E080E090E00E94B383DB
:10AAA00068EB78E018CF66E676E0CE0101960E946A
:10AAB000F67FBE016F5F7F4FCE018E960E94417E72
:10AAC000182FCE0101960E94577F1123A9F06BEA3F
:10AAD00078E0CE0101960E94E47F64E670E0CE014A
:10AAE00001960E94AF8ECE0101960E94577FF0E042
:10AAF000E0E019950C94594C6DE676E0CE014C9649
:10AB00000E94F67FBE01645E7F4F81EC91E10E945E
:10AB1000417E11E0811115C065E776E0CE01019616
:10AB20000E94F67FBE016F5F7F4F81EC91E10E9432
:10AB3000417E11E0811101C010E0CE0101960E941A
:10AB4000577FCE014C960E94577F112389F16DE704
:10AB500076E0CE0101960E94F67F6AE873E1CE01AD
:10AB600001960E94727EBC0189EA91E10E94077FF2
:10AB7000CE0101960E94577F69E078E0CE010196F0
:10AB80000E94F67F69EA71E1CE0101960E94727E11
:10AB9000BC01CE014C960E94ED7FCE014C960E94E6
:10ABA000E61FCE014C960E94577FCE0101966CC5E0
:10ABB00067E876E0CE014C960E94F67FBE01645EA7
:10ABC0007F4F81EC91E10E94417E11E0811115C01F
:10ABD0006EE876E0CE0101960E94F67FBE016F5FBF
:10ABE0007F4F81EC91E10E94417E11E0811101C013
:10ABF00010E0CE0101960E94577FCE014C960E9434
:10AC0000577F112369F06DE978E089EA91E10E94AC
:10AC1000E27E60E973E189EA91E10E94DB7EACCFDC
:10AC200065E976E0CE0101960E94F67FBE016F5F76
:10AC30007F4FCE018E960E94417E182FCE01019645
:10AC40000E94577F112331F00E9426321092300269
:10AC50000C94594C6EE976E0CE014C960E94F67F3A
:10AC6000BE01645E7F4F81EC91E10E94417E11E064
:10AC7000811115C063EA76E0CE0101960E94F67F4D
:10AC8000BE016F5F7F4F81EC91E10E94417E11E038
:10AC9000811101C010E0CE0101960E94577FCE01C4
:10ACA0004C960E94577F112309F441C064E676E078
:10ACB000CE0101960E94F67F4091C5115091C611B8
:10ACC0008D819E81481B590BBE016F5F7F4F81ECC8
:10ACD00091E10E947AA5AC014F5F5F4F61EC71E199
:10ACE000CE014C960E94A320BE01645E7F4F83EA92
:10ACF00091E10E941E7FCE014C960E94577FCE01AB
:10AD000001960E94577F83EA91E10E94A87D611518
:10AD1000710531F481E08093EE020E944F9A96CF44
:10AD20006130710509F092CF1092EE02F6CF68EA19
:10AD300076E0CE0101960E94F67FBE016F5F7F4FE5
:10AD4000CE018E960E94417E182FCE0101960E9460
:10AD5000577F112309F43BC143E050E061EC71E1FE
:10AD6000CE0101960E94A320BE016F5F7F4F83EA50
:10AD700091E10E941E7FCE0101960E94577F63EAF7
:10AD800071E1CE0101960E94ED7FCE0101960E94F5
:10AD90005826CE0101960E94577F84EF91E0909350
:10ADA00083028093820263EA71E1CE0101960E94E0
:10ADB000ED7F60E0CE0101960E94C37EBC0186E972
:10ADC00093E10E94077FCE0101960E94577F63EABC
:10ADD00071E1CE0101960E94ED7F60E0CE01019607
:10ADE0000E94C37EBC0180E993E10E94077FCE01EF
:10ADF00001960E94577F40919A1350919B1368E0EF
:10AE000073E186E993E10E946B7B4091941350912A
:10AE1000951363E173E180E993E10E946B7B68E441
:10AE200072E180918202909183020E94EE096CEAA5
:10AE300076E0CE0101960E94F67F63EA71E1CE01D1
:10AE400001960E94727EBC01CE0182960E94ED7F27
:10AE5000CE0101960E94577F8091041390910513B3
:10AE6000892B39F4BE016E5D7F4F88EB9EE00E9416
:10AE70002E8168EB7BE080E090E00E94B3838091BC
:10AE8000041390910513029709F087C063EA71E1FA
:10AE9000CE0188960E94ED7F64EB76E0CE010196AC
:10AEA0000E94F67FCE0101960E947B9ACE01019608
:10AEB0000E94577F64EF71E080E090E00E94B383CE
:10AEC00067EB76E0CE0101960E94F67FCE010196F7
:10AED0000E947B9ACE0101960E94577F6CED75E02F
:10AEE00080E090E00E94B38360EC76E0CE010196B2
:10AEF0000E94F67FCE0101960E947B9ACE010196B8
:10AF00000E94577F64EF71E080E090E00E94B3837D
:10AF10006EEC76E0CE0101960E94F67FCE0101969E
:10AF20000E947B9ACE0101960E94577F64EF71E0E8
:10AF300080E090E00E94B3836CEA76E0CE01019657
:10AF40000E94F67FBE01685D7F4FCE0101960E9490
:10AF5000727EBC01CE014C960E94ED7FCE0101961F
:10AF60000E94577FCE014C960E94B37DBE01645E65
:10AF70007F4FCE0101960E94ED7FCE0101960E9487
:10AF80007B9ACE0101960E94577FCE014C960E947B
:10AF9000577FCE0188960E94577F68EB7BE080E068
:10AFA00090E00E94B38368E073E1CE0101960E94B5
:10AFB000F67FCE0101960E945826CE0101960E948E
:10AFC000577F10923002CE0182960C94E54E6CEDC4
:10AFD00076E0CE0101960E94F67FBE016F5F7F4F43
:10AFE000CE018E960E94417E182FCE0101960E94BE
:10AFF000577F112309F486C044E050E061EC71E111
:10B00000CE0101960E94A320BE016F5F7F4F83EAAD
:10B0100091E10E941E7FCE0101960E94577F61EE52
:10B0200076E0CE0101960E94F67F63EA71E1CE01DF
:10B0300001960E94727EBC01CE014C960E94ED7F6B
:10B04000CE0101960E94577F8091041390910513C1
:10B05000892B39F4BE01645E7F4F88EB9EE00E942D
:10B060002E8168E873E180E090E00E94B3838091D4
:10B07000041390910513029759F568EE76E0CE011E
:10B0800001960E94F67F8091A7119091A811892BBB
:10B0900019F561EF76E0CE0101960E943A7DBE017E
:10B0A000645E7F4FCE0182960E94ED7FCE01829634
:10B0B0000E947B9ACE0182960E94577F68E873E1D6
:10B0C00080E090E00E94B383CE0101960E94577FFA
:10B0D000109230020C94E34EBE016F5F7F4FCE01A1
:10B0E00082960E94ED7FCE0182960E947B9ACE01CD
:10B0F00082960E94577F60E777E180E090E00E94AF
:10B10000B383CDCF6AEF76E0CE0101960E94F67F41
:10B11000BE016F5F7F4FCE018E960E94417E182F39
:10B12000CE0101960E94577F112309F462C061ECA1
:10B1300071E183EA91E10E94077F81E08093300210
:10B1400061EC71E1CE0101960E94ED7FCE01019686
:10B150000E945826CE0101960E94577F80910413C9
:10B1600090910513029709F163EA71E188EB9EE083
:10B170000E942E8168EB7BE080E090E00E94B38328
:10B18000CE0101960E94149BBE016F5F7F4F81EC40
:10B1900091E10E941E7FCE0101960E94577F60EDD3
:10B1A00077E080E090E00E94B38380910413909157
:10B1B0000513029771F463EA71E1CE0101960E94D2
:10B1C000ED7FCE0101960E947B9ACE0101960E94EE
:10B1D000577F8091C5119091C611892B09F436CD06
:10B1E00069E078E0CE0101960E94F67F61EC71E1A2
:10B1F000CBCC6EEF76E0CE0101960E94F67FBE01C9
:10B200006F5F7F4FCE018E960E94417E182FCE0138
:10B2100001960E94577F112309F492C18091041373
:10B2200090910513019709F011CD64E077E0CE010C
:10B2300088960E94F67FBE01685D7F4F88EB9EE096
:10B240000E942E816CE271E080E090E00E94B38366
:10B25000CE0182960E94149B64E670E080E090E04C
:10B260000E94B38310E000E025E0C22ED12C3AE02A
:10B27000A32EB12C6FE077E0CE0101960E94F67FFD
:10B2800050E040E0BE016F5F7F4FCE0182960E948A
:10B29000C1A67C01CE0101960E94577FA7014F5F96
:10B2A0005F4FBE016E5D7F4FCE0101960E94A320CD
:10B2B000BE016F5F7F4FCE0188960E941E7FCE0138
:10B2C00001960E94577F8CA59DA5892B09F170E0FE
:10B2D00060E0CE0188960E94107E082E000C990B2B
:10B2E000C0970A97A8F461E177E0CE0101960E9429
:10B2F000F67FBE016F5F7F4FCE0188960E94417E30
:10B30000E82ECE0101960E94577FFF24F394E110AE
:10B31000F12C6CE377E0CE0101960E94E47F64E1BA
:10B3200070E0CE0101960E9497A7CE0101960E947F
:10B33000577F0F5F1F4F62E370E080E090E00E9454
:10B34000B383C801B6010E94C0B30197C1F4CE0116
:10B3500001960E9484268D819E81892B09F4BBC0B1
:10B36000BE016F5F7F4F81EC91E10E94077F0E94D9
:10B37000404BFF24F394CE0101960E94577FCE01EB
:10B3800001960E94149BBE016F5F7F4FCE01829693
:10B390000E941E7FCE0101960E94577F62E370E0FB
:10B3A00080E090E00E94B3830436110519F0FF207D
:10B3B00009F460CF80919D0B8823F1F069E078E07B
:10B3C000CE014C960E94F67FBE01685D7F4FCE0194
:10B3D0004C960E94727EBC01CE0101960E94ED7FC8
:10B3E000CE0101960E94E61FCE0101960E94577F72
:10B3F000CE014C960E94577F8CA59DA5892B69F0A4
:10B4000070E060E0CE0188960E94107E082E000C4D
:10B41000990BC0970A9708F477C069E177E0CE01ED
:10B4200001960E94F67FCE0182960E94577FCE0140
:10B4300088960E94577F8D819E81009709F446C0AF
:10B44000E981FA812081222309F440C00797F0F1B5
:10B4500064E978E0CE014C960E94E47F68EC70E0ED
:10B46000CE014C960E9497A7CE014C960E94577F22
:10B47000BE016F5F7F4FCE014C960E94ED7F60ED65
:10B4800077E0CE014C960E94AF8ECE014C960E9482
:10B49000577F65E277E0CE014C960E94F67F61EC23
:10B4A00071E1CE014C960E94727EBC01CE01829663
:10B4B0000E94ED7FCE0182960E94E61FCE01829609
:10B4C0000E94577FCE014C960E94577FCE01019675
:10B4D0000E94577FBBCB043111050CF44CCFC8013F
:10B4E000B5010E94C0B3892B09F045CFBE01685D4C
:10B4F0007F4F88EB9EE00E942E8168EC70E080E038
:10B5000090E00E94B38337CF61E177E0CE010196EE
:10B510000E94F67FBE016F5F7F4FCE0188960E942A
:10B52000417E182FCE0101960E94577F111175CFD1
:10B53000BE01685D7F4FCE0101960E94DB7F73CF15
:10B5400063E377E0CE0101960E94F67FBE016F5F54
:10B550007F4FCE018E960E94417E182FCE0101961C
:10B560000E94577F112309F4E8C025E030E044E051
:10B5700050E061EC71E1CE0101960E940B80BE01AA
:10B580006F5F7F4F83EA91E10E941E7FCE0101969B
:10B590000E94577F61EC71E1CE0101960E94ED7F20
:10B5A000CE0101960E945826CE0101960E94577F37
:10B5B00083EA91E10E94A87D6130710509F067C0BE
:10B5C00070930513609304136BE677E0CE01019648
:10B5D0000E94E47FCE0101960E945826CE0101967A
:10B5E0000E94577F68E377E0CE014C960E94F67F79
:10B5F00060E973E1CE014C960E94727EBC01CE01DF
:10B6000001960E94ED7F48EC50E06FEF7FEFCE0196
:10B6100001960E94F620CE0101960E94577FCE012E
:10B620004C960E94577F0E9433A540E052EC61E0A7
:10B6300070E088EB9EE00E944F7A84EF91E0909357
:10B6400083028093820268E472E10E94EE0967E45B
:10B6500077E0CE014C960E94F67F6AE873E1CE0156
:10B660004C960E94727EBC01CE0101960E94ED7F35
:10B6700060ED77E0CE0101960E94AF8ECE0101967B
:10B680000E94577FCE014C960E94577FDFCA6115FA
:10B690007105D1F510920513109204136DE577E052
:10B6A000CE0101960E94E47FCE0101960E945826A9
:10B6B000CE0101960E94577F6EE377E0CE014C9653
:10B6C0000E94F67F60E973E1CE014C960E94727E83
:10B6D000BC01CE0101960E94ED7F48EC50E06FEF77
:10B6E0007FEFCE0101960E94F620CE0101960E94C6
:10B6F000577FCE014C960E94577F0E9433A540E8A9
:10B7000055E260E070E095CF6230710509F09ECAA5
:10B7100070930513609304136CE477E0CE010196F7
:10B720000E94E47FCE0101960E945826CE01019628
:10B730000E94577F62E477E0C1CF6CE477E0CE01EE
:10B7400001960E94F67FBE016F5F7F4FCE018E96FD
:10B750000E94417E182FCE0101960E94577F11232F
:10B7600009F441C047E050E061EC71E1CE0101967F
:10B770000E94A320BE016F5F7F4F83EA91E10E9488
:10B780001E7FCE0101960E94577F67E177E0CE01D0
:10B7900001960E94F67FBE016F5F7F4F83EA91E1C1
:10B7A0000E94417E182FCE0101960E94577F1111F1
:10B7B00010927F0C60ED74E0CE0101960E94F67F3E
:10B7C000BE016F5F7F4F83EA91E10E94417E182F97
:10B7D000CE0101960E94577F112309F401CD81E02B
:10B7E00080937F0CFDCC64E577E0CE0101960E944A
:10B7F000F67FBE016F5F7F4FCE018E960E94417E25
:10B80000182FCE0101960E94577F112381F146E047
:10B8100050E061EC71E1CE0101960E94A320BE01CF
:10B820006F5F7F4F83EA91E10E941E7FCE010196F8
:10B830000E94577F83EA91E10E949D7D60934C13A3
:10B8400070934D1380934E1390934F1384EF91E0B8
:10B85000909383028093820268E472E10E94EE0971
:10B8600064E670E080E090E00E94B383B9CC6BE5C1
:10B8700077E0CE0101960E94F67FBE016F5F7F4F99
:10B88000CE018E960E94417E182FCE0101960E9415
:10B89000577F112301F148E050E061EC71E1CE01E6
:10B8A00001960E94A320BE016F5F7F4F83EA91E162
:10B8B0000E941E7FCE0101960E94577F83EA91E18C
:10B8C0000E949D7D60935213709353138093541381
:10B8D00090935513BBCF64E677E0CE0101960E94AA
:10B8E000F67FBE016F5F7F4FCE018E960E94417E34
:10B8F000182FCE0101960E94577F112301F149E0D4
:10B9000050E061EC71E1CE0101960E94A320BE01DE
:10B910006F5F7F4F83EA91E10E941E7FCE01019607
:10B920000E94577F83EA91E10E949D7D60935613A8
:10B9300070935713809358139093591387CF6EE6E3
:10B9400077E0CE0101960E94F67FBE016F5F7F4FC8
:10B95000CE018E960E94417E182FCE0101960E9444
:10B96000577F1123F1F049E050E061EC71E1CE0125
:10B9700001960E94A320BE016F5F7F4F83EA91E191
:10B980000E941E7FCE0101960E94577F83EA91E1BB
:10B990000E949D7D0E9474B370935D1360935C134D
:10B9A00055CF68E777E0CE0101960E94F67FBE0191
:10B9B0006F5F7F4FCE018E960E94417E182FCE0181
:10B9C00001960E94577F1123F1F04AE050E061ECAC
:10B9D00071E1CE0101960E94A320BE016F5F7F4FEF
:10B9E00083EA91E10E941E7FCE0101960E94577F5B
:10B9F00083EA91E10E949D7D0E9474B370935B1372
:10BA000060935A1323CF63E877E0CE0101960E943A
:10BA1000F67FBE016F5F7F4FCE018E960E94417E02
:10BA2000182FCE0101960E94577F112311F14BE090
:10BA300050E061EC71E1CE0101960E94A320BE01AD
:10BA40006F5F7F4F83EA91E10E941E7FCE010196D6
:10BA50000E94577F83EA91E10E949D7D0E9474B30A
:10BA600060935E1370935F138093601390936113E0
:10BA7000EDCE6FE877E0CE0101960E94F67FBE0121
:10BA80006F5F7F4FCE018E960E94417E182FCE01B0
:10BA900001960E94577F1123E1F045E050E061ECF0
:10BAA00071E1CE0101960E94A320BE016F5F7F4F1E
:10BAB00083EA91E10E941E7FCE0101960E94577F8A
:10BAC00083EA91E10E94A87D709351136093501313
:10BAD000BDCE65E977E0CE0101960E94F67FBE01FA
:10BAE0006F5F7F4FCE018E960E94417E182FCE0150
:10BAF00001960E94577F112359F00E94DA8A6093C1
:10BB00000E0C70930F0C8093100C9093110C9EC828
:10BB10006BE977E0CE0101960E94F67FBE016F5F70
:10BB20007F4FCE018E960E94417E182FCE01019646
:10BB30000E94577F112389F143E050E0BE01625D0E
:10BB40007F4FCE0101960E94A320BE016F5F7F4F01
:10BB500083EA91E10E941E7FCE0101960E94577FE9
:10BB60008091A7119091A811892B41F083EA91E16E
:10BB70000E94A87D70938902609388028091880258
:10BB8000909189020197029708F42ACB81E090E016
:10BB9000909389028093880223CB6CE777E0CE01F3
:10BBA0004C960E94F67FBE01645E7F4FCE018E965A
:10BBB0000E94417E11E0811115C06EED77E0CE014B
:10BBC00001960E94F67FBE016F5F7F4FCE018E9679
:10BBD0000E94417E11E0811101C010E0CE0101966A
:10BBE0000E94577FCE014C960E94577F112309F483
:10BBF00068C06CE777E0CE0101960E94F67FBE0137
:10BC00006F5F7F4FCE018E960E94417E182FCE012E
:10BC100001960E94577F1123A1F046E050E0BE013B
:10BC2000625D7F4FCE0101960E94A320BE016F5F2F
:10BC30007F4F83EA91E10E941E7FCE0101960E9410
:10BC4000577F6EED77E0CE0101960E94F67FBE0130
:10BC50006F5F7F4FCE018E960E94417E182FCE01DE
:10BC600001960E94577F1123A1F042E050E0BE01EF
:10BC7000625D7F4FCE0101960E94A320BE016F5FDF
:10BC80007F4F83EA91E10E941E7FCE0101960E94C0
:10BC9000577F8091A7119091A811892B09F4A0CA10
:10BCA00063EA71E1CE0101960E94ED7F61E070E0F0
:10BCB000CE0101960E94DE37CE0101960E94577F89
:10BCC0008FCA68EA77E0CE0182960E94F67FBE01B5
:10BCD0006E5D7F4FCE018E960E94417E11E08111F4
:10BCE00029C06FE977E0CE014C960E94F67FBE0135
:10BCF000645E7F4FCE018E960E94417E11E08111DD
:10BD000015C067EA77E0CE0101960E94F67FBE017A
:10BD10006F5F7F4FCE018E960E94417E11E08111B0
:10BD200001C010E0CE0101960E94577FCE014C96D3
:10BD30000E94577FCE0182960E94577F112309F4FB
:10BD4000E6C068EA77E0CE0101960E94F67FBE0168
:10BD50006F5F7F4FCE018E960E94417E182FCE01DD
:10BD600001960E94577F112309F466C046E050E017
:10BD7000BE01625D7F4FCE0101960E94A320BE01ED
:10BD80006F5F7F4F83EA91E10E941E7FCE01019693
:10BD90000E94577F83EA91E10E949D7D6B017C01A7
:10BDA00020E030E0A9010E94AAB318160CF08EC062
:10BDB000A701960160E070E08AE794E40E9402B374
:10BDC0000E9474B360932C0270932D0280932E0214
:10BDD00090932F0280912C0290912D02A0912E021F
:10BDE000B0912F02181619061A061B0664F081E09E
:10BDF00090E0A0E0B0E080932C0290932D02A093FD
:10BE00002E02B0932F028091880290918902813096
:10BE1000910509F068C080912C0290912D02A091AB
:10BE20002E02B0912F028093280290932902A093B2
:10BE30002A02B0932B02D4C947E050E0BE01625DF4
:10BE40007F4FCE0101960E94A320BE016F5F7F4FFE
:10BE500083EA91E10E941E7FCE0101960E94577FE6
:10BE600068E774E0CE0101960E94F67FBE016F5F25
:10BE70007F4FCE018E960E94417E182FCE010196F3
:10BE80000E94577F112331F081E090E09093890266
:10BE90008093880265EB76E0CE0101960E94F67FE2
:10BEA000BE016F5F7F4FCE018E960E94417E182F9C
:10BEB000CE0101960E94577F112309F46BCF82E0D7
:10BEC00090E0909389028093880264CF81E090E0B3
:10BED000A0E0B0E080932C0290932D02A0932E025C
:10BEE000B0932F0277CF029709F07AC980912C0284
:10BEF00090912D02A0912E02B0912F0280932402E6
:10BF000090932502A0932602B093270269C96FEA95
:10BF100077E0CE014C960E94F67FBE01645E7F4FB3
:10BF2000CE018E960E94217E11E0811115C064EB36
:10BF300077E0CE0101960E94F67FBE016F5F7F4FD2
:10BF4000CE018E960E94417E11E0811101C010E069
:10BF5000CE0101960E94577FCE014C960E94577FDA
:10BF6000112309F48CC269E378E0CE0101960E94A6
:10BF7000F67FBE016F5F7F4FCE018E960E94417E9D
:10BF8000182FCE0101960E94577F112309F4FBC0A0
:10BF900001E010E010938902009388021093500290
:10BFA00000934F0269EC75E083EA91E10E943A7DCB
:10BFB0001093500200934F0281E090E0A0E0B0E0C7
:10BFC00080932C0290932D02A0932E02B0932F0207
:10BFD0008093280290932902A0932A02B0932B0207
:10BFE00063EA71E1CE0101960E94ED7F62E070E0AC
:10BFF000CE0101960E94DE37CE0101960E94577F46
:10C0000063E878E0CE0101960E94E47FCE010196BC
:10C010000E94E61FCE0101960E94577F63E778E0F9
:10C02000CE0101960E94E47FCE0101960E948F28E6
:10C03000CE0101960E94577F67E177E083EA91E1A4
:10C040000E943A7D63EA71E1CE0101960E94ED7F84
:10C0500063E070E0CE0101960E94DE37CE010196CA
:10C060000E94577F82E090E090938902809388023B
:10C0700062E678E0CE0101960E94E47FCE0101964F
:10C080000E94E61FCE0101960E94577F66E578E088
:10C09000CE0101960E94E47FCE0101960E948F2876
:10C0A000CE0101960E94577F69EC75E083EA91E129
:10C0B0000E943A7D80916E1390916F1397FF06C096
:10C0C0006DEC75E083EA91E10E943A7D63EA71E1EB
:10C0D000CE0101960E94ED7F62E070E0CE010196F4
:10C0E0000E94DE37CE0101960E94577F67E177E01C
:10C0F00083EA91E10E943A7D82E090E09093890288
:10C100008093880263EA71E1CE0101960E94ED7F7F
:10C1100063E070E0CE0101960E94DE37CE01019609
:10C120000E94577F84EF91E0909383028093820274
:10C1300068E472E10E94EE0964E670E080E090E05D
:10C140000E94B38381E090E09093890280938802FB
:10C150001092D8021092D70282E090E0A0E0B0E006
:10C160008093C1029093C202A093C302B093C40211
:10C170000E94DA8A6093E1027093E2028093E30204
:10C180009093E4022DC86FEA77E0CE0101960E94F9
:10C19000F67FBE016F5F7F4FCE018E960E94417E7B
:10C1A000182FCE0101960E94577F111119C868E718
:10C1B00074E0CE0101960E94F67FBE016F5F7F4F53
:10C1C000CE018E960E94417E182FCE0101960E94CC
:10C1D000577F112331F081E090E0909389028093A2
:10C1E000880265EB76E0CE0101960E94F67FBE01E3
:10C1F0006F5F7F4FCE018E960E94417E182FCE0139
:10C2000001960E94577F112331F082E090E09093D5
:10C2100089028093880281E090E0A0E0B0E0809302
:10C220002C0290932D02A0932E02B0932F028091A6
:10C230008802909189028130910509F099C090930C
:10C24000500280934F0264EB77E0CE0101960E948A
:10C25000F67FBE016F5F7F4FCE018E960E94417EBA
:10C26000182FCE0101960E94577F112319F146E045
:10C2700050E0BE01625D7F4FCE014C960E94A3202C
:10C280006BEB77E0CE0101960E94F67FBE01645E03
:10C290007F4FCE0101960E94727EBC0183EA91E13C
:10C2A0000E94077FCE0101960E94577FCE014C96D7
:10C2B0000E94577F80912C0290912D02A0912E0216
:10C2C000B0912F028093280290932902A0932A0212
:10C2D000B0932B0269EC75E083EA91E10E943A7D0C
:10C2E00063EA71E1CE0101960E94ED7F62E070E0A9
:10C2F000CE0101960E94DE37CE0101960E94577F43
:10C3000065E478E0CE0101960E94E47FCE010196BB
:10C310000E94E61FCE0101960E94577F81E090E0C7
:10C320009093500280934F0267E177E083EA91E1B6
:10C330000E943A7D63EA71E1CE0101960E94ED7F91
:10C3400063E070E0CE0101960E94DE37CE010196D7
:10C350000E94577F65E378E0CE0101960E94E47F5A
:10C36000CE0101960E948F28CE0101960E94577F30
:10C370008091880290918902029711F00C94F058F4
:10C3800069EC75E083EA91E10E943A7D80916E1339
:10C3900090916F1397FF06C06DEC75E083EA91E111
:10C3A0000E943A7D01E010E01093500200934F028A
:10C3B00063EA71E1CE0101960E94ED7F62E070E0D8
:10C3C000CE0101960E94DE37CE0101960E94577F72
:10C3D00067E177E083EA91E10E943A7D64E278E0E8
:10C3E000CE0101960E94E47FCE0101960E94E61FD5
:10C3F000CE0101960E94577F63EA71E1CE0101965A
:10C400000E94ED7F63E070E0CE0101960E94DE376E
:10C41000CE0101960E94577F68E178E0CE01019637
:10C420000E94E47FCE0101960E948F28CE010196E2
:10C430000E94577F80916E1390916F139195819513
:10C44000910990936F1380936E1310935002009391
:10C450004F0284EF91E0909383028093820268E41C
:10C4600072E10E94EE0964E670E080E090E00E94D4
:10C47000B38310938902009388020C94F0586DEBFB
:10C4800077E0CE0188960E94F67FBE01685D7F4FFF
:10C49000CE018E960E94417E01E081113DC06EE08A
:10C4A00078E0CE0182960E94F67FBE016E5D7F4FDE
:10C4B000CE018E960E94417E01E0811129C06DE07F
:10C4C00078E0CE014C960E94F67FBE01645E7F4FFD
:10C4D000CE018E960E94417E01E0811115C064EC70
:10C4E00077E0CE0101960E94F67FBE016F5F7F4F1D
:10C4F000CE018E960E94417E01E0811101C000E0D4
:10C50000CE0101960E94577FCE014C960E94577F24
:10C51000CE0182960E94577FCE0188960E94577F57
:10C52000002309F41FC26DEB77E0CE0101960E9453
:10C53000F67FBE016F5F7F4FCE018E960E94417ED7
:10C54000082FCE0101960E94577F46E050E001116E
:10C5500017C06EE078E0CE0101960E94F67FBE0122
:10C560006F5F7F4FCE018E960E94417E082FCE01D5
:10C5700001960E94577F002309F48BC042E050E0EF
:10C58000BE01625D7F4FCE0101960E94A320BE01D5
:10C590006F5F7F4F83EA91E10E941E7FCE0101967B
:10C5A0000E94577F8091A7119091A811892B11F4B7
:10C5B0000C94F0586BEB77E0CE014C960E94F67F1E
:10C5C000BE01645E7F4F83EA91E10E94417E81114A
:10C5D00014C06DEB75E0CE0101960E94F67FBE019E
:10C5E0006F5F7F4F83EA91E10E94417E11E08111EC
:10C5F00010E0CE0101960E94577FCE014C960E941A
:10C60000577FC12CD12C7601112309F46AC183EA2A
:10C6100091E10E949D7D6B017C0180918802909147
:10C620008902019709F09FC083EA91E10E949D7DF4
:10C630009B01AC016091C60B7091C70B8091C80B38
:10C640009091C90B0E9496B26093C60B7093C70B72
:10C650008093C80B9093C90B8090C60B9090C70B2A
:10C66000A090C80BB090C90B20E030E044EB53E43D
:10C67000C501B4010E94AAB387FD86C020E030E066
:10C6800044EB53E4C501B4010E9495B24B015C0137
:10C69000EBCF43E050E0BE01625D7F4FCE010196DB
:10C6A0000E94A320BE016F5F7F4F83EA91E10E9449
:10C6B0001E7FCE0101960E94577F68E774E0CE018D
:10C6C00001960E94F67FBE016F5F7F4FCE018E966E
:10C6D0000E94417E082FCE0101960E94577F0023C1
:10C6E000B1F081E090E0909389028093880280917C
:10C6F000190C90911A0CA0911B0CB0911C0C8093FA
:10C70000C60B9093C70BA093C80BB093C90B65EBF6
:10C7100076E0CE0101960E94F67FBE016F5F7F4FEB
:10C72000CE018E960E94417E082FCE0101960E9476
:10C73000577F002309F436CF82E090E0909389027E
:10C74000809388028091150C9091160CA091170C83
:10C75000B091180C8093C60B9093C70BA093C80B95
:10C76000B093C90B1FCF83EA91E10E949D7D9B018D
:10C77000AC016091C60B7091C70B8091C80B909172
:10C78000C90B0E9495B260CF20E030E0A901C5013D
:10C79000B4010E94E8B087FF0BC020E030E044EB1A
:10C7A00053E4C501B4010E9496B24B015C01ECCF89
:10C7B0008092C60B9092C70BA092C80BB092C90B87
:10C7C00020E030E0A901C701B6010E94AAB387FDAD
:10C7D00015C06DEB75E0CE0101960E94F67F63EA0D
:10C7E00071E1CE0101960E94727EBC0183EA91E163
:10C7F0000E94077FCE0101960E94577F20E030E023
:10C80000A901C701B6010E94E8B087FF6AC0809104
:10C81000880290918902019799F520E030E0A90102
:10C82000C701B6010E94AAB318160CF092C020E00E
:10C8300030E040E251E4C701B6010E9496B222E026
:10C84000AB01BC01CE014C960E945F7F6BEB77E0A1
:10C85000CE0101960E94F67FBE01645E7F4FCE013D
:10C8600001960E94727EBC0183EA91E10E94077FDB
:10C87000CE0101960E94577FCE014C960E94577FB1
:10C880008091880290918902019759F120E030E06F
:10C89000A901C701B6010E94AAB3B701A6011816E3
:10C8A0000CF0705822E0CE014C960E945F7F6BEB3B
:10C8B00077E0CE0101960E94F67FBE01645E7F4F55
:10C8C000CE0101960E94727EBC0183EA91E10E9432
:10C8D000077FCE0101960E94577FCE014C960E94A1
:10C8E000577F81E090E09093500280934F0263EA7B
:10C8F00071E1CE0101960E94ED7F62E070E0CE0111
:10C9000001960E94DE37CE0101960E94577F20E0FB
:10C9100030E0A901C701B6010E94E8B087FD02C05E
:10C920000C94F0588091880290918902019711F03F
:10C930000C94F05868EC77E083EA91E10E943A7D2C
:10C9400063EA71E1CE0101960E94ED7F62E070E042
:10C95000AFC9A701960160E070E080E291E40E9417
:10C9600095B26DCF6DEC77E0CE0182960E94F67F96
:10C97000BE016E5D7F4FCE018E960E94417E11E01A
:10C98000811129C06CEC77E0CE014C960E94F67FB5
:10C99000BE01645E7F4FCE018E960E94417E11E003
:10C9A000811115C063ED77E0CE0101960E94F67FFC
:10C9B000BE016F5F7F4FCE018E960E94417E11E0D7
:10C9C000811101C010E0CE0101960E94577FCE0177
:10C9D0004C960E94577FCE0182960E94577F11236A
:10C9E00009F49BC0CE018E960E94B37D69EC75E080
:10C9F00083EA91E10E943A7D68E774E0CE010196F6
:10CA00000E94F67FBE016F5F7F4FCE018E960E941F
:10CA1000417E182FCE0101960E94577F112331F0DD
:10CA200081E090E0909389028093880265EB76E044
:10CA3000CE0101960E94F67FBE016F5F7F4FCE014F
:10CA40008E960E94417E182FCE0101960E94577F3C
:10CA5000112391F082E090E0909389028093880204
:10CA600080916E1390916F1397FF06C06DEC75E087
:10CA700083EA91E10E943A7D81E090E09093500238
:10CA800080934F0263EA71E1CE0101960E94ED7F2F
:10CA900062E070E0CE0101960E94DE37CE01019681
:10CAA0000E94577F6DEC77E0CE0101960E94F67FE1
:10CAB000BE016F5F7F4FCE018E960E94417E182F80
:10CAC000CE0101960E94577F45E050E0111102C04F
:10CAD00046E050E0BE01625D7F4FCE0101960E94AC
:10CAE000A320BE016F5F7F4F83EA91E10E941E7F0A
:10CAF000CE0101960E94577F8091A7119091A811B5
:10CB0000892B11F40C94F05863EA71E1CE0101967F
:10CB10000E94ED7F63E070E0CBC86BED77E0CE0163
:10CB200082960E94F67FBE016E5D7F4FCE018E968B
:10CB30000E94417E11E0811129C06AED77E0CE01AB
:10CB40004C960E94F67FBE01645E7F4FCE018E96AA
:10CB50000E94417E11E0811115C061EE77E0CE01A7
:10CB600001960E94F67FBE016F5F7F4FCE018E96C9
:10CB70000E94417E11E0811101C010E0CE010196BA
:10CB80000E94577FCE014C960E94577FCE0182961D
:10CB90000E94577F112309F426C16BED77E0CE0187
:10CBA00001960E94F67FBE016F5F7F4FCE018E9689
:10CBB0000E94417E182FCE0101960E94577F1123BB
:10CBC00009F443C045E050E0BE01625D7F4FCE01F5
:10CBD00001960E94A320BE016F5F7F4F83EA91E11F
:10CBE0000E941E7FCE0101960E94577F8091A7115F
:10CBF0009091A811892B61F083EA91E10E949D7DBB
:10CC00006093C60B7093C70B8093C80B9093C90BAE
:10CC1000C090C60BD090C70BE090C80BF090C90B2A
:10CC200020E030E044EB53E4C701B6010E94AAB310
:10CC300087FD55C020E030E044EB53E4C701B60166
:10CC40000E9495B26B017C01EBCF46E050E0BE0143
:10CC5000625D7F4FCE0101960E94A320BE016F5FEF
:10CC60007F4F83EA91E10E941E7FCE0101960E94D0
:10CC7000577F68E774E0CE0101960E94F67FBE01FF
:10CC80006F5F7F4FCE018E960E94417E182FCE019E
:10CC900001960E94577F112331F081E090E090933C
:10CCA00089028093880265EB76E0CE0101960E94AE
:10CCB000F67FBE016F5F7F4FCE018E960E94417E50
:10CCC000182FCE0101960E94577F112309F48ECFB1
:10CCD00082E090E0909389028093880287CF20E0E1
:10CCE00030E0A901C701B6010E94E8B087FF0BC080
:10CCF00020E030E044EB53E4C701B6010E9496B255
:10CD00006B017C01ECCFC092C60BD092C70BE092B6
:10CD1000C80BF092C90B809188029091890201970B
:10CD200071F4C092190CD0921A0CE0921B0CF09284
:10CD30001C0C60E175E089EA91E10E943A7D8091E6
:10CD4000C60B9091C70BA091C80BB091C90B209155
:10CD50008802309189022230310571F48093150CDC
:10CD60009093160CA093170CB093180C60E275E02A
:10CD700089EA91E10E943A7D4091C60B5091C70B20
:10CD80006091C80B7091C90B21E0CE014C960E94B6
:10CD90005F7F69EA71E1CE0101960E94ED7FBE01DD
:10CDA000645E7F4FCE0101960E94727E6BE175E05A
:10CDB0000E945C7EBC0189EA91E10E94077FCE015E
:10CDC00001960E94577FCE014C960E94577F69EAD8
:10CDD00071E1CE0101960E94ED7FCE0101960E9485
:10CDE0008F280C945C5E69EE77E0CE0182960E94FB
:10CDF000F67FBE016E5D7F4FCE018E960E94417E12
:10CE000011E0811129C068EE77E0CE014C960E94B6
:10CE1000F67FBE01645E7F4FCE018E960E94417EFA
:10CE200011E0811115C06EEE77E0CE0101960E94EF
:10CE3000F67FBE016F5F7F4FCE018E960E94417ECE
:10CE400011E0811101C010E0CE0101960E94577FD0
:10CE5000CE014C960E94577FCE0182960E94577F4A
:10CE6000112309F412C2C0902C02D0902D02E09040
:10CE70002E02F0902F0264EF77E0CE0101960E941F
:10CE8000F67FBE016F5F7F4FCE018E960E94417E7E
:10CE9000182FCE0101960E94577F112309F465C017
:10CEA00044E050E0BE01625D7F4FCE0101960E94DA
:10CEB000A320BE016F5F7F4F83EA91E10E941E7F36
:10CEC000CE0101960E94577F80918802909189023D
:10CED0008130910509F093C0C0902802D0902902BA
:10CEE000E0902A02F0902B0281E090E0A0E0B0E018
:10CEF0008093280290932902A0932A02B0932B02D8
:10CF00008091A7119091A811892B09F090C069EF29
:10CF100077E083EA91E10E943A7D8091A711909198
:10CF2000A811892B81F063EA71E1CE0101960E947C
:10CF3000ED7F70E060E0CE0101960E94DE37CE0109
:10CF400001960E94577F80918802909189028130DA
:10CF5000910509F08CC1C0922802D0922902E0927A
:10CF60002A02F0922B020C94F05845E050E0BE01EA
:10CF7000625D7F4FCE0101960E94A320BE016F5FCC
:10CF80007F4F83EA91E10E941E7FCE0101960E94AD
:10CF9000577F68E774E0CE0101960E94F67FBE01DC
:10CFA0006F5F7F4FCE018E960E94417E182FCE017B
:10CFB00001960E94577F112331F081E090E0909319
:10CFC00089028093880265EB76E0CE0101960E948B
:10CFD000F67FBE016F5F7F4FCE018E960E94417E2D
:10CFE000182FCE0101960E94577F112309F46CCFB0
:10CFF00082E090E0909389028093880265CF029747
:10D0000009F07ECFC0902402D0902502E090260245
:10D01000F090270281E090E0A0E0B0E0809324024D
:10D0200090932502A0932602B093270269CF6FEF59
:10D0300077E0CE0101960E94F67FBE016F5F7F4FC1
:10D0400083EA91E10E94217E182FCE0101960E9471
:10D05000577F112309F477CF83EA91E10E949D7DE8
:10D0600020E030E0A9010E94E8B0811128C0809141
:10D07000880290918902019731F462E078E083EAB6
:10D0800091E10E943A7D80918802909189020297F5
:10D0900031F469EF77E083EA91E10E943A7D809173
:10D0A000A7119091A811892B09F44DCF63EA71E182
:10D0B000CE0101960E94ED7F61E070E03CCF64E616
:10D0C00076E0CE0101960E94F67FBE016F5F7F4F32
:10D0D00083EA91E10E94217E182FCE0101960E94E1
:10D0E000577F112309F42FCF41E050E063EA71E14B
:10D0F000CE0101960E94A320CE0101960E949D7D43
:10D100004B015C01CE0101960E94577F20E030E088
:10D11000A901C501B4010E94E8B0181634F0812CB1
:10D12000912C90E8A92E9FE3B92E009188021091CE
:10D1300089020130110509F075C0A501940160E074
:10D1400070E48CE995E40E9402B36093200270932E
:10D1500021028093220290932302609366137093BE
:10D160006713809368139093691360931C02709304
:10D170001D0280931E0290931F02B801CE014C96AF
:10D180000E94447D67E078E0CE0101960E94F67F20
:10D19000BE01645E7F4FCE0101960E94727EBC018B
:10D1A000CE0182960E94ED7FCE0182960E94FD1FE5
:10D1B000CE0182960E94577FCE0101960E94577F32
:10D1C000CE014C960E94577F66E078E0CE01019632
:10D1D0000E94E47FCE0101960E94FD1FCE010196C0
:10D1E0000E94577F409120025091210260912202BB
:10D1F0007091230225E0CE0101960E945F7FCE014F
:10D2000001960E94E61FCE0101960E94577F84EF8F
:10D2100091E0909383028093820268E472E10E941D
:10D22000EE0991CE0230110509F0A7CFA5019401B6
:10D2300060E070E48CE196E40E9402B36093200207
:10D2400070932102809322029093230260936A13C9
:10D2500070936B1380936C1390936D13609318020B
:10D260007093190280931A0290931B0286CF029743
:10D2700011F00C94F058C0922402D0922502E09252
:10D280002602F09227020C94F0586CE078E0CE0170
:10D2900082960E94F67FBE016E5D7F4FCE018E9614
:10D2A0000E94417E11E0811129C06BE078E0CE013F
:10D2B0004C960E94F67FBE01645E7F4FCE018E9633
:10D2C0000E94417E11E0811115C061E178E0CE013C
:10D2D00001960E94F67FBE016F5F7F4FCE018E9652
:10D2E0000E94417E11E0811101C010E0CE01019643
:10D2F0000E94577FCE014C960E94577FCE018296A6
:10D300000E94577F112309F429C18AA99BA9059777
:10D3100010F40C94F05844E050E0BE01625D7F4F81
:10D32000CE0101960E94A320BE016F5F7F4F83EA6A
:10D3300091E10E941E7FCE0101960E94577F6CE012
:10D3400078E0CE0101960E94F67FBE016F5F7F4FAD
:10D35000CE018E960E94417E182FCE0101960E942A
:10D36000577F112309F49BC044E050E0BE01625D89
:10D370007F4FCE0101960E94A320BE016F5F7F4FB9
:10D3800083EA91E10E941E7FCE0101960E94577FA1
:10D3900083EA91E10E949D7D20E030E0A9010E9496
:10D3A000AAB3181614F00C94F05883EA91E10E9485
:10D3B0009D7D6093200270932102809322029093BE
:10D3C000230220918802309189022130310509F031
:10D3D000B0C0609366137093671380936813909343
:10D3E000691360931C0270931D0280931E02909338
:10D3F0001F02B901CE014C960E94447D67E078E09F
:10D40000CE0101960E94F67FBE01645E7F4FCE0181
:10D4100001960E94727EBC01CE0182960E94ED7F31
:10D42000CE0182960E94FD1FCE0182960E94577FF8
:10D43000CE0101960E94577FCE014C960E94577FE5
:10D4400064EF77E0CE0101960E94E47FCE01019661
:10D450000E94FD1FCE0101960E94577F409120023D
:10D4600050912102609122027091230225E0CE01A9
:10D4700001960E945F7FCE0101960E94E61FCE01B9
:10D4800001960E94577F84EF91E0909383028093EE
:10D49000820268E472E10E94EE090C94F05845E0C3
:10D4A00050E0BE01625D7F4FCE0101960E94A32035
:10D4B000BE016F5F7F4F83EA91E10E941E7FCE0124
:10D4C00001960E94577F68E774E0CE0101960E94A2
:10D4D000F67FBE016F5F7F4FCE018E960E94417E28
:10D4E000182FCE0101960E94577F112331F081E061
:10D4F00090E0909389028093880265EB76E0CE01FC
:10D5000001960E94F67FBE016F5F7F4FCE018E961F
:10D510000E94417E182FCE0101960E94577F112351
:10D5200009F436CF82E090E09093890280938802DC
:10D530002FCF2230310509F05CCF60936A137093CE
:10D540006B1380936C1390936D1360931802709318
:10D55000190280931A0290931B024BCF68EF75E07B
:10D56000CE014C960E94F67FBE01645E7F4FCE01D5
:10D570008E960E94417E11E0811115C067E178E02E
:10D58000CE0101960E94F67FBE016F5F7F4FCE01F4
:10D590008E960E94417E11E0811101C010E0CE0103
:10D5A00001960E94577FCE014C960E94577F11230F
:10D5B00009F463C068EF75E0CE0101960E94F67F22
:10D5C000BE016F5F7F4FCE018E960E94417E182F65
:10D5D000CE0101960E94577F112399F042E050E05E
:10D5E00061EC71E1CE0101960E94A320BE016F5F44
:10D5F0007F4F83EA91E10E941E7FCE0101960E9437
:10D60000577F67E178E0CE0101960E94F67FBE0168
:10D610006F5F7F4FCE018E960E94417E182FCE0104
:10D6200001960E94577F112399F043E050E061EC8E
:10D6300071E1CE0101960E94A320BE016F5F7F4F72
:10D6400083EA91E10E941E7FCE0101960E94577FDE
:10D6500083EA91E10E94A87D653B710510F40C946A
:10D66000F05861EE77E0CE0101960E94E47FCE0192
:10D6700001960E94FD1F0C945C5E6BE178E0CE0188
:10D6800001960E94F67FBE016F5F7F4FCE018E969E
:10D690000E94417E182FCE0101960E94577F1123D0
:10D6A00009F47EC026E030E044E050E061EC71E136
:10D6B000CE0101960E940B80BE016F5F7F4F83EA0F
:10D6C00091E10E941E7FCE0101960E94577F64E681
:10D6D00076E0CE0101960E94F67F4091C5115091EF
:10D6E000C6118D819E81481B590BBE016F5F7F4F14
:10D6F00081EC91E10E947AA5AC014F5F5F4F61EC34
:10D7000071E1CE014C960E94A320BE01645E7F4F62
:10D7100083EA91E10E941E7FCE014C960E94577FC2
:10D72000CE0101960E94577F83EA91E10E949D7D80
:10D7300088E2EEE9FBE0AFE1B3E101900D928A955A
:10D74000E1F784EF91E0909383028093820268E492
:10D7500072E10E94EE0960EC77E089EA91E10E94B3
:10D76000E27E44E050E061EC71E1CE0101960E945E
:10D77000A320BE016F5F7F4F89EA91E10E94DB7EAB
:10D78000CE0101960E94577F69EA71E1CE010196B0
:10D790000E94ED7FCE0101960E94E61F0C94665A0E
:10D7A0006FE178E0CE0101960E94F67FBE016F5FC7
:10D7B0007F4FCE018E960E94417E182FCE0101969A
:10D7C0000E94577F11110C94B25B67E278E0CE01A2
:10D7D00001960E94F67FBE016F5F7F4FCE018E964D
:10D7E0000E94417E182FCE0101960E94577F11237F
:10D7F00071F141E066E972E0CE0101960E94A397C3
:10D80000BE016F5F7F4F88EA93E10E94142088EA8F
:10D8100093E10E948B12811104C064E777E00C94BD
:10D820006B5488EA93E10E948307892B51F088EAC0
:10D8300093E10E944D09682F85E59FE00E94ED77F6
:10D84000F0CF88EA93E10E9497120C94594C6EE253
:10D8500078E0CE0101960E94F67FBE016F5F7F4F98
:10D86000CE018E960E94417E182FCE0101960E9415
:10D87000577F1123E9F08DB79EB78E5291400FB6B6
:10D88000F8949EBF0FBE8DBFADB7BEB711968EE2A6
:10D8900091E0E8E4F2E101900D920197E1F70E9436
:10D8A00047340FB6F894DEBF0FBECDBF0C94594C71
:10D8B00067E378E0CE0101960E94F67FBE016F5FBC
:10D8C0007F4FCE018E960E94417E182FCE01019689
:10D8D0000E94577F112309F457C0EDB7FEB7EE52EF
:10D8E000F1400FB6F894FEBF0FBEEDBFADB7BEB7A7
:10D8F00011968EE291E0E8E4F2E101900D92019739
:10D90000E1F70E94DE2D0FB6F894DEBF0FBECDBF4B
:10D910006FEA77E0CE0101960E94E47FADB7BEB713
:10D92000AE52B1400FB6F894BEBF0FBEADBF119658
:10D930008EE291E0E8E4F2E101900D920197E1F7C7
:10D940000E9436240FB6F894DEBF0FBECDBF8DB750
:10D950009EB78E5291400FB6F8949EBF0FBE8DBFFA
:10D96000ADB7BEB711968EE291E0E8E4F2E1019026
:10D970000D920197E1F70E9447340FB6F894DEBF8D
:10D980000FBECDBF0C944F5169E378E0CE010196F4
:10D990000E94F67FBE016F5F7F4FCE018E960E9480
:10D9A000417E182FCE0101960E94577F1123F9F076
:10D9B0006DE977E0CE0101960E94E47FBE016F5FC2
:10D9C0007F4FCE014C960E94ED7FCE014C960E9477
:10D9D000E61FCE014C960E94577FEDB7FEB7EE5280
:10D9E000F1400FB6F894FEBF0FBEEDBFB9CF6DE3A7
:10D9F00078E0CE0101960E94F67FBE016F5F7F4FF7
:10DA0000CE018E960E94417E182FCE0101960E9473
:10DA1000577F112309F4F5C061E877E0CE018296C3
:10DA20000E94E47FBE016E5D7F4FCE0101960E9491
:10DA3000ED7FAE014F5F5F4F62E070E08EE592E0F8
:10DA40000E94812F182FCE0101960E94577F11113D
:10DA500022C0BE016E5D7F4FCE014C960E94ED7FCD
:10DA600061E478E0CE014C960E945C7E64EF71E147
:10DA70000E94727EBC01CE0101960E94ED7FCE0114
:10DA800001960E94E61FCE0101960E94577FCE01AB
:10DA90004C960E94577F68EE73E080E090E00E9411
:10DAA000B383BE016E5D7F4FCE0101960E94ED7F74
:10DAB000AE014F5F5F4F63E070E081E592E00E944E
:10DAC000812F182FCE0101960E94577F111122C07D
:10DAD000BE016E5D7F4FCE014C960E94ED7F6FEAD6
:10DAE00075E0CE014C960E945C7E64EF71E10E946D
:10DAF000727EBC01CE0101960E94ED7FCE0101969F
:10DB00000E94E61FCE0101960E94577FCE014C96DF
:10DB10000E94577F68EE73E080E090E00E94B3833C
:10DB200068EE71E1CE0101960E94ED7FAE014F5F7C
:10DB30005F4F61E070E080EB92E00E94812F182F30
:10DB4000CE0101960E94577F111121C068EE71E14C
:10DB5000CE014C960E94ED7F6FEA75E0CE014C96A7
:10DB60000E945C7E64EF71E10E94727EBC01CE0176
:10DB700001960E94ED7FCE0101960E94E61FCE0124
:10DB800001960E94577FCE014C960E94577F68EE07
:10DB900073E080E090E00E94B38380917F0C882343
:10DBA00011F40C94E35743E160EB72E0CE0101966F
:10DBB0000E94A397BE016F5F7F4F8EED93E10E949D
:10DBC00014208EED93E10E948B12882311F40C94A3
:10DBD000E35768EE71E18EED93E10E943C8166E9C6
:10DBE00070E080E090E00E94B3838EED93E10E94AC
:10DBF000971262E370E080E090E00E94B3830C949F
:10DC0000E35761E578E0CE0101960E94F67FBE0100
:10DC10006F5F7F4FCE018E960E94417E182FCE01FE
:10DC200001960E94577F1123C1F00CED1BE082EE9C
:10DC3000E82E8BE0F82ED8018C910E5F1F4F60E02C
:10DC40000E9440826CE271E080E090E00E94B38329
:10DC5000E016F10681F70C94594C65E578E0CE01A9
:10DC600001960E94F67FBE016F5F7F4FCE018E96B8
:10DC70000E94417E182FCE0101960E94577F1123EA
:10DC8000A9F00CED1BE0F80180810E5F1F4F61E0F1
:10DC90000E9440826CE271E080E090E00E94B383D9
:10DCA000FBE0023E1F0779F70C94594C6AE578E0D7
:10DCB000CE0101960E94F67FBE016F5F7F4FCE01BD
:10DCC0008E960E94417E182FCE0101960E94577FAA
:10DCD000112311F40C94594C27E030E046E050E059
:10DCE00061EC71E1CE0101960E940B80BE016F5F75
:10DCF0007F4F83EA91E10E941E7FCE0101960E9430
:10DD0000577F83EA91E10E94A87D672B71F41092FE
:10DD10009D0B61EC71E1CE0101960E94ED7FCE0179
:10DD200001960E9458260C94665A81E080939D0BC0
:10DD3000F0CF4F925F926F927F928F929F92AF92AD
:10DD4000BF92CF92DF92EF92FF920F931F93CF93E8
:10DD5000DF93CDB7DEB72C970FB6F894DEBF0FBEBA
:10DD6000CDBF68E370E080916B0290916C020E94DD
:10DD7000C40A84E1482E512C612C712CD12CC12C69
:10DD8000AFEFCA1ADA0AC301B2010E94B383E0906E
:10DD90006B02F0906C0268E370E0C7010E94C40A55
:10DDA0008C01B3E0CB16D10434F08EE1C816D10457
:10DDB00044F4012B51F094E1490E511C611C711C7B
:10DDC000DFCF0115110509F0AEC08BE0E816F104B4
:10DDD00009F08EC080907A1390907B13A0907C13F2
:10DDE000B0907D138091761390917713A091781362
:10DDF000B091791389879A87AB87BC8764E670E016
:10DE000080E090E00E94B38369E275E0CE01019664
:10DE10000E94E47FCE0101960E948F28CE010196D8
:10DE20000E94577F61E082E00E94828E21E0B5016E
:10DE3000A401CE0101960E945F7FBE016F5F7F4FFC
:10DE40008AEF93E10E942E81CE0101960E94577FB6
:10DE50006FED8AEF93E10E94E08E64E275E08AEF55
:10DE600093E10E94508120E049855A856B857C852D
:10DE7000CE0101960E945F7FBE016F5F7F4F8AEFE8
:10DE800093E10E942E81CE0101960E94577F61E6A8
:10DE900078E08AEF93E10E94268189829A82AB82A0
:10DEA000BC8289859A85AB85BC858D839E83AF8333
:10DEB000B88729813A814B815C816D817E818F8118
:10DEC00098852C960FB6F894DEBF0FBECDBFDF91BC
:10DED000CF911F910F91FF90EF90DF90CF90BF9067
:10DEE000AF909F908F907F906F905F904F9008952C
:10DEF00096E1E916F10409F46DCFACE0EA16F104FD
:10DF000009F07CCF8090C60A9090C70AA090C80AFA
:10DF1000B090C90A8091C20A9091C30AA091C40A24
:10DF2000B091C50A67CF0F3F9FEF1907CCF066E1AC
:10DF300075E0CE0101960E94E47F4AE050E070E077
:10DF400060E0CE0101960E94F620CE0101960E946B
:10DF5000577F63EF74E089EA91E10E94E27E32C06C
:10DF60000E3FAFEF1A07B9F165EE74E0CE010196EE
:10DF70000E94E47F4AE050E070E060E0CE0101964C
:10DF80000E94F620CE0101960E94577F66ED74E054
:10DF900089EA91E10E94E27EB801CE0101960E94D9
:10DFA000447DBE016F5F7F4F89EA91E10E94DB7E75
:10DFB000CE0101960E94577F60EC74E089EA91E1FE
:10DFC0000E94857E19821A821B821C821D821E82FB
:10DFD0001F8218866ECF65EB74E0CE0101960E9419
:10DFE000E47F4AE050E070E060E0CE0101960E94DC
:10DFF000F620CE0101960E94577F65E974E0ABCF11
:10E000002F923F924F925F926F927F928F929F9248
:10E01000AF92BF92CF92DF92EF92FF920F931F9336
:10E02000CF93DF93CDB7DEB7AC970FB6F894DEBFD2
:10E030000FBECDBF8C017B018091130C9091140C0D
:10E0400001969093140C8093130C2091120C2223B0
:10E0500041F06AE070E00E94C0B3181619060CF493
:10E06000B4C281E08093120C1092140C1092130C25
:10E0700050E040E068E174E0C8010E945E2082E068
:10E08000E816F10409F4BAC267E174E082EE91E1A6
:10E090000E943A7D68E370E080916B0290916C027F
:10E0A0000E94C40A1C0168E07BE0C8010E94452070
:10E0B00063E678E0C8010E94268164E873E1CE013E
:10E0C00001960E94ED7FBE016F5F7F4FC8010E94E5
:10E0D0002E81CE0101960E94577F6CE678E0C80140
:10E0E0000E94268164EF75E0C8010E9450816AE8B1
:10E0F00073E1CE0101960E94ED7FBE016F5F7F4FFD
:10E10000C8010E942E816AEE75E0C8010E9450810C
:10E1100060EA72E1CE0109960E94F67FBE01675F58
:10E120007F4FC8010E942E816DED75E0C8010E94ED
:10E13000508168E073E1CE010F960E94F67FBE0128
:10E14000615F7F4FC8010E942E8166ED75E0C801B6
:10E150000E945081CE010F960E94577FCE010996F2
:10E160000E94577FCE0101960E94577F0E948286AF
:10E1700028EE33E040E050E00E9432B229013A013B
:10E180006CEC75E0C8010E945081CE0101960E949E
:10E19000C228BE016F5F7F4FC8010E942E81CE0151
:10E1A00001960E94577FC301B20120E13EE040E0AA
:10E1B00050E00E9454B24B015C01B901CE01879638
:10E1C0000E948C214CE3C42ED12CE12CF12CC501F2
:10E1D000B401A70196010E9454B2B901CE01019683
:10E1E0000E948C2165E477E0CE0109960E94F67FBB
:10E1F000BE016F5F7F4FCE0109960E94727EBC0107
:10E20000CE0187960E94DB7ECE0109960E94577F41
:10E21000CE0101960E94577FC301B201A70196016A
:10E220000E9454B2CE0101960E948C2165E477E0F1
:10E23000CE0109960E94F67FBE016F5F7F4FCE012F
:10E2400009960E94727EBC01CE0187960E94DB7EF9
:10E25000CE0109960E94577FCE0101960E94577FFA
:10E2600062E778E0CE0109960E94F67FBE01695D03
:10E270007F4FCE0109960E94727E65E778E00E948A
:10E280005C7EBC01CE0101960E94ED7FBE016F5FF6
:10E290007F4FC8010E942E81CE0101960E94577FB8
:10E2A000CE0109960E94577F63E878E0C8010E947A
:10E2B0002681CE0101960E94DE1EB801CE01019694
:10E2C0000E94B2806EE778E0C8010E9412810E942D
:10E2D000996E29833A834B835C836D837E838F831E
:10E2E000988749815A816B817C8121E0CE010F960C
:10E2F0000E945F7FBE01615F7F4FCE0109960E9441
:10E30000ED7F6BE878E0CE0109960E945C7EBC014F
:10E3100082EE91E10E94077FCE0109960E94577F0D
:10E32000CE010F960E94577F62E978E0CE010F96EA
:10E330000E94F67F62EE71E1CE010F960E94727E1E
:10E34000BC01CE0109960E94ED7FBE01675F7F4F41
:10E35000C8010E942E81CE0109960E94577FCE01EE
:10E360000F960E94577F4D815E816F81788521E0F5
:10E37000CE0109960E945F7FBE01675F7F4F82EEEC
:10E3800091E10E941E7FCE0109960E94577F64EAA8
:10E3900078E0CE010F960E94F67F62EE71E1CE0129
:10E3A0000F960E94727E65EB78E00E945C7EBC0155
:10E3B000CE0109960E94ED7FBE01675F7F4FC801C5
:10E3C0000E942E81CE0109960E94577FCE010F96A2
:10E3D0000E94577F4091190C50911A0C60911B0CB0
:10E3E00070911C0C22E0CE010F960E945F7F6CEBB7
:10E3F00078E0CE0145960E94F67FBE01615F7F4FB7
:10E40000CE0145960E94727E6EEC78E00E945C7EA2
:10E41000BC01CE0109960E94ED7FBE01675F7F4F70
:10E42000C8010E942E81CE0109960E94577FCE011D
:10E4300045960E94577FCE010F960E94577F4091CC
:10E44000150C5091160C6091170C7091180C22E06D
:10E45000CE010F960E945F7F67ED78E0CE01459672
:10E460000E94F67FBE01615F7F4FCE0145960E94FC
:10E47000727E6EEC78E00E945C7EBC01CE01099653
:10E480000E94ED7FBE01675F7F4FC8010E942E8111
:10E49000CE0109960E94577FCE0145960E94577F74
:10E4A000CE010F960E94577FE6EF2E16EFEF3E0645
:10E4B0002CF463E07CE0C8010E94452068EE7AE01D
:10E4C000C8010E94452094E6C92E92E1D92E27ED7D
:10E4D000A22E22E0B22EEE24E394F12CB701CE015D
:10E4E0000F960E94447D69E078E0CE0145960E9437
:10E4F000F67FBE01615F7F4FCE0145960E94727E1E
:10E5000061E676E00E945C7EBC01CE0109960E9425
:10E51000ED7FBE01675F7F4FC8010E942E81B6016B
:10E52000CE014B960E94F67FBE01655E7F4FC8010B
:10E530000E942E8165EE78E0C8010E942681F501D7
:10E54000619171915F01660F771F660F771F6C5A9B
:10E550007D4ECE0181960E94F67FBE016F5D7F4F9A
:10E56000C8010E942E816AEE78E0C8010E942681CF
:10E57000CE0181960E94577FCE014B960E94577F15
:10E58000CE0109960E94577FCE0145960E94577F83
:10E59000CE010F960E94577FFFEFEF1AFF0A88E027
:10E5A000C80ED11CE4E0EE16F10409F097CFCE01BD
:10E5B00087960E94577F81E08093820C61EC7BE01C
:10E5C000C8010E9445201092120CAC960FB6F89428
:10E5D000DEBF0FBECDBFDF91CF911F910F91FF9096
:10E5E000EF90DF90CF90BF90AF909F908F907F90F3
:10E5F0006F905F904F903F902F90089563E07CE084
:10E60000C8010E944520DACF8F929F92AF92BF92AD
:10E61000CF92DF92EF92FF920F931F93CF93DF93EE
:10E62000CDB7DEB7A0970FB6F894DEBF0FBECDBF53
:10E6300067E174E08CE092E10E943A7D67E174E06A
:10E6400080E092E10E943A7D4BE3842E42E0942EDA
:10E650005FECC52E52E0D52E64E6A62E62E1B62E02
:10E6600075EDE72E72E0F72E01E010E0F4018191E4
:10E670009191A191B1914F01892B8A2B8B2B19F587
:10E68000F70182819381F6012081318182179307FE
:10E69000D1F0880F991FFC01E756F44FD801AA0F5B
:10E6A000BB1FA652B44F60818C910E944082F7013B
:10E6B00082819381F6019183808364E670E080E03B
:10E6C00090E00E94B383F601619171916F01CE01D8
:10E6D00045960E94447DB801CE010F960E94447D6C
:10E6E000B501CE0109960E94F67F61E676E0CE0183
:10E6F00001960E94F67FBE01675F7F4FCE010196B3
:10E700000E94727E6FEE78E00E945C7EBE01615FC7
:10E710007F4F0E94727E64E676E00E945C7EBE01BE
:10E720006B5E7F4F0E94727EBC018CE092E10E9482
:10E73000DB7ECE0101960E94577FCE0109960E9492
:10E74000577FCE010F960E94577FCE0145960E94BB
:10E75000577F0F5F1F4FF8E0AF0EB11C22E0E20EB3
:10E76000F11C0430110509F081CFE0916213F091A2
:10E770006313EE0FFF1FE353FD4F60817181CE01E4
:10E7800001960E94447D46E050E0BE016F5F7F4FDE
:10E79000CE0109960E94AF20BE01675F7F4F80E0E7
:10E7A00092E10E94DB7ECE0109960E94577FCE0146
:10E7B00001960E94577FE0916413F0916513EE0F6C
:10E7C000FF1FE353FD4F60817181CE0101960E94CE
:10E7D000447D46E050E0BE016F5F7F4FCE01099659
:10E7E0000E94AF20BE01675F7F4F80E092E10E94F0
:10E7F000DB7ECE0109960E94577FCE0101960E94D2
:10E80000577F61E676E0CE0145960E94F67F0E9432
:10E81000828628EE33E040E050E00E9432B2690187
:10E820007A0167E174E0CE014B960E94F67F67E1C2
:10E8300074E082E192E10E943A7DCE0101960E944D
:10E84000C22844E150E0BE016F5F7F4FCE010996C0
:10E850000E94AF20BE01675F7F4F82E192E10E947C
:10E860001E7FCE0109960E94577FCE0101960E941D
:10E87000577F2AE0B701A601CE0109960E94957F35
:10E8800048E050E0BE01675F7F4FCE010F960E94C7
:10E89000AF2062E172E1CE0101960E94ED7FBE01E0
:10E8A000615F7F4FCE0101960E94727EBC0186E0BF
:10E8B00092E10E94077FCE0101960E94577FCE0110
:10E8C0000F960E94577FCE0109960E94577F2AE03B
:10E8D000B701A601CE0109960E94957F62EF78E00C
:10E8E000CE0101960E94F67FBE01675F7F4FCE0189
:10E8F00001960E94727EBE016B5E7F4F0E94727E07
:10E90000BC0182E192E10E94DB7ECE0101960E9471
:10E91000577FCE0109960E94577F4091190C509164
:10E920001A0C60911B0C70911C0C21E0CE01019619
:10E930000E945F7FBE016F5F7F4FCE014B960E94AA
:10E940001E7FCE0101960E94577F69EF78E0CE01CD
:10E9500001960E94F67FBE01655E7F4FCE01019653
:10E960000E94727EBE016B5E7F4F0E94727EBC0170
:10E9700082E192E10E94DB7ECE0101960E94577FE8
:10E98000BE01655E7F4FCE0101960E94ED7F46E09D
:10E9900050E0BE016F5F7F4FCE0109960E94AF200D
:10E9A000BE01675F7F4F86E092E10E94DB7ECE0171
:10E9B00009960E94577FCE0101960E94577F409191
:10E9C000150C5091160C6091170C7091180C21E0E9
:10E9D000CE0101960E945F7FBE016F5F7F4FCE0127
:10E9E0004B960E941E7FCE0101960E94577F67E0E2
:10E9F00079E0CE0101960E94F67FBE01655E7F4FF1
:10EA0000CE0101960E94727EBE016B5E7F4F0E9416
:10EA1000727EBC0182E192E10E94DB7ECE01019612
:10EA20000E94577FBE01655E7F4FCE0101960E9416
:10EA3000ED7F46E050E0BE016F5F7F4FCE0109964B
:10EA40000E94AF20BE01675F7F4F86E092E10E9487
:10EA5000DB7ECE0109960E94577FCE0101960E946F
:10EA6000577F00916B0210916C0268E370E0C8015F
:10EA70000E94C40A9093E30B8093E20B892B49F028
:10EA800068E370E0C8010E94C40A9093E30B80938E
:10EA9000E20B8091E20B9091E30B8C3F9F4F0CF4C3
:10EAA000F0C00E94996E29833A834B835C836D8307
:10EAB0007E838F83988749815A816B817C8121E095
:10EAC000CE0109960E945F7FBE01675F7F4FCE0136
:10EAD0004B960E941E7FCE0109960E94577F61E1EE
:10EAE00079E0CE0109960E94F67FBE01655E7F4FF8
:10EAF000CE0109960E94727EBE016B5E7F4F0E941E
:10EB0000727EBC0182E192E10E94DB7ECE01099619
:10EB10000E94577FBE01655E7F4FCE0109960E941D
:10EB2000ED7F46E050E0BE01675F7F4FCE010F965C
:10EB30000E94AF20BE01615F7F4F86E092E10E949C
:10EB4000DB7ECE010F960E94577FCE0109960E9470
:10EB5000577F4D815E816F81788521E0CE010996D6
:10EB60000E945F7FBE01675F7F4FCE014B960E9480
:10EB70001E7FCE0109960E94577F6CE179E0CE019D
:10EB800009960E94F67FBE01655E7F4FCE01099611
:10EB90000E94727EBE016B5E7F4F0E94727EBC013E
:10EBA00082E192E10E94DB7ECE0109960E94577FAE
:10EBB000BE01655E7F4FCE0109960E94ED7F46E063
:10EBC00050E0BE01675F7F4FCE010F960E94AF20DD
:10EBD000BE01615F7F4F86E092E10E94DB7ECE0145
:10EBE0000F960E94577FCE0109960E94577F6CE0D6
:10EBF00072E182E192E10E94DB7E61E676E0CE0185
:10EC000001960E94F67F60E072E1CE0101960E94BB
:10EC1000727EBC0186E092E10E94DB7ECE0101960D
:10EC20000E94577F66E072E1CE0101960E94ED7F5F
:10EC3000CE0101960E94E61FCE0101960E94577FE9
:10EC40006AE070E080E090E00E94B383CE014B96D2
:10EC50000E94577FCE0145960E94577FA0960FB61F
:10EC6000F894DEBF0FBECDBFDF91CF911F910F9102
:10EC7000FF90EF90DF90CF90BF90AF909F908F90DC
:10EC8000089562E279E082E192E10E94D17E61E33F
:10EC900079E086E092E10E94D17E68E379E082E14A
:10ECA00092E10E94D17E61E379E086E092E10E94E8
:10ECB000D17E9DCFBF92CF92DF92EF92FF920F93C2
:10ECC0001F93CF93DF93CDB7DEB7C455D1090FB6ED
:10ECD000F894DEBF0FBECDBF6C018B0165965FAFB0
:10ECE0004EAF65978091130C9091140C0196909300
:10ECF000140C8093130C8091120C81113CC0BB2426
:10ED0000B394B092120C1092140C1092130C67E191
:10ED100074E0CE01895B9F4F0E94F67F67E174E04B
:10ED2000CE01835B9F4F0E94F67F50E040E068E198
:10ED300074E0C6010E945E200130110509F0A6C0F2
:10ED400067E174E082E192E10E943A7D6596EEAD62
:10ED5000FFAD65978081811124C00E940473B09239
:10ED6000820CCE01835B9F4F0E94577FCE01895B4F
:10ED70009F4F0E94577F0FB6F894DEBF0FBECDBFE6
:10ED8000CC5ADF4F0FB6F894DEBF0FBECDBFDF9178
:10ED9000CF911F910F91FF90EF90DF90CF90BF9098
:10EDA00008956596EEADFFAD65978081882309F4DF
:10EDB00067C000E210E09E012F5F3F4F40E250E04D
:10EDC000BE016F5D7F4FCE018D5A9F4F0E94937A97
:10EDD000049739F3BE016F5D7F4FCE018F5B9F4F6C
:10EDE0000E94F67FBE016F5B7F4FCE01895B9F4F14
:10EDF0000E941E7FCE018F5B9F4F0E94577FBE01F6
:10EE00006F5F7F4FCE018F5B9F4F0E94F67FBE01E9
:10EE10006F5B7F4FCE01835B9F4F0E941E7FCE01B1
:10EE20008F5B9F4F0E94577FBE01695B7F4F82E1DE
:10EE300092E10E94DB7E63968EAD9FAD6397892B36
:10EE400009F4AFCF64E676E0CE018F5B9F4F0E945E
:10EE5000F67FBE01635B7F4FCE018F5B9F4F0E94A9
:10EE6000727E61E676E00E945C7EBC0182E192E106
:10EE70000E94DB7ECE018F5B9F4F0E94577F91CF18
:10EE800062E172E18EEE91E10E94077F1092120C16
:10EE900068CF0895089508950895AF92BF92CF92D4
:10EEA000DF92EF92FF920F931F93CF93DF936C014A
:10EEB0007B018B01040F151FEB015E01AE18BF082B
:10EEC000C017D10759F06991D601ED91FC910190DD
:10EED000F081E02DC6011995892B79F7C501DF91E5
:10EEE000CF911F910F91FF90EF90DF90CF90BF9047
:10EEF000AF900895FC01538D448D252F30E0842F71
:10EF000090E0821B930B541710F0CF960895019751
:10EF10000895FC01918D828D981761F0A28DAE0F3E
:10EF2000BF2FB11D5D968C91928D9F5F9F73928FC5
:10EF300090E008958FEF9FEF0895FC01918D828DF1
:10EF4000981731F0828DE80FF11D858D90E00895BE
:10EF50008FEF9FEF0895FC01918D228D892F90E016
:10EF6000805C9F4F821B91098F739927089588EBCE
:10EF70009EE00E94AB7721E0892B09F420E0822FEC
:10EF8000089585E59FE00E94AB7721E0892B09F485
:10EF900020E0822F0895FC01A48DA80FB92FB11D88
:10EFA000A35ABF4F2C91848D90E001968F739927BF
:10EFB000848FA689B7892C93A089B1898C9183709D
:10EFC00080648C93938D848D981306C00288F38996
:10EFD000E02D80818F7D80830895EF92FF920F93C3
:10EFE0001F93CF93DF93EC0181E0888F9B8D8C8DF5
:10EFF00098131AC0E889F989808185FF15C09FB7E9
:10F00000F894EE89FF896083E889F98980818370AB
:10F01000806480839FBF81E090E0DF91CF911F915A
:10F020000F91FF90EF900895F62E0B8D10E00F5F7B
:10F030001F4F0F731127E02E8C8D8E110CC00FB651
:10F0400007FCFACFE889F989808185FFF5CFCE01E9
:10F050000E94CB77F1CFEB8DEC0FFD2FF11DE35A22
:10F06000FF4FF0829FB7F8940B8FEA89FB8980816C
:10F070008062CFCFCF93DF93EC01888D8823B9F0E6
:10F08000AA89BB89E889F9898C9185FD03C08081B3
:10F0900086FD0DC00FB607FCF7CF8C9185FFF2CF30
:10F0A000808185FFEDCFCE010E94CB77E9CFDF9144
:10F0B000CF91089580E090E0892B29F00E94C177DC
:10F0C00081110E94000080E090E0892B49F080E0EF
:10F0D00090E0892B29F00E94000081110E9400001D
:10F0E00080E090E0892B49F080E090E0892B29F0C6
:10F0F0000E94000081110E94000080E090E0892BB6
:10F1000029F00E94B77781110C9400000895815076
:10F11000823108F05AC0E82FF0E08827ED56F74812
:10F120008F4F0C94D4B3B378B778A578AB78AF7819
:10F13000E578BA78C078C478CA78CE78D278D878AA
:10F14000DC78E578E078E678EA78809180008F775F
:10F15000809380000895809180008F7DF9CF809109
:10F160008000877FF5CF84B58F7784BD089584B5FF
:10F170008F7DFBCF8091B0008F778093B000089592
:10F180008091B0008F7DF9CF809190008F77809330
:10F1900090000895809190008F7DF9CF809190002C
:10F1A000877FF5CF8091A0008F778093A00008958E
:10F1B0008091A0008F7DF9CF8091A000877FF5CF4F
:10F1C000809120018F778093200108958091200104
:10F1D0008F7DF9CF80912001877FF5CFCF93DF938B
:10F1E000282F30E0F901EE5BF34F8491F901ED52E5
:10F1F000F34FD491F901E75EF24FC491CC23A1F013
:10F2000081110E948778EC2FF0E0EE0FFF1FE85D80
:10F21000F34FA591B491EC91ED2381E090E009F4D6
:10F2200080E0DF91CF91089580E090E0FACF2091C7
:10F230003114260F3327331F21323105ECF420918E
:10F24000AD0EFC0190E080E0243069F082E008958A
:10F25000A09131142191AC014F5E5B4EA40FB52FEC
:10F26000B11D2C930196861798F380913114680F85
:10F270006093311480E0089581E00895E091760C68
:10F280008091750CE81730F4F0E0EB51F44F808179
:10F2900090E008958FEF9FEF08959091760C809104
:10F2A000750C2FEF3FEF981748F4E92FF0E0EB5182
:10F2B000F44F208130E09F5F9093760CC901089550
:10F2C0008091750C9091760C891B990B0895CF92C3
:10F2D000DF92EF92FF920F931F93CF93DF937C0106
:10F2E000CB018A012091B30E222389F0EB016B013F
:10F2F000C40ED51ECC15DD0569F06991D701ED91DD
:10F30000FC910190F081E02DC7011995F3CF642F96
:10F310000E941779C801DF91CF911F910F91FF9043
:10F32000EF90DF90CF900895CF93DF931F92CDB7EA
:10F33000DEB769832091B30E2223F9F02091B60E37
:10F34000203258F021E030E0FC013383228390E04A
:10F3500080E00F90DF91CF9108958091B40EE82F57
:10F36000F0E0EA54FA4E998190838F5F8093B40E57
:10F370008093B60E81E090E0ECCF61E0CE01019683
:10F380000E941779F7CF0E94FDB50F931F93CF937B
:10F39000DF93EC0188819981009759F02A813B81A4
:10F3A0002617370730F081E0DF91CF911F910F9141
:10F3B00008958B016F5F7F4F0E941CB5009759F035
:10F3C000998388831B830A832C813D81232B59F7E2
:10F3D000FC011082E8CF80E0E7CFEF92FF920F931D
:10F3E0001F93CF93DF936115710541F480E0DF91A6
:10F3F000CF911F910F91FF90EF9008954115510506
:10F40000B1F07B01EC010C811D81040F151FB801C7
:10F410000E94C579882351F3288139818C819D818F
:10F42000B701820F931F0E944DB61D830C8381E0AC
:10F43000DECFCF93DF93EC0188819981009711F0A3
:10F440000E9493B4198218821D821C821B821A8228
:10F45000DF91CF910895EF92FF920F931F93CF9377
:10F46000DF93EC017B018A01BA010E94C579811109
:10F470000BC0CE010E94197ACE01DF91CF911F916E
:10F480000F91FF90EF9008951D830C83B701888141
:10F4900099810E944DB6F0CF8CBD9DBD0895CF934C
:10F4A000DF93EC019A01AB01E889F98982E080835E
:10F4B000211581EE38074105510581F160E079E0C1
:10F4C0008DE390E00E9432B2215031094109510987
:10F4D0005695479537952795EC85FD851082EE85E5
:10F4E000FF852083188EEC89FD8986E08083EA8978
:10F4F000FB89808180618083EA89FB8980818860C3
:10F500008083EA89FB89808180688083EA89FB891E
:10F5100080818F7D8083DF91CF910895E889F9897B
:10F52000108220E1D9CF2F923F924F925F926F923B
:10F530007F928F929F92AF92BF92CF92DF92EF9283
:10F54000FF920F931F93CF93DF9300D0CDB7DEB719
:10F550001C013B014A0129015801FC01C080D180F6
:10F5600070E060E0C3010E9432B6A80170E060E084
:10F57000C2010E9432B6F601808110E000E08111E4
:10F5800062C004E010E004C07601F101F182E08283
:10F59000C8010F900F900F90DF91CF911F910F91A5
:10F5A000FF90EF90DF90CF90BF90AF909F908F90A3
:10F5B0007F906F905F904F903F902F9008956B32A7
:10F5C00009F482C06D3309F04EC081818823E9F2CD
:10F5D000F7018FEFE81AF80A6081653209F452C02A
:10F5E0000CF048C0662309F456C082E0A816B104A6
:10F5F0000CF061C0012B09F46BC003E010E0E8CF10
:10F6000081818983882309F282818A83760181112D
:10F6100004C0F2E0EF0EF11CB8CF83E0E80EF11C5D
:10F620001B8240E150E070E060E0CE0101960E9454
:10F63000ABA819C0F3016083F1E08F1A9108C301F0
:10F6400001963C0167017601FFEFEF1AFF0AF60110
:10F650006081663209F499CF0CF0B1CF662309F4CA
:10F6600093CF653269F2F2E08F1691041CF701E046
:10F6700010E0E8CF663209F488CF6B3209F0B5CFDD
:10F6800060E2B3CF81818983882301F182818A83FB
:10F69000811103C032967F0178CF7F0193E0E90E9C
:10F6A000F11C1B8240E150E070E060E0CE01019669
:10F6B0000E94ABA89ACFF2016083F1E0AF1AB108C3
:10F6C000C20101962C0184CF60E2CDCFF701E3CFD8
:10F6D00002E010E07DCF0F931F93CF93DF9341158E
:10F6E000510541F0FC01048115810115110539F422
:10F6F000FB011082DF91CF911F910F91089541502E
:10F7000051094017510708F48A01EB01FC0160819F
:10F710007181A801CE010E9462B6C00FD11F18826C
:10F72000E9CF20E3FC0120833296862F82958F70EB
:10F730006F706A3030F4605D6293682F8111F5CF8D
:10F740000895695CF9CF5F926F927F928F929F923A
:10F75000AF92BF92CF92DF92EF92FF920F931F93DF
:10F76000CF93DF93CDB7DEB7C754D1090FB6F89466
:10F77000DEBF0FBECDBF5C013B0119A218A28EE611
:10F7800093E09F8F8E8F1BA21C821B829A8389839A
:10F790001E8210E000E06E018EE1C80ED11C88E2EE
:10F7A000E82E80E1F82EF501E00FF11F80818F3205
:10F7B00011F40F5F1F4FD501A00FB11FFE01FB9683
:10F7C00090E080E04F012D912F3249F0222339F053
:10F7D0000F5F1F4F019621938C309105A1F7880D83
:10F7E000991DFC011082F501E00FF11F80818F321D
:10F7F00011F40F5F1F4FF501E00FF11F508041E042
:10F80000511040E030E020E0B401C701F301199548
:10F81000811121C0F8E2EF16F0E1FF06C1F480E0AB
:10F82000C95BDF4F0FB6F894DEBF0FBECDBFDF91CF
:10F83000CF911F910F91FF90EF90DF90CF90BF90ED
:10F84000AF909F908F907F906F905F900895C701C9
:10F850000E94BD0DE4CF552091F021E0A401B70135
:10F86000C6010E94C30E982E88E2E81680E1F806D1
:10F8700081F0C7010E94BD0D911010C0D0CF98E259
:10F88000E91690E1F90619F0C7010E94BD0D81E06B
:10F89000C7CF992021F2FE0131967F019E2D8F2D39
:10F8A0007601C92ED82E7FCF8F929F92AF92BF92B2
:10F8B000CF92DF92EF92FF920F931F93CF93DF933C
:10F8C000CDB7DEB760970FB6F894DEBF0FBECDBFE1
:10F8D0007C0190917A0C992351F108E0933309F45B
:10F8E00004E06B0180E591E00E944C7A9E012F5F5D
:10F8F0003F4F5901490110E0812F0E947A14F40111
:10F9000081934F018823D9F01F5F0113F5CF00E0E9
:10F91000F50181915F018D3161F0883151F08A519B
:10F92000823038F00F5F1013F3CF0E94F51518E006
:10F930008AC060E170E0802F0E94D814102FA12EA1
:10F94000B12CF501EE0FFF1FEB59F34F118210821E
:10F9500083EE93E00197F1F742E870E060E0812FD9
:10F960000E94BB144FEF62E070E0812F0E94BB1435
:10F97000B601C114D10491F480918E0290918F024E
:10F9800001968115F0EC9F0708F471C090938F02E7
:10F9900080938E0260918E0270918F02812F0E945F
:10F9A000A51486E0E3E2F3E0DE01199601900D92E2
:10F9B0008A95E1F7F70183818F778C8784818D8722
:10F9C00085818E87A7014E5F5F4F24E030E06CE0B9
:10F9D00070E0812F0E947E14B601812F0E948F1447
:10F9E00026E030E0AE01475F5F4F66E070E0812FB8
:10F9F0000E947E1461E070E0812F0E94D81427E0FD
:10FA00002A9DC0012B9D900D11249C01235D334F35
:10FA10007901F9011182108222E030E0AE01415FEC
:10FA20005F4F68E270E0812F0E94E8148F8598890B
:10FA3000982789279827F701938382831682158256
:10FA400014820E94F515812F60960FB6F894DEBFE0
:10FA50000FBECDBFDF91CF911F910F91FF90EF901F
:10FA6000DF90CF90BF90AF909F908F90089580E0EF
:10FA700090EC8CCFFB0101900020E9F73197AF01AA
:10FA8000461B570B0C942B7A0F931F93CF93DF9346
:10FA9000CDB7DEB762970FB6F894DEBF0FBECDBF0D
:10FAA0008C01CB01F801118210821382128215821F
:10FAB00014824AE0BE016F5F7F4F0E94F2A9BE012F
:10FAC0006F5F7F4FC8010E943A7D62960FB6F8942F
:10FAD000DEBF0FBECDBFDF91CF911F910F91089573
:10FAE0000F931F93CF93DF93CDB7DEB7A1970FB6D8
:10FAF000F894DEBF0FBECDBF8C01CB01BA01F80177
:10FB00001182108213821282158214822AE0AE01C1
:10FB10004F5F5F4F0E942CAABE016F5F7F4FC801ED
:10FB20000E943A7DA1960FB6F894DEBF0FBECDBFFE
:10FB3000DF91CF911F910F910895FC0180819181F8
:10FB4000009711F00C94AEA960E070E0CB0108952D
:10FB5000FC0180819181009711F00C94B2A960E0C2
:10FB600070E0CB010895AF92BF92CF92DF92EF92F7
:10FB7000FF920F931F93CF93DF93DC01CD90DC9026
:10FB80001197C114D10439F01496CD91DC918C01F8
:10FB90007601209761F4DF91CF911F910F91FF9033
:10FBA000EF90DF90CF90BF90AF900895750157010F
:10FBB000BFEFAB1ABB0AF7018081082E000C990B2E
:10FBC0000E94D9A9892B91F72197CC0DDD1D888141
:10FBD000082E000C990B0E94D9A9892B29F0CE156B
:10FBE000DF0510F02197F3CFAE014F5F5F4F4E1945
:10FBF0005F09D80115965C934E931497CE14DF04D9
:10FC000020F4B701C6010E9417B6D801ED91FC910E
:10FC1000119714968D919C91E80FF91F1082BBCF1C
:10FC2000FC01248135816217730748F4808191813A
:10FC3000009729F0860F971FFC018081089580E0CE
:10FC40000895FC0124813581FB01448155812417ED
:10FC50003507A0F0FC0180819181009779F0FB01CC
:10FC6000608171816115710549F0241B350B820F8C
:10FC7000931F0E9444B621E0892B09F020E0822FD7
:10FC80000895FB0144815581FC01248135812417AD
:10FC9000350778F080819181009759F0FB016081F0
:10FCA00071816115710529F00E9454B621E0892BFC
:10FCB00009F020E0822F0895CF93DF93EC01FB0140
:10FCC00001900020E9F73197AF01461B570B0E94C6
:10FCD000ED79811103C0CE010E94197ACE01DF9126
:10FCE000CF910895CF93DF93EC01FB0144815581BF
:10FCF000608171810E94ED79811103C0CE010E9463
:10FD0000197ACE01DF91CF910895EF92FF920F9370
:10FD10001F93CF93DF93EC017B01CB010E94E9A9F4
:10FD20000097A9F00C811D81080F191FB801CE01A1
:10FD30000E94C579882361F0288139818C819D8159
:10FD4000B701820F931F0E94E2A91D830C8381E0FB
:10FD5000DF91CF911F910F91FF90EF900895CF9376
:10FD6000DF931F921F92CDB7DEB769831A8241E0FD
:10FD700050E0BE016F5F7F4F0E94ED790F900F90B2
:10FD8000DF91CF910895CF93DF93EC010E94AF7E76
:10FD9000811103C0CE010E94197ACE01DF91CF916B
:10FDA0000895FB0101900020E9F73197AF01461B50
:10FDB000570B0C94ED79FB01448155816081718171
:10FDC0000C94ED79EF92FF920F931F93CF93DF93F3
:10FDD000EC018B01CB010E94E9A97C01BC01CE01A1
:10FDE0000E94C57981110BC0CE010E94197ACE0103
:10FDF000DF91CF911F910F91FF90EF900895FD82B9
:10FE0000EC82B801888199810E94E2A9F0CFCF935A
:10FE1000DF93EC01FB018617970749F06081718140
:10FE20006115710541F0448155810E942B7ACE0104
:10FE3000DF91CF9108950E94197AF9CF0F931F9304
:10FE4000CF93DF938C01EB01FC01808191810097BE
:10FE5000E1F06881798161157105A9F042815381D2
:10FE60002C813D814217530770F00E944DB68C8162
:10FE70009D81F801958384831D821C82DF91CF913F
:10FE80001F910F9108950E9493B488819981F80180
:10FE9000918380838A819B81938382838C819D81DE
:10FEA00095838483198218821B821A82E5CFFC0114
:10FEB00080819181009711F00C9493B40895EF9292
:10FEC000FF920F931F93CF93DF93CDB7DEB7A19728
:10FED0000FB6F894DEBF0FBECDBF7C01CB01BA01D7
:10FEE000F70111821082138212821582148242E07D
:10FEF000420F8E010F5F1F4F0E94E9A7009789F004
:10FF0000BC01C7010E943A7DA1960FB6F894DEBFEE
:10FF10000FBECDBFDF91CF911F910F91FF90EF905A
:10FF20000895C7010E94197AEFCF0F931F93CF93C3
:10FF3000DF93CDB7DEB7A2970FB6F894DEBF0FBE42
:10FF4000CDBF8C01CB01BA01F8011182108213825E
:10FF500012821582148230E0AE014F5F5F4F0E9423
:10FF6000FDA9BE016F5F7F4FC8010E943A7DA29636
:10FF70000FB6F894DEBF0FBECDBFDF91CF911F91BA
:10FF80000F910895CF93DF931F921F92CDB7DEB7E5
:10FF9000FC011182108213821282158214826983FD
:10FFA0001A82BE016F5F7F4F0E943A7D0F900F90C3
:10FFB000DF91CF910895FC01118210821382128289
:10FFC000158214820C941E7FFC0111821082138210
:10FFD0001282158214820C94E27EFC01118210823E
:10FFE00013821282158214820C94077FFC01118205
:10FFF000108213821282158214826115710551F0EC
:020000021000EC
:10000000FB0101900020E9F73197AF01461B570B28
:100010000C942B7A0895AF92BF92CF92DF92EF9219
:10002000FF920F931F93CF93DF936C015B017A01D3
:1000300089012417350720F48F2D7901042F182FFB
:1000400067E174E0C6010E94F67FD5011496CD9158
:10005000DC91EC16FD06E0F40C171D0708F4E8012E
:10006000D501ED91FC911197EC0FFD1F10811082CD
:100070006D917C916E0D7F1DC60161157105A1F01A
:100080000E943A7DF50180819181C80FD91F1883A4
:10009000C601DF91CF911F910F91FF90EF90DF90FC
:1000A000CF90BF90AF9008950E94197AEBCFFB01DB
:1000B00001900020E9F73197AF01461B570BDC0197
:1000C000ED91FC910280F381E02D19948F929F9223
:1000D000AF92BF92EF92FF920F931F93CF93DF9354
:1000E000CDB7DEB7A1970FB6F894DEBF0FBECDBF78
:1000F0007C01FA01CB0119A2223008F42AE08E011A
:100100000F5D1F4F822E912CB12CA12CBF01A50198
:1001100094010E9432B2F901CA016A300CF5605DA7
:10012000D8016E938D01232B242B252B79F790E09A
:1001300080E0109721F0BD01C7010E945780A19671
:100140000FB6F894DEBF0FBECDBFDF91CF911F91E8
:100150000F91FF90EF90BF90AF909F908F90089578
:10016000695CDECF8F929F92AF92BF92CF92DF9267
:10017000EF92FF920F931F93CF93DF937C01EB01DC
:100180006C0182E0C80ED11C4701E5E08E0E911C87
:1001900010E000E0F60141916F0150E070E060E096
:1001A0002AE0CE010E9466805C01E881F98101901D
:1001B000F081E02D6EE2CE0119958A0D9B1D080F8E
:1001C000191FC814D90431F7F701458150E070E0D8
:1001D00060E02AE0CE010E946680800F911FDF91CF
:1001E000CF911F910F91FF90EF90DF90CF90BF9034
:1001F000AF909F908F9008950F931F93CF93DF93AD
:10020000EC01CB01BE010E94B2808C016BEA79E067
:10021000CE010E945780800F911FDF91CF911F91D7
:100220000F9108950F931F93CF93DF93EC010E94DA
:1002300057808C016BEA79E0CE010E945780800FD5
:10024000911FDF91CF911F910F9108956115710555
:1002500011F00C94578090E080E00895DB01149633
:100260004D915C9115976D917C91DC01ED91FC9124
:100270000280F381E02D19940F931F93CF93DF93A6
:10028000EC010E942E818C016BEA79E0CE010E9484
:100290005780800F911FDF91CF911F910F9108958B
:1002A000EF92FF920F931F93CF93DF938C017B010B
:1002B000D0E0C0E0F701EC0FFD1F6491662361F010
:1002C000D801ED91FC910190F081E02DC8011995C4
:1002D000892B11F02196EECFCE01DF91CF911F91A6
:1002E0000F91FF90EF900895DC018CE094E08D93E6
:1002F0009D9384E0FB0101900D928A95E1F70895AA
:100300001F920F920FB60F9211240BB60F922F93DC
:100310003F934F935F936F937F938F939F93AF938D
:10032000BF93EF93FF9388EB9EE00E94CB77FF9102
:10033000EF91BF91AF919F918F917F916F915F915D
:100340004F913F912F910F900BBE0F900FBE0F90CA
:100350001F9018951F920F920FB60F9211240BB693
:100360000F922F938F939F93EF93FF93E091C80E7B
:10037000F091C90E8081E091CE0EF091CF0E82FDFA
:100380001DC090818091D10E8F5F8F732091D20E0E
:10039000821741F0E091D10EF0E0E854F14F958FD3
:1003A0008093D10EFF91EF919F918F912F910F909C
:1003B0000BBE0F900FBE0F901F9018958081F2CF4B
:1003C0001F920F920FB60F9211240BB60F922F931C
:1003D0003F934F935F936F937F938F939F93AF93CD
:1003E000BF93EF93FF9385E59FE00E94CB77FF914A
:1003F000EF91BF91AF919F918F917F916F915F919D
:100400004F913F912F910F900BBE0F900FBE0F9009
:100410001F9018951F920F920FB60F9211240BB6D2
:100420000F922F938F939F93EF93FF93E091650F1C
:10043000F091660F8081E0916B0FF0916C0F82FD5F
:100440001DC0908180916E0F8F5F8F7320916F0F11
:10045000821741F0E0916E0FF0E0EB5AF04F958F6C
:1004600080936E0FFF91EF919F918F912F910F903D
:100470000BBE0F900FBE0F901F9018958081F2CF8A
:100480001F93CF93DF93282F30E0F901EE5BF34FFA
:100490008491F901ED52F34FD491F901E75EF24FE7
:1004A000C491CC23A9F0162F81110E948778EC2FDC
:1004B000F0E0EE0FFF1FE156F34FA591B4918FB717
:1004C000F894EC91111108C0D095DE23DC938FBF16
:1004D000DF91CF911F910895DE2BF8CFAF92BF929D
:1004E000CF92DF92EF92FF920F931F93CF93DF9300
:1004F0006B017A01EC01C95CDA4E28813CE0389F3F
:100500008001399F100D1124A0900616B12C27FFF1
:100510001FC0FB011182108288818F5F88838881D0
:100520009801280F311D87FD3A95F6012A153B05E4
:100530001CF488818C30C4F18081918104968034D0
:100540009C4908F473C0F60180819181049670C0C3
:1005500088819801280F311D87FD3A952A153B05A2
:10056000DCF68881A801480F511D87FD5A95FA01D4
:10057000EE0FFF1FE40FF51FE35BFF4E808186FF48
:10058000CBCF8881F801E80FF11D87FDFA95CF01E7
:10059000EE0FFF1FE80FF91FE35BFF4E808160E065
:1005A0008F730E944082B8CF808191812881A801F9
:1005B000420F511D27FD5A959A01FA01EE0FFF1FB8
:1005C000E20FF31FE35BFF4E21813281820F931F05
:1005D000F7019183808388819801280F311D87FD61
:1005E0003A95F901EE0FFF1FE20FF31FE35BFF4E99
:1005F000808186FF22C08881080F111D87FD1A9512
:10060000F801EE0FFF1FE00FF11FE35BFF4E80814B
:1006100061E08F73DF91CF911F910F91FF90EF9069
:10062000DF90CF90BF90AF900C94408280E49CE923
:10063000F701918380838FEF8883DF91CF911F91A2
:100640000F91FF90EF90DF90CF90BF90AF90089503
:100650001092AD0E81E08093AC0E1092870E61E097
:1006600084E10E94408261E085E10E944082E9EBE2
:10067000F0E080818E7F808380818D7F808388E41D
:100680008093B80085E48093BC0008951092760CA6
:100690001092750C1092B40E1092B60E0E94288320
:1006A0008AE497E790934915809348158BE497E780
:1006B00090934715809346150895CF93DF9390E06C
:1006C000FC01ED52F34F2491875E924FFC0184911F
:1006D0008823D1F090E0880F991FFC01E754F34F75
:1006E000A591B491FC01E156F34FC591D4916111EC
:1006F0000EC09FB7F8948C91E22FE0958E238C93D7
:100700002881E223E8839FBFDF91CF9108958FB7BF
:10071000F894EC91E22BEC938FBFF6CF3FB7F894AF
:100720008091401590914115A0914215B0914315CB
:1007300026B5A89B05C02F3F19F00196A11DB11D3C
:100740003FBFBA2FA92F982F8827BC01CD01620F78
:10075000711D811D911D42E0660F771F881F991F33
:100760004A95D1F708958F929F92AF92BF92CF9200
:10077000DF92EF92FF926B017C010E948E834B010E
:100780005C01C114D104E104F104B9F00E948E832C
:10079000681979098A099B09683E734081059105AA
:1007A00080F321E0C21AD108E108F10888EE880E32
:1007B00083E0981EA11CB11CE4CFFF90EF90DF9066
:1007C000CF90BF90AF909F908F900895AF92BF92BF
:1007D000CF92DF92EF92FF920F931F93CF93DF930D
:1007E000C82FD62F10927E1310927F131092801371
:1007F000109281131092821361E00E945D8360E089
:100800008C2F0E9440826D2F70E090E080E00E946B
:10081000B38360E08C2F0E945D838BE990E00197A9
:10082000F1F700E911E08C2F0E94EE78892B81F41A
:1008300001501109C1F78EEF9FEFDF91CF911F910A
:100840000F91FF90EF90DF90CF90BF90AF90089501
:1008500000E911E08C2F0E94EE78019721F40150FD
:100860001109C1F7E8CF18E2D0E800E090E9E92EDD
:10087000FF24F3948C2F0E94EE78892B29F481E0D9
:10088000E81AF108B9F7D7CF0E948E836B017C017B
:1008900080E9A82EBB24B3948C2F0E94EE78019798
:1008A00029F481E0A81AB108B9F7C5CF0E948E8358
:1008B0006C197D098E099F096932710581059105C1
:1008C00038F0E02FF0E0EA58FC4E80858D2B8087D1
:1008D000D69511F40F5FD0E8115041F690E080E01A
:1008E000ACCF0F931F93CF93DF9300D000D01F9214
:1008F0001F92CDB7DEB78091AC1581112AC010923E
:1009000094151092931588EE93E0A0E0B0E08093E8
:10091000951590939615A0939715B093981586E921
:1009200093E090939215809391158CE094E09093CE
:10093000A01580939F151092A1151092A2151092E8
:10094000A3151092A41588E08093A91581E08093E7
:10095000AC158EE495E190937D0C80937C0C809196
:100960004D1581119DC060E372E080E090E00E942F
:10097000B3831FB7F89480914C15811127C0EEE422
:10098000FDE08491E8E0FDE09491E82FF0E0EE0FC7
:10099000FF1FE754F34FA591B491EC91E92321F4A3
:1009A00061E085E30E94408261E085E30E945D830F
:1009B0008CB580618CBD8CB580648CBD61E084E3B6
:1009C0000E945D8361E083E30E945D8380914C150A
:1009D0008F5F80934C151FBFE3E2FDE0E491F0E0F0
:1009E000EE0FFF1FE156F34F859194919093790C90
:1009F0008093780CEDEDFCE0E491E093770C61E0FE
:100A00008AE00E945D830E94DE1280E591E00E94F0
:100A10004C7A84E380937A0C80E80E9467140E94E9
:100A20005114882309F4F5C088E00E9467140E94DD
:100A30003E14883009F0EDC080E10E9467140E94E6
:100A40003E14803109F0E5C080E00E9467140E94E6
:100A50003E14182F8111DDC041E050E0BE016F5FF0
:100A60007F4F8FE190E00E94E8128981833009F086
:100A7000D0C080E480937B0C42E06EE170E0812F77
:100A80000E94BB1442E06FE170E0812F0E94BB1412
:100A90001F5F183089F70E94F51581E080934D158E
:100AA00080E591E00E944C7A46E050E060E972E017
:100AB00089E090E00E9490138CE094E09A8389830F
:100AC0001B821C821D821E82CE0103960E94EE159F
:100AD0000E94F51580917C0C90917D0CDC01929622
:100AE0001D921D921D921C929597FC0116A217A2B1
:100AF00010A611A69A961D921D921D921C929D976A
:100B000040E65AEE60E070E046AB57AB60AF71AFC5
:100B100040EA5FE060E070E0DA964D935D936D939C
:100B20007C93DD973E9624E1DF011D922A95E9F73B
:100B300026E0E0E9F2E0DC01189601900D922A959A
:100B4000E1F7FC01EE5BFF4F10820E94412B8C010C
:100B5000019709F0CBC080E591E00E944C7A60914A
:100B60007C0C70917D0C625F7F4FCE0101960E94DC
:100B70007481CE0103960E94EE1560917C0C7091F9
:100B80007D0C6A5E7F4FCE0101960E94748144E025
:100B900050E0BE016D5F7F4F81E090E00E949013B6
:100BA00060917C0C70917D0C6E5E7F4FCE01019642
:100BB0000E94748144E050E0BE016D5F7F4F85E08C
:100BC00090E00E9490130E94F51560917C0C70914A
:100BD0007D0C625E7F4FCE0101960E9474818B81F5
:100BE0009C81AD81BE818093491090934A10A0935F
:100BF0004B10B0934C100E948E837F7380918E02B5
:100C000090918F026827792770938F0260938E02EC
:100C10006DC087E380937A0C80E80E9467140E947D
:100C20005114882329F188E00E9467140E943E1421
:100C30008830F1F480E10E9467140E943E14182F5E
:100C40008031B1F480E00E9467140E943E1481114B
:100C50000FC041E050E0BE016F5F7F4F89E390E03D
:100C60000E94E8128981843019F410937B0C13CF11
:100C700083E380937A0C80E80E9467140E945114E9
:100C8000882371F180E10E9467140E943E14803134
:100C900039F582E10E9467140E943E14823101F509
:100CA00080E00E9467140E943E14811119C084E004
:100CB00080937B0C15E5188741E050E0BE01685F2A
:100CC0007F4F8BE190E00E9490131F8341E050E042
:100CD000BE01695F7F4F8AE190E00E949013DBCEF6
:100CE00010927A0C0E94F51510E000E0C8012896D9
:100CF0000FB6F894DEBF0FBECDBFDF91CF911F912D
:100D00000F9108952FB7F89460913C1570913D159F
:100D100080913E1590913F152FBF0895CF92DF929D
:100D2000EF92FF92CF93DF938091F910883050F0CB
:100D3000CFEFDFEFCE01DF91CF91FF90EF90DF900B
:100D4000CF900895E0911E11E11142C00E94828669
:100D50006B017C0128EEC20E23E0D21EE11CF11CC7
:100D60008DEE90E10E945B1A882311F3809154115B
:100D7000882331F080911F1190912011892BC1F2AD
:100D80008DEE90E10E94BE18EC01CF3FDC0771F0C0
:100D900080915411882371F280911F11909120113C
:100DA00001979093201180931F11C4CF0E948286D7
:100DB000C616D706E806F90698F610921E118DEEB3
:100DC00090E10E94B61A8DEE90E10E947D1AB2CF9A
:100DD000E150E0931E11F0E0ED51FF4EC38DD0E0E5
:100DE000A9CF0F931F93CF93DF93EC018C01F801F0
:100DF00081918F018823A1F10E948E86F8012291B2
:100E0000022E000C330B8217930789F38F3F98074C
:100E100081F0A0911E1191E09A0F90931E11B0E005
:100E2000AD51BF4E5B968C93903219F48FE1809355
:100E30001E112FE1EC17FD07C9F092919F3FD1F3EE
:100E4000A0911E1181E08A0F80931E11B0E0AD5178
:100E5000BF4E5B969C93803269F720931E11EACFB8
:100E600081E0DF91CF911F910F91089580E0F9CF3C
:100E70000F931F93CF93DF93EC010E9482868B0127
:100E80000E94D0108F3F69F00E948286601B710B18
:100E90006C177D07A8F380E0DF91CF911F910F9130
:100EA000089581E0F9CF4F925F926F927F928F9277
:100EB0009F92AF92BF92CF92DF92EF92FF920F93E9
:100EC0001F93CF93DF93CDB7DEB763970FB6F89438
:100ED000DEBF0FBECDBF7C016B013A01FB0120E0FC
:100EE00090E080E06AE03191332309F461C040ED85
:100EF000430F4A3008F04DC0689FA001699F500D14
:100F00001124CA01C097830F911D37FD9A958F3F19
:100F1000910549F340F3F701428153816481758162
:100F20008091FC159091FD15A091FE15B091FF15D3
:100F3000481759076A077B0709F40DC28701085F44
:100F40001F4F0E9482866F7077277C5FC8010E94C6
:100F50000E1C813009F004C28CE094E09A838983EE
:100F6000F70182819381A481B5818B839C83AD83BA
:100F7000BE8345E350E0BE016F5F7F4FC8010E9412
:100F8000971C892BA9F5D12CC12CC8010E943A19B4
:100F900017C03E3209F0BFCF233009F4BCCFD301D4
:100FA000A20FB11D12968C932F5F90E080E09BCF33
:100FB000233009F0B0CFF3018583CC24C394D12C26
:100FC000C60163960FB6F894DEBF0FBECDBFDF91AA
:100FD000CF911F910F91FF90EF90DF90CF90BF9036
:100FE000AF909F908F907F906F905F904F900895FB
:100FF0000E948286F7017783668342E050E0B70162
:101000006A5F7F4FC8010E942C1C81E090E09A83A8
:10101000898342E050E0BE016F5F7F4FC8010E94AC
:101020002C1C80E091E09A83898342E050E0BE016D
:101030006F5F7F4FC8010E942C1C1A82198242E008
:1010400050E0BE016F5F7F4FC8010E942C1C42E040
:1010500050E0BE016F5F7F4FC8010E942C1C42E030
:1010600050E0BE016F5F7F4FC8010E942C1C5601EB
:10107000F6018081882301F16501F60181912F013C
:10108000882311F08E32B1F446018A189B08181497
:10109000190474F48D8641E050E0BE01635F7F4F18
:1010A000C8010E942C1CA401B501C8010E942C1C7F
:1010B0005201DECF6201E1CF1D8641E050E0BE016A
:1010C000635F7F4FC8010E942C1CC12CDD24D39488
:1010D000DA82C98242E050E0BE016F5F7F4FC801F3
:1010E0000E942C1CDA82C98242E050E0BE016F5F90
:1010F0007F4FC8010E942C1CC8010E94661C892BCE
:1011000009F441CFF3E0AF2EB12C230122E0420ECF
:10111000511CD4C0F7014281538164817581808D57
:10112000918DA28DB38D481759076A077B0709F087
:1011300008C1848D958DC59709F003C181A192A145
:101140005DEFC52EDD24DA940C970CF4ADC04CE0B5
:1011500050E0BE016F5F7F4FC8010E9419188B815C
:101160009C819827892798279A8B898BF70146813C
:10117000578129813A814217530709F0E7C097FF49
:10118000E5C08F7092703BEFC32EDD24DA94892B7B
:1011900009F08AC06F8078847624672476242AEF49
:1011A000C22EDD24DA946114710409F47DC0D12CBF
:1011B000C12C8D819E81982789279827C816D9062A
:1011C000F8F441E050E0BE01635F7F4FC8010E9428
:1011D00019184D85442331F050E070E060E0C801FB
:1011E0000E9419188D858111ECCF44E050E070E029
:1011F00060E0C8010E941918FFEFCF1ADF0AD9CFAB
:10120000912C812C41E050E0BE016D5E7F4FC80102
:101210000E9419184B89842F807C09F06CC04423EC
:1012200031F050E070E060E0C8010E9419188B892D
:101230008111E8CF42E050E0BE01615F7F4FC801FD
:101240000E94191842E050E0BE01635F7F4FC80161
:101250000E94191844E050E070E060E0C8010E946C
:10126000191842E050E0BE016F5E7F4FC8010E9436
:1012700019188F85988949895A898115914009F0F3
:1012800043C0CD84DE84DC24CD24DC2481E0C81678
:10129000D104D1F54115544009F04AC044E050E072
:1012A000B201C8010E94191821E0A21AB10809F47C
:1012B0006CCEFFEFCF16DF0609F067CE0E94828664
:1012C0003B014C01C8010E946218181619060CF463
:1012D00021CF0E94828666197709880999096938A1
:1012E00073418105910548F562E370E080E090E08C
:1012F0000E94B383E7CF41E050E070E060E0C801B6
:101300000E9419181B8A93CF54274527542770E051
:1013100060E0C8010E941918FFEF8F1A9F0A681435
:10132000790409F06FCF96EFC92EDD24DA94BCCF93
:10133000E7EFCE2EDD24DA94B7CFCC24CA94DC2C90
:10134000B3CF6EEFC62EDD24DA94AECF4CEFC42EB1
:10135000DD24DA94A9CF8EEFC82EDD24DA9430CEC6
:10136000D12CC12C2DCE1F920F920FB60F921124AB
:101370002F933F938F939F93AF93BF9380913C158F
:1013800090913D15A0913E15B0913F1530913B15C0
:1013900023E0230F2D3758F50196A11DB11D209391
:1013A0003B1580933C1590933D15A0933E15B0934B
:1013B0003F158091401590914115A0914215B09133
:1013C00043150196A11DB11D8093401590934115C1
:1013D000A0934215B0934315BF91AF919F918F9108
:1013E0003F912F910F900FBE0F901F90189526E8F8
:1013F000230F0296A11DB11DD2CF1F920F920FB6DF
:101400000F9211240BB60F922F933F934F935F933C
:101410006F937F938F939F93AF93BF93EF93FF93BC
:1014200048E251E064E271E090E080E00E946E8268
:10143000FF91EF91BF91AF919F918F917F916F91AC
:101440005F914F913F912F910F900BBE0F900FBE68
:101450000F901F9018951F920F920FB60F921124A4
:101460000BB60F922F933F934F935F936F937F939E
:101470008F939F93AF93BF93EF93FF9348EA50E00E
:1014800064EA70E083E090E00E946E82FF91EF9149
:10149000BF91AF919F918F917F916F915F914F918C
:1014A0003F912F910F900BBE0F900FBE0F901F908A
:1014B00018951F920F920FB60F9211240BB60F9230
:1014C0002F933F934F935F936F937F938F939F934C
:1014D000AF93BF93EF93FF9348E950E064E970E066
:1014E00082E090E00E946E82FF91EF91BF91AF91F8
:1014F0009F918F917F916F915F914F913F912F912C
:101500000F900BBE0F900FBE0F901F9018951F925B
:101510000F920FB60F9211240BB60F922F933F9399
:101520004F935F936F937F938F939F93AF93BF93EB
:10153000EF93FF9348E850E064E870E081E090E0CA
:101540000E946E82FF91EF91BF91AF919F918F9119
:101550007F916F915F914F913F912F910F900BBEB3
:101560000F900FBE0F901F901895609333157093D6
:1015700034158093351590933615645D7E4F8F4FEB
:101580009F4F60932F157093301580933115909372
:10159000321582E090E090932E1580932D150E94D5
:1015A00082866093291570932A1580932B1590934A
:1015B0002C150895CF92DF92EF92FF920F931F9315
:1015C0000E9482868B019C01C0902915D0902A151B
:1015D000E0902B15F0902C15609133157091341517
:1015E00080913515909136150C191D092E093F096A
:1015F000083E134021053105E0F0DC01CB010196E6
:10160000A11DB11D8093331590933415A09335150A
:10161000B0933615B701A60148515C4F6F4F7F4F0D
:101620004093291550932A1560932B1570932C1510
:10163000C7CF1F910F91FF90EF90DF90CF9008954B
:10164000CF93DF93EC010E94DA8A9E01220F331FB1
:10165000220F331FF901E352FD4F608371838283B0
:101660009383CE01880F991FFC01EB52FD4F4081FF
:1016700051811416150644F4FC01E353FD4F4081DB
:10168000518114161506ECF08B529D4F41E050E04D
:10169000FC015183408323543D4F88E097E0A0E054
:1016A000B0E0F90180839183A283B383CE010E94CD
:1016B000FA1E64EF71E080E090E0DF91CF910C942E
:1016C000B383DF91CF9108954F925F926F927F9293
:1016D0008F929F92AF92BF92CF92DF92EF92FF9242
:1016E0000F931F93CF93DF934B015C0180912515DE
:1016F00090912615A0912715B09128158815990568
:10170000AA05BB0509F4C6C08CE3C82ED12CE12C78
:10171000F12CC501A70196010E9432B26093050C1D
:10172000CA01B901A70196010E9432B26093060C6A
:10173000C501B40120E13EE040E050E00E9432B239
:10174000CA01B90128E130E040E050E00E9432B225
:101750006093070CC501B40120E831E541E050E099
:101760000E9432B269017A01CA01B9016C5F7F4FF0
:101770008F4F9F4F27E030E040E050E00E9432B2B0
:101780006F5F6093080C412C512C320140E004E65D
:1017900010E0C0E9D1E0242F30E02E54384FF90199
:1017A000E370FF273097F9F4C901B8010E94C0B374
:1017B000892B31F4C901BE010E94C0B3892B99F471
:1017C0008EE691E0A0E0B0E0480E591E6A1E7B1E36
:1017D000D301C201AA27BB27C816D906EA06FB0611
:1017E00038F04F5FD8CF8DE691E0A0E0B0E0ECCFCD
:1017F00040930B0CC90164E670E00E94C0B3EC0199
:10180000C90160E971E00E94C0B3309721F42097CC
:10181000D9F40097C9F04DE651E060E070E0441A59
:10182000550A660A770AC418D508E608F708A3E33C
:10183000B3E020E0213069F43097E9F5209711F406
:101840000097C9F54DE106C04EE651E060E070E05A
:10185000E6CF4C9150E070E060E031E0320FC4160A
:10186000D506E606F70640F0C41AD50AE60AF70AD6
:101870001196232F3C30F1F62F5F20930A0CC3946E
:10188000C092090C8092251590922615A0922715DA
:10189000B0922815DF91CF911F910F91FF90EF909B
:1018A000DF90CF90BF90AF909F908F907F906F9080
:1018B0005F904F9008954CE1CDCF0E94DA8A0E944C
:1018C000648B80910B0C90E08E54984F08950E9489
:1018D000DA8A0E94648B80910A0C90E008950E943D
:1018E000DA8A0E94648B8091090C90E008950E942E
:1018F000DA8A0E94648B8091060C90E008950E9421
:10190000DA8A0E94648B8091070C90E008951F9200
:101910000F920FB60F9211240BB60F922F933F9395
:101920004F935F936F937F938F939F93AF93BF93E7
:10193000EF93FF93809155140E94EE7820915814F4
:10194000309159142F5F3F4F3093591420935814FE
:1019500090915714953618F096E090935414909106
:101960005414943009F46EC0F8F4923031F193308D
:1019700009F44CC090915614992319F0811171C04B
:101980002F9AFF91EF91BF91AF919F918F917F918E
:101990006F915F914F913F912F910F900BBE0F90E0
:1019A0000FBE0F901F901895953009F457C09630D0
:1019B00009F791E0909324154FC08111DBCF20915E
:1019C0005814309159142436310528F410925914C2
:1019D00010925814CFCF1092241510925714E09102
:1019E000571491E09E0F90935714F0E020915814F3
:1019F00030915914EE0FFF1FE65AFB4E31832083BE
:101A0000109259141092581493E019C0813009F0C3
:101A1000B1CFE091571491E09E0F90935714F0E0EE
:101A20002091581430915914EE0FFF1FE65AFB4EC7
:101A300031832083109259141092581494E090939B
:101A4000541498CF882359F2209158143091591486
:101A50002536310508F48ECF95E0F1CF81118ACF7C
:101A6000B5CF2F988ECFCF93DF9391E09093101442
:101A70008823B9F0C091B800D091BA008091BC0021
:101A80008A7B8093BC0060E084E10E94408260E039
:101A900085E10E9440820E942883D093BA00C093BF
:101AA000B800DF91CF9108958F929F92AF92BF922D
:101AB000CF92DF92EF92FF920F931F93CF93DF931A
:101AC000D091B60ED13208F0D7C0182FC091B50E04
:101AD0000E948E836B017C018091AD0E81116BC0E1
:101AE00082E08093AD0E1093AC0E8FEF8093AB0E1F
:101AF0001092AA0ED093A90EA6EBB5E1E9E8FEE09C
:101B000080E0D81391C01092880E8091880ECC0F7F
:101B1000C82BC093880E8091870E813009F088C051
:101B20001092870E0E948E836B017C018091880E3B
:101B30008093BB008091AF0E9091B00EA091B10E3A
:101B4000B091B20E892B8A2B8B2BA1F00E948E8331
:101B50000091AF0E1091B00E2091B10E3091B20EE7
:101B60006C197D098E099F09061717072807390781
:101B700008F442C08091BC0083FDD8CF85EC8093EF
:101B8000BC000E948E836B017C018091AD0E82307F
:101B900009F450C08091AB0E8F3F09F46FC0809163
:101BA000AB0E803209F46CC08091AB0E803309F427
:101BB00069C084E026C08091AF0E9091B00EA091D4
:101BC000B10EB091B20E892B8A2B8B2B09F484CFE6
:101BD0000E948E838090AF0E9090B00EA090B10EB8
:101BE000B090B20E6C197D098E099F098616970672
:101BF000A806B90608F070CF8091AE0E0E94338D12
:101C000085E01092B40E1092B60E1092B30EDF91D2
